:100000000C94C3180C94EE180C94EE180C94EE1883
:100010000C94EE180C94EE180C94EE180C94EE1848
:100020000C94EE180C94EE180C94EE180C94EE1838
:100030000C94EE180C9470190C94EE180C94EE18A5
:100040000C94EE180C941C7C0C94EE180C94EE1886
:100050000C94EE180C94EE180C94D6840C94CF19D2
:100060000C94EE180C94E2510C94EE180C94EE18CB
:100070000C94EE180C94EE180C94EE180C94EE18E8
:100080000C94EE180C94EE180C94EE180C94EE18D8
:100090000C94EE180C94EE180C94EE180C9409972E
:1000A0000C94EE180C94EE180C94EE180C94EE18B8
:1000B0000C94EE180C94EE180C94EE180C94EE18A8
:1000C0000C94EE180C94EE180C94EE180C94EE1898
:1000D0000C94EE180C94EE180C94EE180C94EE1888
:1000E0000C94EE18084AD73B3BCE016E84BCBFFD92
:1000F000C12F3D6C74319ABD56833DDA3D00C77FF8
:1001000011BED9E4BB4C3E916BAAAABE0000008090
:100110003F05A84CCDB2D44EB93836A9020C50B91F
:10012000918688083CA6AAAA2ABE000000803F0249
:1001300000002100240027002A002D003000330099
:1001400001010000040107010A010000220025004E
:1001500028002B002E0031003400020100000501B0
:1001600008010B01000020002300260029002C00BC
:100170002F003200000100000301060109010505FE
:100180000505070508080808020202020A0A08080D
:10019000040404040101010101010101030303033B
:1001A00003030303040707070C0C0C0C0C0C0C0CCA
:1001B0000202020206060606060606060B0B0B0BDB
:1001C0000B0B0B0B01021020200808102040102000
:1001D000408002010201080402010102040810200B
:1001E0004080804020100804020180040201804009
:1001F0002010080402010804020101020408102072
:10020000408001020408102040800000090A020812
:100210000B0C0D07060304010000000000000000A5
:1002200000000000000000000000000000000000CE
:1002300000000000000011100F000000000000008E
:1002400000000000000000000000000000000000AE
:100250004D383420582059205A2045006563686F76
:100260003A0043616E6E6F7420656E746572207320
:1002700075626469723A20004D3234004D32332089
:100280002573006175746F25692E67004572726F62
:10029000723A006572726F722077726974696E6764
:1002A00020746F2066696C6500436172642065721A
:1002B000726F723A004E6F74205344207072696EF0
:1002C00074696E67002F005344207072696E746900
:1002D0006E67206279746520002E0044656C657439
:1002E000696F6E206661696C65642C2046696C6577
:1002F0003A200046696C652064656C657465643AF3
:10030000002E006F70656E206661696C65642C203C
:1003100046696C653A200057726974696E6720748B
:100320006F2066696C653A20002E006F70656E2044
:100330006661696C65642C2046696C653A20002E04
:10034000006F70656E206661696C65642C2046697B
:100350006C653A200046696C652073656C65637452
:100360006564002053697A653A200046696C65200F
:100370006F70656E65643A20002E006F70656E20A8
:100380006661696C65642C2046696C653A2000538F
:10039000442063617264206F6B006F70656E526FF2
:1003A0006F74206661696C656400766F6C756D654D
:1003B0002E696E6974206661696C6564005344201F
:1003C000696E6974206661696C006563686F3A00E4
:1003D00048617264636F6465642044656661756C2E
:1003E000742053657474696E6773204C6F61646523
:1003F000640053746F7265642073657474696E670A
:10040000732072657472696576656400204400200B
:1004100049002020204D33303120500050494420E5
:1004200073657474696E67733A00205A002059002E
:1004300020204D323036205800486F6D65206F66A1
:100440006673657420286D6D293A00204500205A96
:100450000020580020420020540020204D3230352A
:10046000205300416476616E636564207661726931
:1004700061626C65733A20533D4D696E2066656517
:10048000647261746520286D6D2F73292C20543D92
:100490004D696E2074726176656C20666565647264
:1004A00061746520286D6D2F73292C20423D6D6984
:1004B0006E696D756D207365676D656E7420746906
:1004C0006D6520286D73292C20583D6D6178696D0C
:1004D000756D205859206A65726B20286D6D2F73D9
:1004E000292C20205A3D6D6178696D756D205A2048
:1004F0006A65726B20286D6D2F73292C2020453D75
:100500006D6178696D756D2045206A65726B202874
:100510006D6D2F73290020540020204D323034207F
:100520005300416363656C65726174696F6E3A2054
:10053000533D616363656C65726174696F6E2C20F5
:10054000543D7265747261637420616363656C65A8
:10055000726174696F6E00204500205A00205900B6
:1005600020204D3230312058004D6178696D756D15
:1005700020416363656C65726174696F6E20286DDC
:100580006D2F7332293A00204500205A002059006F
:1005900020204D3230332058004D6178696D756DE3
:1005A0002066656564726174657320286D6D2F73B4
:1005B000293A00204500205A0020590020204D39BA
:1005C0003220580053746570732070657220756E08
:1005D00069743A0053657474696E67732053746F5D
:1005E000726564006563686F3A004572726F723AB3
:1005F000005072696E7465722073746F70706564F8
:100600002064756520746F206572726F72732E207E
:1006100046697820746865206572726F7220616E19
:100620006420757365204D39393920746F207265E7
:1006300073746172742E202854656D7065726174D4
:100640007572652069732072657365742E20536519
:1006500074206974206166746572207265737461B8
:100660007274696E6729005072696E7465722068D1
:10067000616C7465642E206B696C6C282920636141
:100680006C6C656421006F6B00526573656E643A33
:1006900020002200556E6B6E6F776E20636F6D6D5C
:1006A000616E643A2022002200556E6B6E6F776E89
:1006B00020636F6D6D616E643A2022007A5F6D6118
:1006C000783A2000795F6D61783A2000785F6D6933
:1006D0006E3A20005A3A00593A0020436F756E7402
:1006E00020583A2000453A005A3A00593A00583A00
:1006F000004649524D574152455F4E414D453A4D96
:1007000061726C696E2056313B20537072696E7451
:1007100065722F6772626C206D61736875702066F8
:100720006F722067656E36204649524D57415245DB
:100730005F55524C3A687474703A2F2F6669726D27
:10074000776172652E756C74696D616B65722E636D
:100750006F6D2050524F544F434F4C5F564552538C
:10076000494F4E3A312E30204D414348494E455F66
:10077000545950453A556C74696D616B65722045EA
:10078000585452554445525F434F554E543A310ADE
:100790000020423A0020453A00543A0020573A00DF
:1007A00020453A00543A002042403A0020403A00A6
:1007B000202F0020423A00202F006F6B20543A0077
:1007C0002569206D696E2C202569207365630045BD
:1007D0006E642066696C65206C697374004265679D
:1007E000696E2066696C65206C6973740000000096
:1007F00000000061430000664300000000000000AC
:100800000000000000000066430000614300006635
:10081000430000664300006143000066430000A0FF
:10082000400000A04000004040FF01012569206811
:100830006F757273202569206D696E75746573001C
:10084000446F6E65207072696E74696E67206669A8
:100850006C65005072696E7465722073746F70708D
:1008600065642064756520746F206572726F7273A1
:100870002E2046697820746865206572726F722038
:10088000616E6420757365204D39393920746F208D
:10089000726573746172742E202854656D70657270
:1008A00061747572652069732072657365742E209A
:1008B0005365742069742061667465722072657373
:1008C00074617274696E6729006F6B004E6F204C03
:1008D000696E65204E756D62657220776974682057
:1008E000636865636B73756D2C204C617374204C69
:1008F000696E653A20004E6F20436865636B7375BF
:100900006D2077697468206C696E65206E756D6204
:1009100065722C204C617374204C696E653A20001E
:10092000636865636B73756D206D69736D61746366
:10093000682C204C617374204C696E653A20004C21
:10094000696E65204E756D626572206973206E6FE9
:1009500074204C617374204C696E65204E756D6215
:1009600065722B312C204C617374204C696E653A92
:1009700020004D31313000446F6E6520736176691F
:100980006E672066696C652E006F6B004D32390012
:100990002020506C616E6E657242756666657242AB
:1009A000797465733A20002046726565204D656D47
:1009B0006F72793A20004F6374203239203230311F
:1009C0003300436F6D70696C65643A200056657240
:1009D00073696F6E2031332E31302D3300207C202F
:1009E000417574686F723A20004F63742032392069
:1009F000323031332031333A32383A343100204CFE
:100A000061737420557064617465643A2000312EFE
:100A1000302E30004D61726C696E200020536F667D
:100A20007477617265205265736574002057617434
:100A30006368646F67205265736574002042726F4B
:100A4000776E206F75742052657365740020457849
:100A50007465726E616C20526573657400506F77B7
:100A600065725570007374617274002200656E7156
:100A70007565696E672022002200656E7175656973
:100A80006E672022006563686F3A0020746F6F20E4
:100A90006C6F6E6720657874727573696F6E207005
:100AA000726576656E7465640020636F6C642065A2
:100AB0007874727573696F6E2070726576656E7486
:100AC00065640000002110422063308440A550C6B8
:100AD00060E770088129914AA16BB18CC1ADD1CE7C
:100AE000E1EFF13112100273325222B5529442F703
:100AF00072D662399318837BB35AA3BDD39CC3FFCC
:100B0000F3DEE36224433420040114E664C774A4D2
:100B10004485546AA54BB528850995EEE5CFF5AC1B
:100B2000C58DD55336722611163006D776F66695E2
:100B300056B4465BB77AA719973887DFF7FEE79D6B
:100B4000D7BCC7C448E5588668A778400861180232
:100B5000282338CCC9EDD98EE9AFF9488969990ABB
:100B6000A92BB9F55AD44AB77A966A711A500A3342
:100B70003A122AFDDBDCCBBFFB9EEB799B588B3B0B
:100B8000BB1AABA66C877CE44CC55C222C033C6092
:100B90000C411CAEED8FFDECCDCDDD2AAD0BBD685B
:100BA0008D499D977EB66ED55EF44E133E322E5122
:100BB0001E700E9FFFBEEFDDDFFCCF1BBF3AAF59AB
:100BC0009F788F8891A981CAB1EBA10CD12DC14E1C
:100BD000F16FE18010A100C230E3200450254046AF
:100BE000706760B9839893FBA3DAB33DC31CD37FCE
:100BF000E35EF3B1029012F322D2323542145277FF
:100C0000625672EAB5CBA5A89589856EF54FE52C9D
:100C1000D50DC5E234C324A014810466744764244E
:100C2000540544DBA7FAB79987B8975FE77EF71DAD
:100C3000C73CD7D326F2369106B01657667676159E
:100C40004634564CD96DC90EF92FE9C899E9898AFD
:100C5000B9ABA94458654806782768C018E10882EE
:100C600038A3287DCB5CDB3FEB1EFBF98BD89BBB0D
:100C7000AB9ABB754A545A376A167AF10AD01AB33E
:100C80002A923A2EFD0FED6CDD4DCDAABD8BADE85D
:100C90009DC98D267C076C645C454CA23C832CE08E
:100CA0001CC10C1FEF3EFF5DCF7CDF9BAFBABFD9ED
:100CB0008FF89F176E367E554E745E932EB23ED1DE
:100CC0000EF01E7C3C3E5E2B3D3F2F5B5D3B2C2A95
:100CD000225C0045313A200045303A20005A3A2043
:100CE00000593A2000583A20004D53312C4D5332D0
:100CF0002050696E730A0024F404D9201BC40C5CD4
:100D00000E9804C4095F0265077101F405F900FB40
:100D100004B30048048700C1036900580355000369
:100D2000034500BE023A008402310053022A002922
:100D300002250004022000E4011C00C8011900AFD4
:100D40000117009801140084011300710110006163
:100D500001100051010E0043010D0036010B002B64
:100D6000010B0020010B00150109000C0109000313
:100D7000010800FB000800F3000800EB000700E496
:100D8000000600DE000600D8000600D2000600CCF7
:100D9000000500C7000500C2000500BD000400B941
:100DA000000400B5000400B1000400AD000400A977
:100DB000000400A5000300A20003009F0004009BA4
:100DC00000030098000300950002009300030090C8
:100DD0000003008D0002008B0003008800020086E3
:100DE00000020084000300810002007F0002007DF9
:100DF0000002007B0002007900020077000100760B
:100E00000002007400020072000100710002006F15
:100E10000002006D0001006C0002006A0001006920
:100E20000002006700010066000100650001006427
:100E30000002006200010061000100600001005F2B
:100E40000002005D0001005C0001005B0001005A2F
:100E50000001005900010058000100570001005630
:100E60000001005500010054000100530000005330
:100E70000001005200010051000100500001004F2C
:100E80000001004E0000004E0001004D0001004C2A
:100E90000001004B0000004B0001004A0001004926
:100EA0000001004800000048000100470001004622
:100EB000000000460001004500000045000100441C
:100EC0000001004300000043000100420000004216
:100ED0000001004100000041000100400001003F0E
:100EE0000000003F0001003E0000003E0001003D08
:100EF0000000003D0001003C0000003C0000003C00
:100F00000001003B0000003B0001003A0000003AF5
:100F100000010039000000390001003800000038ED
:100F200000000038000100370000003700010036E3
:100F300000000036000000360001003500000035DA
:100F400000000035000100340000003400000034CF
:100F500000010033000000330000003300010032C4
:100F600000000032000000320001003100000031BA
:100F700000000031000100300000003000000030AF
:100F80000001002F0000002F0000002F0000002FA4
:100F90000001002E0000002E0000002E0001002D98
:100FA0000000002D0000002D0000002D0001002C8D
:100FB0000000002C0000002C0000002C0001002B81
:100FC0000000002B0000002B0000002B0001002A75
:100FD0000000002A0000002A0000002A0001002969
:100FE000000000290000002900000029000000295D
:100FF0000001002800000028000000280000002850
:101000000000002800010027000000270000002742
:101010000000002700000027000100260000002635
:101020000000002600000026000000260001002528
:10103000000000250000002500000025000000251C
:10104000000000250001002400000024000000240E
:101050000000002400000024000100230000002301
:1010600000000023000000230000002300000023F4
:1010700000000023000100220000002200000022E6
:1010800000000022000000220000002200010021D8
:1010900000000021000000210000002100000021CC
:1010A00000000021000000210001002000000020BD
:1010B00000000020000000200000002000000020B0
:1010C00000000020000000200001001F0000001FA1
:1010D0000000001F0000001F0000001F0000001F94
:1010E0000000001F0001001E0000001E0000001E86
:1010F0000000001E00000024F4D43050C38E20C233
:10110000A24017828B7011127A910D816CD90AA8B6
:1011100061E108C7586607615143061E4B5D05C172
:1011200045A7041A411104093D9803713931034060
:1011300036DB0265339102D4305402802E1D0263E7
:101140002CEE01752AC501B028A001102781018F5E
:101150002564012B244B01E0223401AC211F018DB9
:10116000200D01801FFC00841EED00971DDF00B8DC
:101170001CD200E61BC600201BBC00641AB200B2E1
:1011800019A8000A19A0006A189900D11791004007
:10119000178B00B516840031167E00B31579003A1E
:1011A000157300C7146F0058146A00EE13660088A8
:1011B00013630025135E00C7125B006C1257001505
:1011C000125400C111510070114F0021114B00D673
:1011D0001049008D1047004610440002104200C024
:1011E0000F4000800F3E00420F3C00060F3B00CB3B
:1011F0000E3800930E37005C0E3500270E3400F3D6
:101200000D3200C10D3100900D3000600D2E003206
:101210000D2D00050D2C00D90C2B00AE0C290085DE
:101220000C29005C0C2700350C27000E0C2600E86A
:101230000B2400C40B2400A00B23007D0B23005AB9
:101240000B2100390B2100180B2000F80A1F00D9D0
:101250000A1E00BB0A1E009D0A1D00800A1D0063B5
:101260000A1C00470A1B002C0A1B00110A1A00F76F
:10127000091A00DD091900C4091900AB0919009207
:101280000917007B091800630917004C091600367E
:10129000091600200916000A091500F5081500E0D6
:1012A000081400CC081400B8081400A40814009016
:1012B0000813007D0812006B08130058081200463E
:1012C000081200340811002308110012081100014F
:1012D000081100F0071000E0071000D0071000C050
:1012E000071000B0070F00A107100091070E008340
:1012F000070F0074070F0065070E0057070E00491F
:10130000070E003B070D002E070E0020070D0013EF
:10131000070D0006070D00F9060C00ED060D00E0B4
:10132000060C00D4060C00C8060C00BC060C00B06D
:10133000060C00A4060B0099060C008D060B00821B
:10134000060B0077060B006C060B0061060A0057BF
:10135000060B004C060A0042060A0038060A002E58
:10136000060A0024060A001A060A001006090007E9
:10137000060A00FD050900F4050900EB050900E275
:10138000050900D9050900D0050900C7050900BEF7
:10139000050900B5050800AD050800A50509009C74
:1013A000050800940508008C050800840508007CE9
:1013B000050800740508006C050700650508005D58
:1013C000050700560508004E0507004705070040C1
:1013D00005080038050700310507002A0507002326
:1013E0000507001C050600160507000F0507000885
:1013F00005060002050700FB040600F5040700EEE1
:10140000040600E8040600E2040700DB040600D539
:10141000040600CF040600C9040600C3040600BD8C
:10142000040600B7040600B1040500AC040600A6DB
:10143000040600A00405009B040600950405009026
:101440000406008A04050085040500800406007A6D
:1014500004050075040500700405006B04050066B2
:10146000040500610405005C0405005704050052F2
:101470000405004D04050048040500430405003E32
:101480000404003A04050035040500300404002C6F
:1014900004050027040400230405001E0404001AA8
:1014A00004040016040500110404000D04040009DE
:1014B0000405000404040000040400FC030400F814
:1014C000030400F4030400F0030400EC030400E848
:1014D000030400E4030400E0030400DC030400D878
:1014E000030400D4030400D0030400CC030400C8A8
:1014F000030300C50303006563686F3A00205A3A8E
:101500000020593A0020583A00656E6473746F7079
:1015100073206869743A20004572726F723A005401
:10152000656D70657261747572652068656174655A
:101530006420626564207377697463686564206FF2
:1015400066662E204D415854454D5020747269678F
:101550006765726564202121003A204578747275B0
:10156000646572207377697463686564206F66666A
:101570002E204D494E54454D502074726967676561
:101580007265642021003A20457874727564657232
:10159000207377697463686564206F66662E204DDA
:1015A000415854454D50207472696767657265648F
:1015B000202100202D20496E76616C6964206578B9
:1015C000747275646572206E756D6265722021009B
:1015D00000000000300E0100C00E0A00500F140081
:1015E000D00F1E0060102800E010320070113C0087
:1015F000F01146007012500000135A00801364006E
:1016000000146E00901478001015820090158C0064
:10161000101696009016A0001017AA009017B4009C
:101620001018BE009018C8001019D2009019DC00E4
:10163000101AE600801AF000001BFA00801B04015B
:10164000F01B0E01701C1801F01C2201601D2C0102
:10165000E01D3601501E4001D01E4A01401F5401BA
:10166000B01F5E0130206801A020720110217C01B2
:1016700090218601002290016026F401902A5802F0
:10168000802EBC0250322003E03584035039E80339
:10169000803C4C04504944204175746F74756E65EC
:1016A0002066696E697368656421205075742074C2
:1016B0006865204B702C204B6920616E64204B6460
:1016C00020636F6E7374616E747320696E746F2023
:1016D000436F6E66696775726174696F6E2E68001C
:1016E000504944204175746F74756E652066616958
:1016F0006C6564212074696D656F75740020403AD3
:10170000006F6B20543A006F6B20423A00504944FE
:10171000204175746F74756E65206661696C6564CF
:10172000212054656D706572617475726520746FE7
:101730006F206869676800204B643A2000204B697D
:101740003A2000204B703A200020436C617369639B
:101750002050494420002054753A2000204B753A0F
:101760002000206D61783A2000206D696E3A2000DB
:1017700020643A200020626961733A20004D41499B
:101780004E54454E414E4345004D4154455249410A
:101790004C005052494E5400737570706F72744013
:1017A000756C74696D616B65722E636F6D00436F4C
:1017B0006E746163743A005361666574792063697D
:1017C00072637569740054656D702073656E736F14
:1017D00072204245440054656D702073656E736FCE
:1017E00072004552524F52202D2053544F505045B5
:1017F0004400801506060606FEFEFEFEFC00000004
:1018000000000000FCFEFEFEFC0000000EFEFEFEDE
:10181000FE0000E0FCFEFEFCE0E0000000CECECECC
:10182000000000C0C0C0C0C0C080000000000000B8
:1018300080C0C0800000000000008080C0C0C0C028
:10184000C0C0C080800000000006FEFEFEFE00005A
:10185000000080C0C0C00000000000008080C0C048
:10186000C080808000000000C0C0C0C00080C0C038
:10187000C0C08000000000007FFFFFFFFF8000006D
:1018800000000080FFFFFFFFFF00000000FFFFFFE0
:10189000FF000000FFFFFFFF0000000000FFFFFF50
:1018A00000000081F1FFFF3F0F3FFFFCF0F0FCFF65
:1018B0003F0F3FFFFEF880000000C1E1F1F1713100
:1018C000010183FFFFFFFC000000FFFFFFFF000C92
:1018D0003EFFFFF7C301000000FCFEFF870311314C
:1018E00031333F3F3F1E000001FFFFFFFF070301B1
:1018F000010101000000000000010307070F0F0FA6
:101900000F0F0F0F0707070F0F06000000070F0F3D
:1019100007000000070F0F0700000000000F0F0F67
:101920000000060F0F070100000001070F0F07015D
:1019300000000001070F0F06000003070F0F0E0E37
:10194000060703070F0F07000000070F0F0700002F
:101950000000030F0F0F060000000307070F0E0E15
:101960000E0E0E0E06000000000F0F0F0F000000FD
:10197000000000008015090909F90101010103FEB9
:101980000000000000FE0301010103FE001FF10141
:10199000010101FFF01E030101031E10F000FF31E1
:1019A0003131FF00E020202020202060C080000096
:1019B00080C060202060C000000000C04060202087
:1019C00020202020206040C080000FF9010101018B
:1019D000FF0080C060202020E000000080C0406048
:1019E000202020604040C08000E020202020E060D7
:1019F0002020202060C0000000FF80000000007F49
:101A0000C0808080C07F0000000000FF0000FF0059
:101A1000000000FF01FF00000000FF010100FF00C7
:101A20000000FF00C37A0E0000C070C000030E0E5D
:101A30000300C070C00001077CC000E3321A0A0A2C
:101A40008ACAFAC67C00000003FE00FF0000000006
:101A5000FF73C10000083CE68300FE03010078FC30
:101A6000EE4A4E4C404040613F03FE00000000F84B
:101A70000C06020202030000000003060C08181006
:101A80001010101010101808181010190F000F184F
:101A90001010180F000F181010180F0000001F1062
:101AA00010101F0F191010180E0300030E1810103D
:101AB000180E0300030E181010190F070C18101041
:101AC000111119080C181010180F000F1810101809
:101AD0000F0001071C101010190F01070C08181037
:101AE000111111111111190F00001F101010101FEA
:101AF0000000000000002F40000000000000000077
:101B000000000000808080C0E0FEFF191E989898B9
:101B10001818181818189E9F991E38F0E000000039
:101B200000000000000000000000000000000000B5
:101B30003CFEFFFF99F1E1C3FFFF000063636360B8
:101B400060606060606363630000FFFF7C380000DA
:101B500000000000000000000080C060B0D8D81C69
:101B6000FCFF3F0F8FCFC7C7C7C6C6C6C6C6C6C60F
:101B7000C6C6C6C6C6C6C6C6C6C7C7C4CC0C1CF831
:101B8000F870C00000000EFFF92A2B2B2828FCFF5C
:101B9000FF0000FFFFFFFFFFFFFFBFB717B5BDB599
:101BA00000B5B5F717FFBFBFFFFFFFFF0000FFFF46
:101BB000FCFF0700C0F0FFFFFDDD1D19193FFFFF0F
:101BC0000000FFFFFFFFFFFFFFFBF1FBFBEAEEC0A2
:101BD000EEEAFAF0FAFAFFFFFFFFFF0000FFFF0F47
:101BE0001FF8E00003070F0F1B1819FBFEFFFFF0A3
:101BF000E0C0C1E1F1F1F1F1F1F1F1F1F1F1F1F94F
:101C0000F9F9F9F9F9797979F1F010181F07060354
:101C1000030000000000000000F8FFEFDFBF7FFFBF
:101C2000FFFF404143437F212020217FFFFFFF3FF3
:101C3000B091D1DFD050581F1FF0F000000000001D
:101C40000000000000000003070F1E3D7B77EED16F
:101C5000DEDECF4B4B6969686868603F3F373737D6
:101C6000353430101018181A1B0F06000000000041
:101C7000100FFC0E0FCFCFCFCECCCCCCCCCCCCDC4D
:101C8000C0C007707E7F7F7F7F7F7F7F7F7F7F7F6A
:101C90000F017120FFFFFFFFFFFFFFFFFFFFFCE0D1
:101CA00000000000000000000000E0FCFFFFFFFF5C
:101CB000FFFFFFFFFFFF000000000000000000002A
:101CC0000000000000000000000000000000000014
:101CD000FFFFFFFFFFFFFF0000000000000000000B
:101CE00000000000000000000000000000000000F4
:101CF00000000000000000000000000000000000E4
:101D00000000000000FFFFFFFFFFFFFF7FFFFFFF5E
:101D1000FFFFF8800000000080F0FFFFFFFFFF3FA3
:101D2000FFFFFFFFFFFFFF00000030F8F8FCFC7E24
:101D30007E7E3E3E3E3E7E7EFEFEFCFCF8E0800067
:101D400000FFFFFFFFFFFFFF000080C0E0F0F8FC96
:101D5000FEFE7E3E1E0E06C0E0F0F8FCFCFE7E3E5F
:101D60003E3E3E3E7EFEFCFCF8F0C0800000FEFEE3
:101D7000FEFEFEFEFEFEFFFFFFFFFFFFFF00031F54
:101D8000FFFFFFFFFFFCE0E0FCFFFFFFFFFF1F0185
:101D900000FFFFFFFFFFFFFF0000C0E0F0F0F8F8DA
:101DA000FC7C7C3C3C3E1E1E1EFFFFFFFFFFFFFF36
:101DB0000000FFFFFFFFFFFFFFFEFFFFFFFFFFFF32
:101DC000FFF1C080000000FFFFFFFFFFFFFF3C3C72
:101DD0003C3C3C3C3C3C3C3F3F3F3F3F3F000000E5
:101DE00000000000000000FFFFFFFFFFFFFF0000FA
:101DF0000000073FFFFFFFFFFFFFFFFF3F0700005F
:101E00000000FFFFFFFFFFFFFF00003F7FFFFFFF1E
:101E1000FFFCFCF8F8F87C7C3C3EFFFFFFFFFFFF77
:101E2000FF0000FFFFFFFFFFFFFF030100000307AC
:101E30001F7FFFFFFFFEFCF0E38F1F3F3F7F7FFE12
:101E4000FCF8F8F0F0F0F8F8FCFC7E7E3C30000086
:101E5000FEFEFEFEFEFEFEFE43414E43454C0020CC
:101E600073656300206D696E0020686F75720020D5
:101E7000686F75727300000000000000005F0000D2
:101E80000007000700147F147F14242A7F2A1223DE
:101E90001308646236495522500005030000001CF7
:101EA0002241000041221C00082A1C2A0808083E82
:101EB00008080050300000080808080800606000AA
:101EC0000020100804023E5149453E00427F400078
:101ED00042615149462141454B311814127F102768
:101EE000454545393C4A49493001710905033649A0
:101EF000494936064949291E003636000000563643
:101F0000000000081422411414141414412214086F
:101F1000000201510906324979413E7E1111117EBC
:101F20007F494949363E414141227F4141221C7F40
:101F3000494949417F090901013E414151327F0828
:101F400008087F00417F41002040413F017F081485
:101F500022417F404040407F0204027F7F040810FE
:101F60007F3E4141413E7F090909063E4151215EC4
:101F70007F09192946464949493101017F01013F3D
:101F80004040403F1F2040201F7F2018207F6314C7
:101F90000814630304780403615149454300007F3A
:101FA0004141020408102041417F00000402010267
:101FB0000440404040400001020400205454547842
:101FC0007F484444383844444420384444487F38A7
:101FD00054545418087E090102081454543C7F08D4
:101FE00004047800447D40002040443D00007F1000
:101FF000284400417F40007C041804787C080404D5
:102000007838444444387C14141408081414187C98
:102010007C080404084854545420043F4440203CA5
:102020004040207C1C2040201C3C4030403C442848
:102030001028440C5050503C4464544C4400083622
:10204000410000007F0000004136080008082A1CFB
:1020500008081C2A08086275696C64706C617465F4
:102060002E006F662061646A757374696E672079EB
:102070006F75720074726F7567687420746865207C
:1020800070726F6365737300492077696C6C2067A9
:102090007569646520796F7500434F4E54494E55FC
:1020A0004500473120462569205A25692058256971
:1020B0002059256900473238205A3020583020599D
:1020C000300066726F6D20746865206275696C649B
:1020D000706C6174652E0061206D696C6C696D6552
:1020E000746572206177617900756E74696C207413
:1020F0006865206E6F7A7A6C6520697300526F7420
:102100006174652074686520627574746F6E003444
:102110002F323100434F4E54494E554500434F4EE8
:1021200054494E554500473120462569205A300014
:1021300047312046256920582569205925690047DF
:102140003120462569205A350066726F6D2074680B
:1021500065206275696C64706C6174652E006973CA
:102160002061206D696C6C696D65746572206177A2
:1021700061790073637265772074696C6C20746890
:1021800065206E6F7A7A6C65005475726E206C658E
:102190006674206275696C64706C61746500352FBB
:1021A000323100434F4E54494E5545004731204689
:1021B0002569205A30004731204625692058256975
:1021C0002059256900473120462569205A35006687
:1021D000726F6D20746865206275696C64706C61E3
:1021E00074652E0069732061206D696C6C696D6582
:1021F000746572206177617900736372657720740A
:10220000696C6C20746865206E6F7A7A6C65005416
:1022100075726E207269676874206275696C64708B
:102220006C61746500362F323100434F4E54494E75
:10223000554500746865206275696C64706C6174E2
:1022400065206C6576656C2E007061706572207417
:102250006F2066696E652D74756E65006E6F7720F0
:102260007573652061207368656574206F66005220
:102270006570656174207468697320737465702C6F
:102280002062757400372F323100434F4E54494E4F
:10229000554500473120462569205A3000473120F6
:1022A000462569205825692059256900473120466F
:1022B0002569205A350062697420726573697374E8
:1022C000616E63652E00756E74696C20796F752080
:1022D0006665656C2061006275696C64706C617420
:1022E0006520616E64206E6F7A7A6C6500536C694C
:1022F0006465206120706170657220626574776525
:10230000656E00382F323100434F4E54494E5545CB
:1023100000434F4E54494E554500746865206C6526
:10232000667420636F726E65722E2E2E0052657079
:10233000656174207468697320666F7200392F328A
:102340003100434F4E54494E554500746865207224
:102350006967687420636F726E65722E2E2E00524C
:102360006570656174207468697320666F720031EE
:10237000302F323100434F4E54494E554500444FA3
:102380004E4500746F20696E73657274206D6174C0
:10239000657269616C2E00746865206E65787420C2
:1023A0007374657020697300746865206275696C68
:1023B00064706C617465004E6F772074686174207E
:1023C0007765206C6576656C65640031312F32313C
:1023D00000434F4E54494E55450047312046313257
:1023E0003030302058313130205930006D61746503
:1023F0007269616C206C6F6164696E6700707269EC
:102400006E74686561642068656174696E672066D2
:102410006F7200506C6561736520776169742C0080
:1024200031322F32310061626F7665207468652029
:102430006172726F772E00796F757220556C7469B6
:102440006D616B6572322C0066726F6D2074686509
:102450002072656172206F6600496E736572742028
:102460006E6577206D6174657269616C0031332F20
:10247000323100434F4E54494E5545004C6F616414
:10248000696E67206D6174657269616C2E2E2E0015
:1024900031342F32310066726F6D206E6F7A7A6C34
:1024A000652E2E2E006D6174657269616C206578F1
:1024B000697473005075736820627574746F6E2050
:1024C0007768656E0031352F323100434F4E5449E5
:1024D0004E554500556C74696D616B6572322E0006
:1024E000696E73657274656420696E207468652016
:1024F000006D6174657269616C20796F7520686127
:102500007665004E6578742C2073656C6563742065
:102510007468650031362F3231005245414459000C
:1025200031372F32310041425300504C4100697322
:1025300020746869732072696768743F0041425370
:10254000206173206D6174657269616C2C00596F34
:102550007520686176652063686F73656E00313839
:102560002F3231004E4F0059455300697420697372
:10257000207573696E672E006F66206D61746572D9
:1025800069616C006B6E6F77732077686174206B84
:10259000696E64004E6F7720796F757220556C7488
:1025A000696D616B6572320031392F323100434FF2
:1025B0004E54494E5545006D616B65206120334492
:1025C000205072696E74210049276D207265616424
:1025D00079206C657427730032302F3231004152FC
:1025E0004520594F552052454144593F00746F20B2
:1025F0007072696E742069742100616E642070725B
:102600006573732074686520627574746F6E006FF3
:102610006E207468652053442D63617264005365B5
:102620006C6563742061207072696E742066696CD9
:10263000650032312F3231004C455427532050521F
:10264000494E540052656164696E6720636172642B
:102650002E2E2E0032312F323100796F75722055B7
:102660006C74696D616B6572322E2E2E0074686118
:10267000742063616D65207769746800506C6561D2
:10268000736520696E736572742053442D636172A3
:10269000640032312F32310069732074686973200D
:1026A00072696768743F00504C41206173206D610E
:1026B00074657269616C2C00596F7520686176656C
:1026C0002063686F73656E0031382F3231004E4FD2
:1026D0000059455300473238205A300062757474EF
:1026E0006F6E20746F20636F6E74696E7565005530
:1026F0006C74696D616B6572212050726573732013
:102700007468650073746172747570206F662079E7
:102710006F75720057656C636F6D6520746F207400
:10272000686520666972737400312F323100434F3F
:102730004E54494E5545006120666972737420728B
:10274000756E2077697A6172642E0077616C6B20F8
:10275000796F75207468726F756768006669727347
:1027600074207374617274757020492077696C6C81
:1027700000426563617573652074686973206973CD
:102780002074686500322F323100434F4E54494E59
:10279000554500473120462569205A2569004732B2
:1027A00038205A3000676F696E6720746F20646F3D
:1027B0002074686174206E6F772E0061646A75738F
:1027C000746D656E74732C20776520617265007777
:1027D00065206E65656420746F20646F20736F6D73
:1027E00065004166746572207472616E73706F72F9
:1027F000746174696F6E00332F323100434F4E5451
:10280000494E554500473120462569205A25692003
:1028100058256920592569004732382058302059F9
:1028200030004300432F00436C69636B20746F20BA
:1028300072657475726E004275696C64706C617457
:10284000652074656D702E3A004300432F00436C81
:1028500069636B20746F2072657475726E004865D1
:1028600061642074656D70657261747572653A009B
:10287000504C415445004255494C442D00504C4168
:102880005445004255494C442D0052455455524E32
:1028900000414456414E43454400004731205A34DC
:1028A0003000473238205A3000473238205A300042
:1028B00047323820583020593000414456414E4369
:1028C000454400746F2064656661756C743F005206
:1028D000657365742065766572797468696E6700E2
:1028E0004E4F005945530056657273696F6E203123
:1028F000332E31302D33004F63742033312032308A
:1029000031332030373A33333A3130005265747501
:10291000726E006D6D2F736563004D61782073706A
:10292000656564205A006D6D2F736563004D617895
:102930002073706565642059006D6D2F73656300A9
:102940004D61782073706565642058006D6D2F733C
:10295000656300582F59204A65726B0030306D6DE9
:102960002F7365635E3200416363656C65726174E9
:10297000696F6E004D4F54494F4E006D6D2F73655A
:1029800063006D6D2F736563006D6D2F736563005C
:102990006D6D2F736563006D6D2F7365635E32001F
:1029A0003F3F3F004D6178207370656564205A0099
:1029B0004D61782073706565642059004D61782001
:1029C0007370656564205800582F59204A65726BF2
:1029D00000416363656C65726174696F6E003C20D1
:1029E00052455455524E006D6D2F7365630052650C
:1029F0007472616374207370656564006D6D00525C
:102A0000657472616374206C656E6774680052450A
:102A10005452414354494F4E006D6D2F736563000E
:102A20006D6D003F3F3F00526574726163742073A7
:102A3000706565640052657472616374206C656EC4
:102A4000677468003C2052455455524E0043004381
:102A50002F00436C69636B20746F2072657475720C
:102A60006E00526F7461746520746F2065787472A3
:102A700075646500486561642074656D7065726198
:102A8000747572653A0025004272696768746E65F4
:102A90007373004C45440025003F3F3F0020476CC6
:102AA0006F77207768656E20646F6E6500204F6ECB
:102AB000207768696C65207072696E74696E670052
:102AC00020416C77617973204F66660020416C77F6
:102AD000617973204F6E004272696768746E657326
:102AE00073003C2052455455524E003F3F3F004634
:102AF0006163746F727920726573657400566572D4
:102B000073696F6E004D6F74696F6E2073657474B6
:102B1000696E67730052657472616374696F6E20C9
:102B200073657474696E6773004D6F7665206D61AF
:102B300074657269616C00526169736520627569C0
:102B40006C64706C617465004C6F7765722062759F
:102B5000696C64706C61746500486F6D65206865B0
:102B6000616400486561747570206275696C647099
:102B70006C61746500486561747570206865616496
:102B8000004C45442073657474696E6773003C2083
:102B900052455455524E0041425300504C41005250
:102BA000455455524E0053455454494E47530043E3
:102BB00048414E4745004D4154455249414C005310
:102BC000656C6563746564206D6174657269616CC0
:102BD0003A004F4B0025004D6174657269616C20AD
:102BE000666C6F7700250046616E207370656564C2
:102BF000006D6D004D6174657269616C204469619E
:102C00006D657465720043004275696C64706C6137
:102C100074652054656D702E00430054656D7065B9
:102C2000726174757265004D4154455249414C00C2
:102C300050524553455453004E657720707265736A
:102C40006574003C2052455455524E002500250025
:102C50006D6D00430043003F3F3F0053746F72654A
:102C60002061732070726573657400466C6F772005
:102C7000250046616E004469616D657465720048A7
:102C80006561746564206275696C64706C617465FB
:102C90000054656D7065726174757265003C2052F8
:102CA000455455524E004D6F6469667920746865CD
:102CB0002073657474696E677300250046616E3A0F
:102CC0002000430043002500466C6F773A006D6D8D
:102CD00000437573746F6D697A65003C20524554EA
:102CE00055524E00666F72206D6174657269616C39
:102CF0002072656D6F76616C0048656174696E67FE
:102D0000207072696E7468656164005265766572E0
:102D100073696E67206D6174657269616C005265DC
:102D20006D6F7665206D6174657269616C004341F9
:102D30004E43454C005245414459004731204625F9
:102D400069205825692059256900473238205830B4
:102D50002059300061626F76652074686520617269
:102D6000726F772E00796F7572206D616368696E7E
:102D7000652C0066726F6D20746865206261636BFC
:102D800073696465206F6600496E73657274206EA6
:102D90006577206D6174657269616C0043414E43D3
:102DA000454C00524541445900466F727761726448
:102DB000696E67206D6174657269616C00636F6D27
:102DC0006573206F757420746865206E6F7A7A6CF5
:102DD0006500576169742074696C6C206D6174655D
:102DE0007269616C0043414E43454C005245414479
:102DF000590053442043415244003B464C41564FF6
:102E0000523A556C746947436F6465003B464C41C8
:102E1000564F523A556C746947436F6465004E6F64
:102E20002066696C657320666F756E6421004F4B78
:102E3000004F4B0052656164696E67206361726484
:102E40002E2E2E00506C6561736520696E7365725D
:102E5000742063617264004E6F2053442D434152CD
:102E60004421003C204241434B003C2052455455F4
:102E7000524E0066726F6D2074686520736C6963D2
:102E800065722E0073657474696E67207769746863
:102E90002073657474696E67006F76657272696419
:102EA00065206D616368696E6500546869732066AA
:102EB000696C652077696C6C0043414E43454C005A
:102EC000434F4E54494E5545004731204631353029
:102ED000302045300047393220452D2569004732E2
:102EE00038004732380047312046313530302045F0
:102EF00030004739322045256900436F64653A0048
:102F000053442D63617264210072656164696E6768
:102F1000004572726F72207768696C650052455483
:102F200055524E20544F204D41494E007468652043
:102F30007072696E742E00596F752063616E207215
:102F4000656D6F7665005072696E742066696E6992
:102F5000736865640043005072696E746572206323
:102F60006F6F6C696E6720646F776E004241434BF0
:102F700020544F204D454E550054696D65206C65B9
:102F800066740054696D65206C65667420756E6B9F
:102F90006E6F776E004300430048656174696E6729
:102FA000206275696C64706C617465004300430055
:102FB00048656174696E67005072696E74696E6706
:102FC0003A0041424F52540054554E450041626F01
:102FD000727420746865207072696E743F004E4F81
:102FE000005945530025004D6174657269616C207C
:102FF000666C6F7700250046616E207370656564AE
:103000000025005072696E74207370656564005409
:10301000554E45006D6D2F73656300526574726186
:103020006374207370656564006D6D005265747221
:10303000616374206C656E67746800524554524138
:103040004354494F4E006D6D2F736563006D6D00E5
:103050003F3F3F0052657472616374207370656511
:10306000640052657472616374206C656E67746885
:10307000003C2052455455524E0025002500430087
:103080004300430043002500526574726163746914
:103090006F6E004D6174657269616C20666C6F774C
:1030A0000046616E207370656564004275696C64EA
:1030B000706C6174652074656D702E0054656D7060
:1030C00065726174757265005370656564003C20BB
:1030D00052455455524E00507265706172696E6768
:1030E00020746F207072696E743A0048656174696B
:1030F0006E672075702E2E2E0041424F52540054A0
:10310000554E45004E6F20696E666F20617661698D
:103110006C61626C65006D006D004D617465726973
:10312000616C3A200054696D653A20003B4D415472
:10313000455249414C3A003B54494D453A00466F8F
:103140006C64657200494E46494E4954594E414E91
:10315000CDCCCC3D0AD7233C17B7D13877CC2B3216
:103160009595E6241FB14F0A000020410000C84297
:1031700000401C4620BCBE4CCA1B0E5AAEC59D74F6
:10318000FC2F7252F72F11241FBECFEFD1E2DEBF0A
:10319000CDBF00E00CBF14E0A0E0B2E0E4ECFAEA3E
:1031A00001E00BBF02C007900D92A433B107D9F71D
:1031B00015E1A4E3B4E001C01D92A33DB107E1F71E
:1031C00011E3C4E8D1E304C02297FE010E9452D566
:1031D000C038D107C9F704D00C9452CC0C9400002D
:1031E000CF93DF9332D10E94644FC0E0D0E00E94C1
:1031F000DB4E2097E1F30E940000F9CFCF92DF92DF
:10320000EF92FF920F931F93CF93DF937C016B019B
:103210008A01C0E0D0E00FC0D6016D916D01D701E9
:10322000ED91FC910190F081E02DC7011995C80F37
:10323000D91F015010400115110571F7CE01DF9122
:10324000CF911F910F91FF90EF90DF90CF90089555
:103250008230B9F0833028F4882351F0813051F561
:103260000AC0843011F18430E8F0853019F520C0AF
:1032700010926E00089580916F008D7F80936F0093
:103280000895809170008D7F8093700081E080931D
:10329000B0008091B100887F84608093B10010926B
:1032A000B30008951092710008951092720008956D
:1032B0001092730008951F93182F80913F03811778
:1032C00011F09FEF06C0EFE2F1E094918FEF809351
:1032D0003F03892FBDDF812F60E0AAD21F9108959F
:1032E0001F920F920FB60F920BB60F9211242F93CD
:1032F0003F934F935F936F937F938F939F93AF937E
:10330000BF93EF93FF938091340490913504A09183
:103310003604B09137040097A105B10551F1E09151
:103320003804F0913904808190913A048927808390
:103330008091340490913504A0913604B091370403
:10334000181619061A061B06BCF4809134049091D5
:103350003504A0913604B09137040197A109B10951
:103360008093340490933504A0933604B0933704CB
:1033700003C080913F039FDFFF91EF91BF91AF9119
:103380009F918F917F916F915F914F913F912F917D
:103390000F900BBE0F900FBE0F901F9018951F92AD
:1033A0000F920FB60F9211242F933F938F939F93F9
:1033B000AF93BF9380913F0490914004A09141044A
:1033C000B0914204309143040196A11DB11D232FF9
:1033D0002D5F2D3720F02D570196A11DB11D209393
:1033E000430480933F0490934004A0934104B0931E
:1033F000420480913B0490913C04A0913D04B09123
:103400003E040196A11DB11D80933B0490933C04A2
:10341000A0933D04B0933E04BF91AF919F918F91D3
:103420003F912F910F900FBE0F901F9018958FB75F
:10343000F89420913F043091400440914104509110
:1034400042048FBFB901CA010895789484B582609F
:1034500084BD84B5816084BD85B5826085BD85B538
:10346000816085BDEEE6F0E0808181608083E1E8E7
:10347000F0E010828081826080838081816080831F
:10348000E0E8F0E0808181608083E1EBF0E0808122
:1034900084608083E0EBF0E0808181608083E1E9FB
:1034A000F0E0808182608083808181608083E0E9B8
:1034B000F0E0808181608083E1EAF0E080818260D9
:1034C0008083808181608083E0EAF0E08081816098
:1034D0008083E1E2F1E0808182608083808181608D
:1034E0008083E0E2F1E0808181608083EAE7F0E0C0
:1034F000808184608083808182608083808181601C
:1035000080838081806880831092C10008951F931A
:10351000CF93DF93182FEB0161E0D7D0209709F408
:10352000CAC0CF3FD10509F4C9C0E12FF0E0E65F82
:10353000FD4F8491893009F466C08A30B0F484303C
:10354000F1F1853040F4823059F1833070F58130EB
:1035500009F0AEC020C0873009F443C0883008F0BD
:1035600048C0863009F0A4C034C08D3009F478C05A
:103570008E3038F48B3009F45AC08C3008F066C0B5
:103580004CC0803109F480C0813109F487C08F308C
:1035900009F08EC06FC084B5806884BDC7BD91C07E
:1035A00084B5806284BDC8BD8CC080918000806875
:1035B00080938000D0938900C093880082C080915E
:1035C0008000806280938000D0938B00C0938A003B
:1035D00078C08091B00080688093B000C093B30041
:1035E00070C08091B00080628093B000C093B4003E
:1035F00068C080919000806880939000D09399007B
:10360000C09398005EC0809190008062809390008B
:10361000D0939B00C0939A0054C080919000886022
:1036200080939000D0939D00C0939C004AC08091ED
:10363000A00080688093A0008091A0008F7B809381
:10364000A000D093A900C093A8003BC08091A00027
:1036500080628093A000D093AB00C093AA0031C0D9
:103660008091A00088608093A000D093AD00C093AB
:10367000AC0027C080912001806880932001D09306
:103680002901C09328011DC0809120018062809390
:103690002001D0932B01C0932A0113C080912001F7
:1036A000886080932001D0932D01C0932C0109C024
:1036B000C038D1051CF4812F60E002C0812F61E089
:1036C000B7D0DF91CF911F910895CF93DF93482F0B
:1036D00050E0CA018C539E4FFC01349142585E4F1A
:1036E000FA018491882369F190E0880F991FFC0109
:1036F000E05DFE4FA591B491FC01E65BFE4FC591E4
:10370000D491662351F42FB7F8948C91932F909510
:1037100089238C93888189230BC0623061F42FB791
:10372000F8948C91932F909589238C938881832B87
:1037300088832FBF06C09FB7F8948C91832B8C93FE
:103740009FBFDF91CF910895893009F449C08A3035
:10375000A0F4843051F1853040F4823079F1833027
:1037600000F5813009F063C026C0873079F18830D8
:1037700098F5863009F05BC025C08D3009F442C051
:103780008E3028F48B30B1F18C30C0F52DC08031F3
:1037900009F442C0813109F445C08F3009F047C0B7
:1037A00037C0809180008F7703C0809180008F7D2B
:1037B00080938000089584B58F7702C084B58F7D93
:1037C00084BD08958091B0008F7703C08091B000D0
:1037D0008F7D8093B0000895809190008F7707C00F
:1037E000809190008F7D03C080919000877F8093AF
:1037F000900008958091A0008F7707C08091A0006D
:103800008F7D03C08091A000877F8093A0000895E2
:10381000809120018F7703C0809120018F7D80935C
:103820002001089580912001877F809320010895D1
:10383000FF920F931F93F62E482F50E0CA01865F28
:103840009D4FFC012491CA018C539E4FFC011491A1
:1038500042585E4FFA0104910023C1F0222311F077
:10386000822F72DFE02FF0E0EE0FFF1FE65BFE4FCE
:10387000A591B4919FB7F894FF2021F48C911095F5
:10388000812302C08C91812B8C939FBF1F910F913C
:10389000FF900895AC01DB01FA0190E02EE28C91DB
:1038A000803229F0983009F421938C9181939F5FA5
:1038B00011969B30A1F71082CA010895FC01128273
:1038C00016A60895FC0186A5882311F081E0828365
:1038D0000895FC018281811112820895CF93DF93B4
:1038E000EC01FC01EB55FE4F8081882309F461C097
:1038F00081508083DE01AC5ABF4FFE01ED58FF4F6F
:103900008BE101900D928150E1F7FE01EE5AFF4FDD
:10391000CF58DF4F88819981C157D04091838083F0
:1039200030E0BE016B557E4F3FC0832F90E0AC016D
:103930004F5F5F4FDC01E5E0AA0FBB1FEA95E1F79F
:10394000A81BB90BAC0FBD1FFA0125E0EE0FFF1F3E
:103950002A95E1F7E41BF50BEC0FFD1FAD58BF4FA7
:10396000ED58FF4F2BE101900D922150E1F7FC0142
:1039700025E0EE0FFF1F2A95E1F7E81BF90BEC0F8E
:10398000FD1FEF58FF4FDA0185E0AA0FBB1F8A9594
:10399000E1F7A41BB50BAC0FBD1FAF58BF4F8D9106
:1039A0009C91918380833F5FFB018081381708F4ED
:1039B000BCCFDF91CF910895FC018DE294E091831B
:1039C00080838781882321F0CF0104960C94956D24
:1039D00008950F931F938C010E94087C0E94047B22
:1039E000C80183539E4F0E94956DF801128280E5B5
:1039F00092E00E94F0501F910F910895CF92DF92B4
:103A0000EF92FF920F931F93DF93CF93CDB7DEB763
:103A10006F970FB6F894DEBF0FBECDBF8C016B0160
:103A2000095A1F4FD8018C9107551040882321F463
:103A30008FE2E82EF12C03C0B0E5EB2EF12CE00E66
:103A4000F11E8DE294E09A8389831C821B82188682
:103A50001D82B7016C5F7F4FCE010596A60121E064
:103A60000E94CE74882391F5ECE5F2E0949108C0B1
:103A70008091C00085FFFCCF9093C6003196949151
:103A80009923B1F7E2E6F2E0949108C08091C0007A
:103A900085FFFCCF9093C600319694919923B1F79E
:103AA00009C08091C00085FFFCCF0894C11CD11CC7
:103AB0009093C600F6019081992399F78091C000F8
:103AC00085FFFCCF8AE08093C60056C0F801EB5515
:103AD000FE4F80818A3008F03EC08F5F8083282FA0
:103AE00030E0C9010197FC01A5E0EE0FFF1FAA9588
:103AF000E1F7E81BF90BED58FF4FE00FF11F2150E4
:103B00003040AF01415E5F4FBF018BE1DB010D90A3
:103B1000BD01DA010D92AD018150C1F79291829100
:103B20003296968F858F7F972115310541F7D80101
:103B3000AD58BF4FF70134968BE101900D92815043
:103B4000E1F70F581F4FF70182819381D8018D93C0
:103B50009C9301571040D801AC5ABF4FFE013596D7
:103B60008BE101900D928150E1F70E5A1F4F8B812E
:103B70009C81F80191838083CE0101961DDF6F96B1
:103B80000FB6F894DEBF0FBECDBFCF91DF911F916E
:103B90000F91FF90EF90DF90CF900895EF92FF92FA
:103BA0000F931F938C019DECE92E91E0F92EE00E0E
:103BB000F11EC7010E94466DC7010E94956DF80174
:103BC000108211821F910F91FF90EF900895CF9274
:103BD000DF92EF92FF920F931F93CF93DF937C01BD
:103BE0006B01DB010D900020E9F78D0101501040C1
:103BF000061B170BEDECF1E0EE0EFF1ED7011C9239
:103C0000E3E3FEEFEE0EFF1ECB016EE470E00E94D8
:103C1000DFCCEC01009731F4F8013197EC0DFD1D7C
:103C200086010EC060E270E00E94DFCC8C010F5F65
:103C30001F4FCE016AE270E00E94DFCCFC01319799
:103C40008DE081838AE082831382C70187539E4F70
:103C5000B8010E94C8758DEC91E0E80EF91ED701FD
:103C60008C91882319F1ECE8F2E0949108C08091DE
:103C7000C00085FFFCCF9093C600319694919923A4
:103C8000B1F7E3E9F2E0949108C08091C00085FFAC
:103C9000FCCF9093C600319694919923B1F780910F
:103CA000C00085FFFCCF8AE08093C600DF91CF91F2
:103CB0001F910F91FF90EF90DF90CF900895CF93D9
:103CC000DF93EC018EA5882309F43DC0E7ECF2E018
:103CD000949108C08091C00085FFFCCF9093C600EE
:103CE000319694919923B1F7C051DE4F48815981A3
:103CF0006A817B81C05FD14080ED98E02AE030E0AE
:103D00000E940953E5ECF2E0949108C08091C00054
:103D100085FFFCCF9093C600319694919923B1F71B
:103D2000C851DE4F488159816A817B81C85ED1408C
:103D300080ED98E02AE030E00E9409538091C000B5
:103D400085FFFCCF12C0E5EBF2E0949108C08091B2
:103D5000C00085FFFCCF9093C600319694919923C3
:103D6000B1F78091C00085FFFCCF8AE08093C60048
:103D7000C955DE4F68816623E1F0E9EAF2E09491EB
:103D800008C08091C00085FFFCCF9093C60031969B
:103D900094919923B1F780ED98E070E04AE050E00B
:103DA0000E9458538091C00085FFFCCF8AE0809329
:103DB000C600DF91CF9108952F923F924F925F926C
:103DC0006F927F928F929F92AF92BF92CF92DF922B
:103DD000EF92FF920F931F93DF93CF93CDB7DEB790
:103DE000AD970FB6F894DEBF0FBECDBF5C014B019F
:103DF0004DA7FC0186A5882309F4E1C13DEC432EC3
:103E000031E0532E4A0C5B1CC2010E94956DF501F6
:103E100012821A8A1D8A198A188A8DE294E09F8775
:103E20008E872EE4C22ED12CCA0CDB1C8FE290E0D0
:103E3000A80EB91EF601B182A08281ED9FEFA80EF7
:103E4000B91EF40180818F3209F08DC0C4016FE288
:103E500070E00E94DFCC7C010894E11CF11C3E0163
:103E60000894611C711C160178C0C7016FE270E0F4
:103E70000E94DFCC6C01009709F483C0E816F906B4
:103E800008F07FC08C010E191F09C301B701A801FA
:103E90000E94FFCC060D171DF8011082F30107C028
:103EA0008091C00085FFFCCF31969093C600908131
:103EB0009923B1F78091C00085FFFCCFFAE0F09321
:103EC000C600F101608171816115710519F460E02E
:103ED00070E002C06C5F7F4FCE014296A30121E0EB
:103EE0000E94CE74882371F5EBE7F3E0949108C04B
:103EF0008091C00085FFFCCF9093C60031969491CD
:103F00009923B1F7FE01319607C08091C00085FF6B
:103F1000FCCF31969093C60090819923B1F7E9E7E1
:103F2000F3E0949108C08091C00085FFFCCF90938E
:103F3000C600319694919923B1F78091C00085FF16
:103F4000FCCF37C18EE090E08C0F9D1FF101918373
:103F5000808376010894E11CF11C92E0E916F104DB
:103F600008F083CF0BC0E0E5F0E0AE0EBF1EF60117
:103F7000B182A08280EB9FEFA80EB91E082DF92C0C
:103F800001C00E2DF501E25BFF4F9DA5992309F4B9
:103F9000ADC0608171816115710519F460E070E058
:103FA00002C06C5F7F4FC201402F5F2D21E00E9455
:103FB000CE74882309F46AC0EEEDF1E0AE0EBF1EA8
:103FC000F50140815181628173818AE090E0A80E01
:103FD000B91EF501408351836283738388E19EEFAC
:103FE000A80EB91EEBE6F3E0949108C08091C000E2
:103FF00085FFFCCF9093C600319694919923B1F739
:10400000802F9F2D9C01F90107C08091C00085FF82
:10401000FCCF31969093C60090819923B1F7E3E6E7
:10402000F3E0949108C08091C00085FFFCCF90938D
:10403000C600319694919923B1F780ED98E02AE07B
:1040400030E00E9409538091C00085FFFCCF8AE0D8
:104050008093C600E0EFF1E0AE0EBF1EF5011082C6
:10406000118212821382E5E5F3E0949108C08091F9
:10407000C00085FFFCCF9093C600319694919923A0
:10408000B1F78091C00085FFFCCF93C0E1E4F3E07D
:10409000949108C08091C00085FFFCCF9093C6002A
:1040A000319694919923B1F7802F9F2D9C01F901AE
:1040B00007C08091C00085FFFCCF31969093C60069
:1040C00090819923B1F7EFE3F3E0949108C08091D8
:1040D000C00085FFFCCF9093C60031969491992340
:1040E000B1F78091C00085FFFCCF63C06081718112
:1040F0006115710519F460E070E002C06C5F7F4FDC
:10410000C201402F5F2D26E50E94CE74882381F5E1
:10411000EBE2F3E0949108C08091C00085FFFCCFF2
:104120009093C600319694919923B1F7802F9F2DDB
:104130009C01F90107C08091C00085FFFCCF31963A
:104140009093C60090819923B1F7E9E2F3E094914E
:1041500008C08091C00085FFFCCF9093C6003196C7
:1041600094919923B1F78091C00085FFFCCF21C0C5
:1041700081E0F5018083E7E1F3E0949108C080914C
:10418000C00085FFFCCF9093C6003196949199238F
:10419000B1F7F40107C08091C00085FFFCCF3196D4
:1041A0009093C60090819923B1F78091C00085FF5C
:1041B000FCCF8AE08093C600CE010E96FDDBAD9663
:1041C0000FB6F894DEBF0FBECDBFCF91DF911F9128
:1041D0000F91FF90EF90DF90CF90BF90AF909F90A6
:1041E0008F907F906F905F904F903F902F900895A9
:1041F000FC0181E08183CF0140E0DECD2F923F9230
:104200004F925F926F927F928F929F92AF92BF92E6
:10421000CF92DF92EF92FF920F931F93DF93CF9392
:10422000CDB7DEB7AC970FB6F894DEBF0FBECDBFEB
:104230005C014B01FC0186A5882309F437C1C50147
:1042400083539E4F0E94956DF50112821A8A1D8A32
:10425000198A188A8DE294E09F878E875EE4C52EC6
:10426000D12CCA0CDB1C2FE230E0A20EB31EF601EB
:10427000B182A08221ED3FEFA20EB31EF401808136
:104280008F3209F090C0C4016FE270E00E94DFCC71
:104290007C010894E11CF11C3E010894611C711C16
:1042A000260142E1242E312C2C0E3D1E77C0C70181
:1042B0006FE270E00E94DFCC6C01009709F481C0CE
:1042C000E816F90608F07DC08C010E191F09C3011C
:1042D000B701A8010E94FFCC060D171DF80110823E
:1042E000F30107C08091C00085FFFCCF3196909309
:1042F000C60090819923B1F78091C00085FFFCCF63
:10430000FAE0F093C600F2016081718161157105D8
:1043100019F460E070E002C06C5F7F4FC101A3013F
:1043200021E00E94CE74882371F5E3E0F3E09491DC
:1043300008C08091C00085FFFCCF9093C6003196E5
:1043400094919923B1F7FE01319607C08091C00086
:1043500085FFFCCF31969093C60090819923B1F7E9
:10436000E1E0F3E0949108C08091C00085FFFCCFAC
:104370009093C600319694919923B1F78091C00033
:1043800085FFFCCF8DC02EE030E02C0F3D1FF201E9
:104390003183208376010894E11CF11CE114F104BF
:1043A00009F085CF0BC080E590E0A80EB91EF6019C
:1043B000B182A08220EB3FEFA20EB31ED82C092DB4
:1043C00002C0DE2C0F2D8EE490E0A80EB91EF50180
:1043D0008081918122EB3FEFA20EB31E009719F46A
:1043E00080E090E001C004966D2D702F0E949A75B8
:1043F000882339F1E3EFF2E0949108C08091C00086
:1044000085FFFCCF9093C600319694919923B1F724
:104410008D2D902F9C01F90107C08091C00085FF70
:10442000FCCF31969093C60090819923B1F780EF2D
:1044300091E0A80EB91EF50110821182128213823A
:1044400032C0EBEDF2E0949108C08091C00085FF8E
:10445000FCCF9093C600319694919923B1F78D2D9E
:10446000902F9C01F90107C08091C00085FFFCCF0F
:1044700031969093C60090819923B1F7E9EDF2E06F
:10448000949108C08091C00085FFFCCF9093C60036
:10449000319694919923B1F78091C00085FFFCCFAC
:1044A0008AE08093C600CE010E9686DAAC960FB6EF
:1044B000F894DEBF0FBECDBFCF91DF911F910F915A
:1044C000FF90EF90DF90CF90BF90AF909F908F9034
:1044D0007F906F905F904F903F902F900895EF9254
:1044E000FF920F931F93CF93DF938C01FC0116A6CD
:1044F00086A9882321F0C801C3960E94956D66EABB
:10450000E62E61E0F62EE00EF11EC70160E045E305
:104510000E94696B882309F5ECE5F2E0949108C0EC
:104520008091C00085FFFCCF9093C6003196949196
:104530009923B1F7EDEBF3E0949108C08091C000AE
:1045400085FFFCCF9093C600319694919923B1F7E3
:104550008091C00085FFFCCF7DC0E801C555DE4FCE
:10456000CE01B70141E00E946576882341F5CE0176
:10457000B70140E00E946576882309F5ECE8F2E097
:10458000949108C08091C00085FFFCCF9093C60035
:10459000319694919923B1F7EAEAF3E0949108C037
:1045A0008091C00085FFFCCF9093C6003196949116
:1045B0009923B1F78091C00085FFFCCF4BC0C801A3
:1045C000C396BE010E946C70882309F5ECE8F2E006
:1045D000949108C08091C00085FFFCCF9093C600E5
:1045E000319694919923B1F7EAE9F3E0949108C0E8
:1045F0008091C00085FFFCCF9093C60031969491C6
:104600009923B1F78091C00085FFFCCF23C081E0E2
:10461000F80186A7ECE5F2E0949108C08091C00013
:1046200085FFFCCF9093C600319694919923B1F702
:10463000EFE8F3E0949108C08091C00085FFFCCFC3
:104640009093C600319694919923B1F78091C00060
:1046500085FFFCCF8AE08093C600D801AC5ABF4FDB
:10466000F801F3968BE101900D928150E1F7F8018A
:1046700081A992A90E5A1F4FF80191838083025598
:104680001040C8018F96025B1F4FF8019183808311
:10469000DF91CF911F910F91FF90EF9008952F928E
:1046A0003F924F925F926F927F929F92AF92BF9292
:1046B000CF92DF92EF92FF920F931F93DF93CF93EE
:1046C000CDB7DEB7CC55D0400FB6F894DEBF0FBEE5
:1046D000CDBF6C01662311F524EF31E0C20ED31E6D
:1046E000D6018C91ECE0FEEFCE0EDF1E882309F49C
:1046F000E7C02CEE31E0C20ED31ED601ED90FD9046
:104700000D911C91E4E1FEEFCE0EDF1E0E94171A00
:10471000E616F7060807190708F4D2C024EF31E0BF
:10472000C20ED31ED6011C92ECE0FEEFCE0EDF1EB1
:10473000D6019E968C91882339F4C601D0DEF6010D
:1047400086A5882309F4BCC000D000D0EDB7FEB721
:1047500031967E010894E11CF11CADB7BEB71296EC
:10476000FC92EE92119783E892E093838283D601C4
:104770009C968D919C919D97958384830E943FCDBB
:104780008701EDB7FEB736960FB6F894FEBF0FBEA1
:10479000EDBF570108C0D8018C9190E00E945DCC1C
:1047A000F80181938F01F50101900020E9F731971D
:1047B000EA19FB09802F8E198E176CF3A3E3AA2E3A
:1047C000B12CAC0CBD1CC50140E050E060E070E0D5
:1047D0000E947C6C9924FDE3EF2EF12CEC0EFD1E63
:1047E0002E010894411C511CEFE16E2E712C6C0EB1
:1047F0007D1E7CE7272E72E0372E42C0D8018C91B7
:1048000090E00E945DCCF80181938F01F701019047
:104810000020E9F73197EE19FF09802F8E198E17C6
:104820006CF327968FAD27978E3751F1C701B201F0
:1048300045E050E00E94F1CC009711F500D000D087
:10484000EDB7FEB73196ADB7BEB712967C926E92B9
:10485000119733822282558244820E943FCDEDB768
:10486000FEB736960FB6F894FEBF0FBEEDBFC3017C
:104870000E94695188E792E00E94F0509924939435
:10488000C501B70140E050E00E948B6F181614F488
:104890008701BCCF992041F48FEF9FEFD6019D9601
:1048A0009C938E939C9706C0F60184A595A50196CE
:1048B00095A784A727EA31E0C20ED31ED6011C9229
:1048C000C45ADF4F0FB6F894DEBF0FBECDBFCF91F5
:1048D000DF911F910F91FF90EF90DF90CF90BF90ED
:1048E000AF909F907F906F905F904F903F902F90F0
:1048F00008952F923F924F925F926F927F928F9284
:104900009F92AF92BF92CF92DF92EF92FF920F935E
:104910001F93DF93CF93CDB7DEB7CD58D0400FB6FE
:10492000F894DEBF0FBECDBF8C013B016A0184E06D
:1049300090E0C80ED91EF8017096C757DF4FF98373
:10494000E883C958D040C8010396C957DF4F9983FF
:104950008883C758D040CA57DF4F1882C658D04006
:1049600036E6E32EF12CEC0EFD1E25EF822E21E023
:10497000922E800E911E96EFA92E91E0B92EA00ED8
:10498000B11E8EE0282E312C2C0E3D1EB7E44B2E8E
:10499000512C4C0E5D1EF2013496C557DF4FF98342
:1049A000E883CB58D040ECE5F2E08491C357DF4F69
:1049B0008883CD58D04021C1F7018385282F30E06E
:1049C000A901487150704031510509F024C1F4012A
:1049D0009081913009F41FC1923009F41CC1CE01BD
:1049E0000196B7010E944A1C1E86F301808188232C
:1049F00029F4C10160E072E00E94D4CCC101B3018E
:104A00000E94D4CCC101BE016F5F7F4F0E94D4CC05
:104A1000C10160E072E00E94D4CC1CA61FA61BA6B8
:104A20001AA68DE294E099A788A7CE018C96B601CC
:104A3000AE014F5F5F4F21E00E94CE74882309F0E2
:104A40003EC0F40180818823D1F5C357DF4F9881A0
:104A5000CD58D040ECE5F2E008C08091C00085FF61
:104A6000FCCF9093C600319694919923B1F7E2E080
:104A7000F2E007C08091C00085FFFCCF3196909393
:104A8000C60090819923B1F78091C00085FFFCCFCB
:104A9000FAE0F093C600FE01319607C08091C00095
:104AA00085FFFCCF31969093C60090819923B1F792
:104AB0008091C00085FFFCCF8AE08093C600C55777
:104AC000DF4FA881B981CB58D040FE01BC968BE165
:104AD00001900D928150E1F78AA59BA5F201938385
:104AE00082838DE294E091838083C801B101A201A9
:104AF00000DFC2010E94DC1CCE0188960E94DC1CF3
:104B00007CC0953E09F479C09E3209F476C09F3589
:104B100009F473C0F8019089992331F09E3209F4A9
:104B20006CC09F3509F469C023FD67C080E0403147
:104B3000510509F481E0F80183A7882349F4F701BE
:104B40008085873409F059C081858E3709F455C0B6
:104B5000C957DF4F88819981C758D040B7010E945B
:104B60004A1CF4018081882329F5F30107C0809154
:104B7000C00085FFFCCF31969093C60090819923A9
:104B8000B1F7C957DF4FE881F981C758D04007C056
:104B90008091C00085FFFCCF31969093C600908134
:104BA0009923B1F78091C00085FFFCCFFAE0F09324
:104BB000C60023C0813039F4F501808191810196CE
:104BC000918380831AC08230C1F4CA57DF4FF881C5
:104BD000C658D0402F2F30E0F501808191812817F1
:104BE0003907F1F0CA57DF4FF881C658D040FF5F50
:104BF000CA57DF4FF883C658D040C601B701C75720
:104C0000DF4F48815981C958D0400E948B6F1816D8
:104C10000CF4D2CE05C0F7019081992309F071CF31
:104C2000C357DF4F0FB6F894DEBF0FBECDBFCF9195
:104C3000DF911F910F91FF90EF90DF90CF90BF9089
:104C4000AF909F908F907F906F905F904F903F902C
:104C50002F900895EF92FF920F931F93DF93CF93BE
:104C6000CDB7DEB76F970FB6F894DEBF0FBECDBFDE
:104C70007C018C01025B1F4F805B9F4FF801918389
:104C8000808325EF31E0E20EF31E21E0F70121934E
:104C90007F01118210822AE03EEFE20EF31E04969D
:104CA00040E050E060E070E00E947C6CF801208100
:104CB0003181DE011596F90134968BE101900D9258
:104CC0008150E1F7F901828193819C838B838DE28E
:104CD00094E09A838983C70165E172E08E010F5FDA
:104CE0001F4FA80106DEC8010E94DC1CF701EA5034
:104CF000FE4F808191816F960FB6F894DEBF0FBE94
:104D0000CDBFCF91DF911F910F91FF90EF9008954C
:104D1000EF92FF920F931F93DF93CF93CDB7DEB740
:104D20006F970FB6F894DEBF0FBECDBF7C018C012C
:104D3000025B1F4F805B9F4FF8019183808325EFBB
:104D400031E0E20EF31E22E0F70120832BE03EEF7C
:104D5000E20EF31EF701EA50FE4F608311820496C3
:104D600040E050E060E070E00E947C6CF80120813F
:104D70003181DE011596F90134968BE101900D9297
:104D80008150E1F7F901828193819C838B838DE2CD
:104D900094E09A838983C70165E172E08E010F5F19
:104DA0001F4FA801A6DDC8010E94DC1C6F960FB63C
:104DB000F894DEBF0FBECDBFCF91DF911F910F9151
:104DC000FF90EF900895EF92FF920F931F93DF9360
:104DD000CF93CDB7DEB76F970FB6F894DEBF0FBE97
:104DE000CDBF7C0185EF91E0E80EF91EF70110823E
:104DF0008BE09EEFE80EF91E87010D5C1F4FC80186
:104E000040E050E060E070E00E947C6CDE011596AE
:104E1000F8018BE101900D928150E1F7F70181A932
:104E200092A99C838B838DE294E09A838983C70146
:104E300065E172E08E010F5F1F4FA8015ADDC801C6
:104E40000E94DC1C6F960FB6F894DEBF0FBECDBF7C
:104E5000CF91DF911F910F91FF90EF9008950F93E5
:104E60001F93CF93DF93DC01D3961C92D397D696F2
:104E70001C92D697D2961C921E92D1978DE294E006
:104E8000D0969C938E939F97AC5ABF4F1C921396CB
:104E90001C92A755B040FD01E05BFF4FAE5ABF4FDB
:104EA00011961C921E92A255B04091838083ED0111
:104EB000C159DF4FFE0120E030E0482F14821782F5
:104EC0001382128240839183215E3F4F7F9681E05F
:104ED0002633380799F7A955BE4F89E18C9313966D
:104EE0001C9258961C921B961C9213961C92A05DC5
:104EF000B140FD01E753FE4FA553BE4F11961C92E2
:104F00001E92408391835D961D921D921D921C926C
:104F1000139718961D921D921D921C921397A05FD5
:104F2000B14012961C9212979E961C929E971C92CC
:104F300011961C9211978D0104511E4FF801108299
:104F4000118212821382AB55BE4F1C92FE01C90121
:104F500011920197E9F7A15BBF4F81E08C93A45FA9
:104F6000B1409D961C921E929C970E94171A6857FA
:104F70007C4E8F4F9F4FF8016083718382839383B0
:104F8000DF91CF911F910F910895DF93CF93CDB70C
:104F9000DEB7E0970FB6F894DEBF0FBECDBFDE01DF
:104FA0001196EDEDF3E080E101900D928150E1F773
:104FB000DE015196EDECF3E080E101900D9281501D
:104FC000E1F7DE019196EDEBF3E080E101900D92C7
:104FD0008150E1F789819A81AB81BC818093E5089A
:104FE0009093E608A093E708B093E80889899A8926
:104FF000AB89BC898093D5089093D608A093D70835
:10500000B093D80889A19AA1ABA1BCA18093F5085F
:105010009093F608A093F708B093F8088D819E81CD
:10502000AF81B8858093E9089093EA08A093EB08D4
:10503000B093EC088D899E89AF89B88D8093D9088B
:105040009093DA08A093DB08B093DC088DA19EA1B1
:10505000AFA1B8A58093F9089093FA08A093FB0834
:10506000B093FC0889859A85AB85BC858093ED0853
:105070009093EE08A093EF08B093F008898D9A8D75
:10508000AB8DBC8D8093DD089093DE08A093DF0884
:10509000B093E00889A59AA5ABA5BCA58093FD08AF
:1050A0009093FE08A093FF08B09300098D859E851C
:1050B000AF85B8898093F1089093F208A093F30824
:1050C000B093F4088D8D9E8DAF8DB8A18093E108CB
:1050D0009093E208A093E308B093E4088DA59EA501
:1050E000AFA5B8A98093010990930209A093030981
:1050F000B09304090E94BA5780E090E4ACE9B5E4AB
:105100008093090990930A09A0930B09B0930C09A5
:1051100080930D0990930E09A0930F09B093100985
:1051200020E030E040E050E020930509309306098C
:10513000409307095093080980E29EE4A0E0B0E0A4
:105140008093D1089093D208A093D308B093D40849
:1051500020931D0930931E0940931F095093200985
:1051600080E090E0A0EAB1E48093110990931209E5
:10517000A0931309B09314098DEC9CECACECBEE346
:105180008093150990931609A0931709B0931809F5
:1051900080E090E0A0EAB0E48093190990931A09A6
:1051A000A0931B09B0931C0920935C0630935D0605
:1051B00040935E0650935F0620935806309359063D
:1051C00040935A0650935B0620935406309355063D
:1051D000409356065093570686E696E6A2E4B1E45D
:1051E00080938D0390938E03A0938F03B0939003CD
:1051F00060E070E080E89FE30E9417846093910371
:105200007093920380939303909394036BE774E1FC
:1052100084E192E40E942384609395037093960343
:1052200080939703909398030E941F8380E090E0FF
:10523000A0E8BFE38093990390939A03A0939B0304
:10524000B0939C0384E195E0909383038093820361
:10525000909385038093840382EE94E09093870378
:105260008093860384E68093B1031092E710EAEC02
:10527000F3E0949108C08091C00085FFFCCF90932B
:10528000C600319694919923B1F7E0EDF3E0949143
:1052900008C08091C00085FFFCCF9093C600319676
:1052A00094919923B1F78091C00085FFFCCF8AE0EB
:1052B0008093C600E0960FB6F894DEBF0FBECDBF58
:1052C000CF91DF910895CF93DF93CAECD3E0FE0135
:1052D000949108C08091C00085FFFCCF9093C600D8
:1052E000319694919923B1F7E4ECF5E0949108C0DC
:1052F0008091C00085FFFCCF9093C60031969491B9
:105300009923B1F78091C00085FFFCCF8AE080939C
:10531000C600FE019491EAECF3E008C08091C00061
:1053200085FFFCCF9093C600319694919923B1F7F5
:105330004091E5085091E6086091E7087091E8080F
:105340008CEB95E00E9401344091E9085091EA0805
:105350006091EB087091EC0889EB95E00E940134B4
:105360004091ED085091EE086091EF087091F008BF
:1053700086EB95E00E9401344091F1085091F208CB
:105380006091F3087091F40883EB95E00E9401347A
:10539000E6E1F2E007C08091C00085FFFCCF3196C6
:1053A0009093C60090819923B1F78091C00085FF4A
:1053B000FCCF8AE08093C600FE019491EAECF3E012
:1053C00008C08091C00085FFFCCF9093C600319645
:1053D00094919923B1F7E9E9F5E0949108C080919F
:1053E000C00085FFFCCF9093C6003196949199231D
:1053F000B1F78091C00085FFFCCF8AE08093C600A2
:10540000FE019491EAECF3E008C08091C00085FFB2
:10541000FCCF9093C600319694919923B1F74091B7
:10542000D5085091D6086091D7087091D80880E9C6
:1054300095E00E9401344091D9085091DA086091BA
:10544000DB087091DC088DE895E00E940134409102
:10545000DD085091DE086091DF087091E0088AE86D
:1054600095E00E9401344091E1085091E20860917A
:10547000E3087091E40887E895E00E940134E6E1D2
:10548000F2E007C08091C00085FFFCCF3196909379
:10549000C60090819923B1F78091C00085FFFCCFB1
:1054A0008AE08093C600FE019491EAECF3E008C024
:1054B0008091C00085FFFCCF9093C60031969491F7
:1054C0009923B1F7E9E6F5E0949108C08091C00016
:1054D00085FFFCCF9093C600319694919923B1F744
:1054E0008091C00085FFFCCF8AE08093C600FE015A
:1054F0009491EAECF3E008C08091C00085FFFCCFF6
:105500009093C600319694919923B1F74091F50894
:105510005091F6086091F7087091F80880E695E0E0
:105520000E9414344091F9085091FA086091FB08E8
:105530007091FC088DE595E00E9414344091FD08BF
:105540005091FE086091FF08709100098AE595E08E
:105550000E9414344091010950910209609103099D
:105560007091040987E595E00E941434E6E1F2E0C9
:1055700007C08091C00085FFFCCF31969093C60094
:1055800090819923B1F78091C00085FFFCCF8AE01C
:105590008093C600FE019491EAECF3E008C080918C
:1055A000C00085FFFCCF9093C6003196949199235B
:1055B000B1F7E2E2F5E0949108C08091C00085FF68
:1055C000FCCF9093C600319694919923B1F78091C6
:1055D000C00085FFFCCF8AE08093C600FE01949155
:1055E000EAECF3E008C08091C00085FFFCCF909307
:1055F000C600319694919923B1F7409109095091D1
:105600000A0960910B0970910C0989E195E00E94EB
:10561000013440910D0950910E0960910F0970916C
:10562000100986E195E00E940134E6E1F2E007C04E
:105630008091C00085FFFCCF31969093C600908189
:105640009923B1F78091C00085FFFCCF8AE0809359
:10565000C600FE019491EAECF3E008C08091C0001E
:1056600085FFFCCF9093C600319694919923B1F7B2
:10567000E3E6F4E0949108C08091C00085FFFCCF80
:105680009093C600319694919923B1F78091C00010
:1056900085FFFCCF8AE08093C600FE019491EAEC7E
:1056A000F3E008C08091C00085FFFCCF9093C60056
:1056B000319694919923B1F74091050950910609CB
:1056C00060910709709108098AE594E00E9401340D
:1056D00040911D0950911E0960911F097091200988
:1056E00087E594E00E9401344091D1085091D2089E
:1056F0006091D3087091D40884E594E00E9414343A
:105700004091110950911209609113097091140987
:1057100081E594E00E9401344091150950911609E9
:1057200060911709709118098EE494E00E94013489
:105730004091190950911A0960911B0970911C0937
:105740008BE494E00E940134E6E1F2E007C080912E
:10575000C00085FFFCCF31969093C60090819923BD
:10576000B1F78091C00085FFFCCF8AE08093C6002E
:10577000FE019491EAECF3E008C08091C00085FF3F
:10578000FCCF9093C600319694919923B1F7E9E349
:10579000F4E0949108C08091C00085FFFCCF909305
:1057A000C600319694919923B1F78091C00085FF8E
:1057B000FCCF8AE08093C600FE019491EAECF3E00E
:1057C00008C08091C00085FFFCCF9093C600319641
:1057D00094919923B1F740915406509155066091E8
:1057E00056067091570680E394E00E940134409180
:1057F00058065091590660915A0670915B068DE2E9
:1058000094E0FFD740915C0650915D0660915E0682
:1058100070915F068AE294E0F4D7E6E1F2E007C017
:105820008091C00085FFFCCF31969093C600908197
:105830009923B1F78091C00085FFFCCF8AE0809367
:10584000C600FE019491EAECF3E008C08091C0002C
:1058500085FFFCCF9093C600319694919923B1F7C0
:10586000ECE1F4E0949108C08091C00085FFFCCF8A
:105870009093C600319694919923B1F78091C0001E
:1058800085FFFCCF8AE08093C600FE019491EAEC8C
:10589000F3E008C08091C00085FFFCCF9093C60064
:1058A000319694919923B1F740918D0350918E03D5
:1058B00060918F037091900382E194E0A2D7609190
:1058C00091037091920380919303909194030E94AD
:1058D0001D84AB01BC018FE094E093D760919503E8
:1058E0007091960380919703909198030E94298468
:1058F000AB01BC018CE094E084D7E6E1F2E007C0A4
:105900008091C00085FFFCCF31969093C6009081B6
:105910009923B1F78091C00085FFFCCF8AE0809386
:10592000C600DF91CF910895EF92FF921F93CF931E
:10593000DF93EC017B01142F888199810E94D5D3DC
:10594000F70181937F0188819981019699838883EA
:10595000115091F7DF91CF911F91FF90EF90089533
:10596000EF92FF920F931F93DF93CF93CDB7DEB7E4
:1059700066970FB6F894DEBF0FBECDBF84E690E009
:105980009A8389838091170290911802A09119023D
:10599000B0911A028B8B9C8BAD8BBE8B8E01015FFD
:1059A0001F4F7E010894E11CF11CC701B80144E0BF
:1059B000BBDFCE014396B80143E050E00E94F1CC3A
:1059C000009709F0A6C0C70165EE78E040E1ACDFC2
:1059D000C70165ED78E040E1A7DFC70165EF78E03A
:1059E00040E1A2DF0E94BA57C70169E079E044E0D4
:1059F0009BDFC7016DE079E044E096DFC70165E019
:105A000079E044E091DFC7016DE179E044E08CDFAB
:105A1000C70161ED78E044E087DFC70161E179E02B
:105A200044E082DFC70165E179E044E07DDFC70142
:105A300069E179E044E078DFC70164E576E04CE0B5
:105A400073DFC701BE016D5F7F4F42E06DDFC701AD
:105A5000BE016B5F7F4F42E067DFC701BE01695F38
:105A60007F4F42E061DFC701BE01675F7F4F42E0C9
:105A70005BDFC701BE01655F7F4F42E055DFC701B5
:105A8000BE01635F7F4F42E04FDFC7016DE873E007
:105A900044E04ADFC70161E973E044E045DFC70144
:105AA00065E973E044E040DFC70162E873E046E087
:105AB0003BDFC70161EB73E041E036DFC70167EE12
:105AC00070E141E031DF0E941F83EAECF3E0949142
:105AD00008C08091C00085FFFCCF9093C60031962E
:105AE00094919923B1F7E2EFF3E0949108C080918B
:105AF000C00085FFFCCF9093C60031969491992306
:105B0000B1F78091C00085FFFCCF8AE08093C6008A
:105B100001C03BDAD8DB66960FB6F894DEBF0FBE45
:105B2000CDBFCF91DF911F910F91FF90EF9008951E
:105B3000EF92FF921F93CF93DF93EC017B01142F21
:105B400088819981F70161917F010E94F0D388815A
:105B50009981019699838883115091F7DF91CF91B4
:105B60001F91FF90EF900895EF92FF920F931F9374
:105B7000DF93CF93CDB7DEB766970FB6F894DEBF4D
:105B80000FBECDBF80911B0290911C02A0911D02FF
:105B9000B0911E028F87988BA98BBA8B84E6E82E72
:105BA000F12CFA82E9828E010F5F1F4FC801BE01FE
:105BB000615F7F4F44E0BCDFC80165EE78E040E103
:105BC000B7DFC80165ED78E040E1B2DFC80165EFFD
:105BD00078E040E1ADDFC80169E079E044E0A8DFAA
:105BE000C8016DE079E044E0A3DFC80165E079E039
:105BF00044E09EDFC8016DE179E044E099DFC8012F
:105C000061ED78E044E094DFC80161E179E044E0CF
:105C10008FDFC80165E179E044E08ADFC80169E10E
:105C200079E044E085DFC80164E576E04CE080DFA0
:105C300084EB90E09C838B8386E490E09E838D834D
:105C400018861F8280EF90E09A878987FC86EB8612
:105C50001E861D86C801BE016D5F7F4F42E068DF72
:105C6000C801BE016B5F7F4F42E062DFC801BE0129
:105C7000695F7F4F42E05CDFC801BE01675F7F4F15
:105C800042E056DFC801BE01655F7F4F42E050DF52
:105C9000C801BE01635F7F4F42E04ADFC8016DE883
:105CA00073E044E045DFC80161E973E044E040DFB0
:105CB000C80165E973E044E03BDFC80162E873E0D6
:105CC00046E036DFC80161EB73E041E031DFC80137
:105CD00067EE70E141E02CDF80911702909118028D
:105CE000A0911902B0911A028B8B9C8BAD8BBE8B4D
:105CF000FA82E982C801BE016D5E7F4F44E018DF81
:105D0000EAECF3E0949108C08091C00085FFFCCFDD
:105D10009093C600319694919923B1F7E4EDF5E0A4
:105D2000949108C08091C00085FFFCCF9093C6007D
:105D3000319694919923B1F78091C00085FFFCCFF3
:105D40008AE08093C60066960FB6F894DEBF0FBE59
:105D5000CDBFCF91DF911F910F91FF90EF900895EC
:105D6000DF93CF930F920F92CDB7DEB72091C71577
:105D70003091C815CE0101962115310519F4835DC6
:105D8000954102C0821B930B9A83898389819A81F2
:105D90000F900F90CF91DF91089520E080914608F9
:105DA00090914708181619060CF421E0822F0895E7
:105DB000AF92BF92CF92DF92EF92FF920F931F9319
:105DC0008C01000F111F000F111FF801E351F84F54
:105DD0006591759185919491F801EC5AF94FC080C5
:105DE000D180E280F38034E4A32E36E0B32EA00EFF
:105DF000B11EA70196010E9470CDF50160837183E9
:105E000082839383F801E750F84F659175918591EE
:105E1000949120E6A22E26E0B22EA00EB11EA7017C
:105E200096010E9470CDF501608371838283938314
:105E3000F801EB5FF74F65917591859194910C5A3C
:105E40001C4FA70196010E9470CDF80160837183F9
:105E5000828393831F910F91FF90EF90DF90CF90FB
:105E6000BF90AF900895EF92FF920F931F93CF933F
:105E7000DF93EC01E0906006F0906106009162060D
:105E800010916306688179818A819B81A8019701BD
:105E90000E9449CE882324F4E882F9820A831B8376
:105EA000E0906406F0906506009166061091670622
:105EB0006C817D818E819F81A80197010E9449CECE
:105EC000882324F4EC82FD820E831F83E090680611
:105ED000F090690600916A0610916B0668857985D5
:105EE0008A859B85A80197010E9449CE882324F4C6
:105EF000E886F9860A871B87E0905403F0905503E3
:105F00000091560310915703688179818A819B81A2
:105F1000A80197010E944CD0181624F4E882F98257
:105F20000A831B83E0905803F090590300915A03B1
:105F300010915B036C817D818E819F81A801970107
:105F40000E944CD0181624F4EC82FD820E831F832D
:105F5000E0905C03F0905D0300915E0310915F039D
:105F6000688579858A859B85A80197010E944CD018
:105F7000181624F4E886F9860A871B87DF91CF91EB
:105F80001F910F91FF90EF90089580917D068111F0
:105F900081E0089580917D060895CF93DF9381304D
:105FA000910541F46F5F7F4FF9F484E494E00E941F
:105FB0002F271AC0892BC1F46F5F7F4FA9F48DE0A2
:105FC00096E00E94DC1CCAECD5E0CE010E94DC1CED
:105FD0006F9784E0C439D807C1F7CE010E94DC1C5A
:105FE000CE0181970E94DC1CDF91CF91089580E063
:105FF00090E06FEF7FEFD1CF81E090E06FEF7FEF28
:10600000CCCF1F93182F0E94088480917D0688238F
:1060100009F035C010937D0680917F06909180062F
:10602000A0918106B09182068093830690938406A6
:10603000A0938506B0938606EAEEF5E0949108C039
:106040008091C00085FFFCCF9093C600319694915B
:106050009923B1F7E1EFF5E0949108C08091C00079
:1060600085FFFCCF9093C600319694919923B1F7A8
:106070008091C00085FFFCCF8AE08093C6001F910D
:106080000895F8940E940884159A469A439A409A73
:106090008CE060E00E94651BEAEEF5E0949108C098
:1060A0008091C00085FFFCCF9093C60031969491FB
:1060B0009923B1F7E7E6F6E0949108C08091C0001B
:1060C00085FFFCCF9093C600319694919923B1F748
:1060D0008091C00085FFFCCF8AE08093C600FFCF8F
:1060E0000E94171A6093870670938806809389062A
:1060F00090938A06E091B006F091B106EE54F94F04
:1061000080818823A9F4E6E8F6E0949108C08091A4
:10611000C00085FFFCCF9093C600319694919923DF
:10612000B1F78091C00085FFFCCF8AE08093C60064
:106130000895EF92FF920F931F930E94171AE09019
:106140008B06F0908C0600918D0610918E062091A2
:106150008706309188064091890650918A06621B15
:10616000730B840B950BE616F7060807190730F436
:10617000E114F1040105110509F083DF8091710339
:1061800090917203A0917303B09174030097A105DD
:10619000B105F9F00E94171A209187063091880600
:1061A0004091890650918A06621B730B840B950BF4
:1061B00020917103309172034091730350917403E5
:1061C000261737074807590720F48091110E809150
:1061D000120E069B02C08AE014DF0E943B5A1F91F8
:1061E0000F91FF90EF9008956F927F928F929F9200
:1061F000AF92BF92CF92DF92EF92FF920F931F93D5
:10620000F82E60918F067091900680919106909182
:1062100092062091930630919406409195065091F4
:1062200096060E9459D03B014C0100D000D00DB71A
:106230001EB70F5F1F4F6091500370915103882765
:1062400077FD8095982F0E94EBCE209175033091B9
:10625000760340917703509178030E941ED120E08D
:1062600030E040E752E40E9450CE20E030E048ECBD
:1062700052E40E9450CE5B016C01F8016082718291
:1062800082829382F48280916C06858384E496E016
:106290006BE976E04FE856E020E001E0E2E0EE2E28
:1062A0000E942D5480919B0690919C06A0919D0682
:1062B000B0919E068093440690934506A0934606AF
:1062C000B093470680919F069091A006A091A106E9
:1062D000B091A2068093480690934906A0934A067F
:1062E000B0934B068091A3069091A406A091A506B9
:1062F000B091A60680934C0690934D06A0934E064F
:10630000B0934F068091A7069091A806A091A90688
:10631000B091AA068093500690935106A09352061E
:10632000B09353068DB79EB706960FB6F8949EBFEE
:106330000FBE8DBF0E94171A609387067093880660
:106340008093890690938A061F910F91FF90EF909A
:10635000DF90CF90BF90AF909F908F907F906F9085
:106360000895CF92DF92EF92FF920F931F938BE9E4
:1063700096E079DD0E94171A60938706709388066D
:106380008093890690938A06609144067091450631
:10639000809146069091470620919B0630919C067D
:1063A00040919D0650919E060E9449CE882309F097
:1063B0007AC0609148067091490680914A06909192
:1063C0004B0620919F063091A0064091A106509166
:1063D000A2060E9449CE882309F065C0609175032A
:1063E00070917603809177039091780320E030E0FC
:1063F00040E752E40E9450CE7B018C018BE996E08D
:106400006FE976E043EA56E027EA36E0FCE6CF2E75
:10641000F6E0DF2E0E94215D80919B0690919C0604
:10642000A0919D06B0919E068093440690934506E8
:10643000A0934606B093470680919F069091A006D0
:10644000A091A106B091A2068093480690934906B8
:10645000A0934A06B0934B068091A3069091A406A0
:10646000A091A506B091A60680934C0690934D0688
:10647000A0934E06B0934F068091A7069091A80670
:10648000A091A906B091AA06809350069093510658
:10649000A0935206B09353061F910F91FF90EF9077
:1064A000DF90CF9008956091500370915103882739
:1064B00077FD8095982F0E94EBCE20917503309147
:1064C000760340917703509178030E941ED120E01B
:1064D00030E040E752E40E9450CE20E030E048EC4B
:1064E00052E488CF80ED98E00E946952E9E8F6E036
:1064F000949108C08091C00085FFFCCF9093C600A6
:10650000319694919923B1F740917F06509180067E
:1065100060918106709182064F5F5F4F6F4F7F4F92
:1065200080ED98E02AE030E00E9425538091C00081
:1065300085FFFCCF8AE08093C600D2CD2F923F9298
:106540004F925F926F927F928F929F92AF92BF9283
:10655000CF92DF92EF92FF920F931F93DF93CF932F
:1065600000D000D0CDB7DEB79E838D8383309105F8
:1065700008F010C15C01AA0CBB1CAA0CBB1CC50115
:106580008C5B994F9A83898380E090E0A0E0B0E033
:10659000E981FA8180839183A283B38384E496E0C6
:1065A00068E476E04CE456E020E536E00E940C58C2
:1065B000F501EF5EF74F6591759185919491ED81AD
:1065C000FE81E75DF74FD490BBE92B2EB6E03B2E62
:1065D0002A0C3B1C20E030E040EC5FE30E941ED11F
:1065E0007B018C016D2D772767FD7095872F972F85
:1065F0000E94EBCE2B013C01C801B701A30192011F
:106600000E941ED1D1016D937D938D939C9313971E
:10661000F501E05CFC4FFC83EB836081718182813A
:1066200093816093750370937603809377039093BF
:10663000780320E030E040E752E40E9450CE7B0136
:106640008C018BE996E06FE976E043EA56E027EAB1
:1066500036E0ACE6CA2EA6E0DA2E0E94215D0E944A
:10666000087C80E090E0A0E0B0E0E981FA818083DE
:106670009183A283B38384E496E068E476E04CE4FB
:1066800056E020E536E00E940C588DE198E0A80E17
:10669000B91EF50185909590A590B490C501B401FF
:1066A0009058A30192010E941ED1D1016D937D9358
:1066B0008D939C93139760917503709176038091ED
:1066C00077039091780320E030E040E752E40E94A5
:1066D00050CE7B018C018BE996E06FE976E043EACE
:1066E00056E027EA36E00E94215D0E94087CC50141
:1066F000B401A50194010E9470CDA30192010E94F2
:106700001ED1F1016083718382839383AB81BC814D
:106710006D917D918D919C9120E030E040E450E4BA
:106720000E9450CE60937503709376038093770335
:106730009093780320E030E040E752E40E9450CE8E
:106740007B018C018BE996E06FE976E043EA56E045
:1067500027EA36E00E94215D0E94087C8D819E819F
:1067600027DBE981FA8180819181A281B381F101E6
:1067700080839183A283B38380E090E0A0E0B0E0C7
:106780008093750390937603A0937703B093780377
:106790000E94977A26960FB6F894DEBF0FBECDBF43
:1067A000CF91DF911F910F91FF90EF90DF90CF90ED
:1067B000BF90AF909F908F907F906F905F904F9021
:1067C0003F902F900895682F2091B0063091B10628
:1067D00080E690E0AC01249FC001259F900D349F7E
:1067E000900D11248454994F70E00E94DFCC9C01DD
:1067F0009093BB068093BA0680E0232B09F081E0DA
:106800000895FC01949108C08091C00085FFFCCFE1
:106810009093C600319694919923B1F780ED98E05A
:1068200022E030E00C942B54FC01949108C080913C
:10683000C00085FFFCCF9093C600319694919923B8
:10684000B1F780ED98E02AE030E00C940953809194
:10685000BA069091BB06019660E070E04AE050E015
:106860000C94FECA8091BA069091BB06019660E036
:1068700070E00C9498C9CF93DF93EC0180916C0683
:1068800080937E0684E59FDF882309F46EC0EADFEB
:106890000E94BDCE262F60937E06662309F465C054
:1068A000E4EEF5E0949108C08091C00085FFFCCF34
:1068B0009093C600319694919923B1F7C936D105CA
:1068C00099F0CA36D10524F4C836D105F1F50FC0C8
:1068D000CD36D10531F0CA3DD105B9F5EFE1F2E091
:1068E00031C0E6E3F2E023C0EDE4F2E015C0E4E6F7
:1068F000F2E007C08091C00085FFFCCF31969093F5
:10690000C60090819923B1F720C08091C00085FF17
:10691000FCCF31969093C60090819923B1F715C0B2
:106920008091C00085FFFCCF31969093C600908186
:106930009923B1F70AC08091C00085FFFCCF319642
:106940009093C60090819923B1F780ED98E0622F73
:1069500040E050E00E9414538091C00085FFFCCFBE
:106960008AE08093C60081E001C080E0DF91CF9192
:1069700008955F926F927F928F929F92AF92BF9293
:10698000CF92DF92EF92FF920F931F93DF93CF93FB
:1069900000D00F92CDB7DEB719821A821B821C82FB
:1069A00084E4C82E86E0D82E0BE9E02E06E0F02E17
:1069B00000E010E03E010894611C711C55245394C2
:1069C000F801E351FC4F8081FEDE882359F14ADF54
:1069D0004B015C01F801E25CF94F8081882311F0E2
:1069E00061E002C06091AB0670E0882777FD80957A
:1069F000982F0E94EBCEF601208131814281538194
:106A00000E941ED19B01AC01C501B4010E9470CD52
:106A1000F7016083718382839383F301E00FF11F99
:106A200050820AC0F60180819181A281B381F70171
:106A300080839183A283B3830F5F1F4F84E090E034
:106A4000C80ED91EE80EF91E0430110509F0B8CFA2
:106A500086E4B9DE8823D9F005DF7B018C016093E1
:106A6000AC067093AD068093AE069093AF0620E01F
:106A700030E040E050E00E944CD0181644F4E09220
:106A80007503F09276030093770310937803809157
:106A90006E06882309F4C1C08981882309F0BDC02E
:106AA0008A81882309F0B9C08B81882309F0B5C099
:106AB0008C81882309F4B1C0A0905006B090510693
:106AC000C0905206D09053066091A7067091A80618
:106AD0008091A9069091AA06A60195010E946FCD0A
:106AE0007B018C012DEC3CEC4CEC5DEB0E9449CE23
:106AF00088230CF04EC080916F06882309F08DC06A
:106B00006091A3067091A4068091A5069091A606B7
:106B10002091690330916A0340916B0350916C039B
:106B20000E9470CD6093A3067093A4068093A5067F
:106B30009093A606C801B701905820916103309147
:106B4000620340916303509164030E946FCD9B01E7
:106B5000AC01C601B5010E946FCD609350067093E1
:106B6000510680935206909353068091650390914D
:106B70006603A0916703B0916803809375039093B7
:106B80007603A0937703B093780381E080936F0638
:106B900044C0C801B7012DEC3CEC4CEC5DE30E9415
:106BA0004CD01816D4F580916F068823B1F160910E
:106BB0006103709162038091630390916403A80163
:106BC00097010E946FCD209170063091710640911F
:106BD0007206509173060E9470CD9B01AC01C601F4
:106BE000B5010E9470CD609350067093510680935A
:106BF00052069093530680916D0390916E03A0917D
:106C00006F03B09170038093750390937603A09304
:106C10007703B093780310926F060F900F900F9048
:106C20000F90CF91DF911F910F91FF90EF90DF9028
:106C3000CF90BF90AF909F908F907F906F905F901C
:106C4000089597DE89E4BFDD882351F00BDE609361
:106C50008F067093900680939106909392060CC0D5
:106C600080E090E0A0E0B0E080938F0690939006E3
:106C7000A0939106B09392068AE4A5DD882351F093
:106C8000F1DD60939306709394068093950690933C
:106C90009606089580E090E0A0E0B0E0809393062F
:106CA00090939406A0939506B093960608952F921C
:106CB0003F924F925F926F927F928F929F92AF928C
:106CC000BF92CF92DF92EF92FF920F931F93DF93C9
:106CD000CF93CDB7DEB76E970FB6F894DEBF0FBE79
:106CE000CDBF1092740687E46EDD882309F455C584
:106CF000B9DD0E94B8CE6A30710509F48BC06B30E3
:106D000071059CF46230710599F16330710524F4CA
:106D1000772334F50C946C4A6330710581F164304B
:106D2000710511F00C946C4A33C06A35710509F491
:106D3000E3C46B35710554F46B30710509F400C17F
:106D40006C31710511F00C946C4A6FC16B35710593
:106D500009F4D6C46C35710511F00C946C4AD5C495
:106D600080917D06882321F404DEFBDA0C948D4AA1
:106D700080917D06882319F464DF81E006C080914C
:106D80007D06882329F45DDF80E02EDA0C948D4A9D
:106D900080E519DD882321F4EE24FF24870105C056
:106DA00061DD0E94BDCE7B018C0183E50CDD882373
:106DB00059F058DD20E030E04AE754E40E941ED14B
:106DC0000E94BDCE7B018C010E94087C0E94171A94
:106DD0005B016C01AE0CBF1CC01ED11E0E94171AB5
:106DE00060938706709388068093890690938A063D
:106DF00081E08093740605C00E9424889AD90E947D
:106E000076910E94171A6A157B058C059D05A0F3E3
:106E10000C946C4A80916F06882311F00C946C4A94
:106E20008091440690914506A0914606B091470690
:106E300080939B0690939C06A0939D06B0939E061C
:106E40008091480690914906A0914A06B0914B0660
:106E500080939F069093A006A093A106B093A206EC
:106E600080914C0690914D06A0914E06B0914F0630
:106E70008093A3069093A406A093A506B093A606BC
:106E80006091610370916203809163039091640348
:106E900020917A0330917B0340917C0350917D03D4
:106EA0000E9450CE9B01AC0160915006709151063A
:106EB00080915206909153060E946FCD9B01AC01C8
:106EC0006093A7067093A8068093A9069093AA06DC
:106ED000E0907503F09076030091770310917803AA
:106EE0006091500670915106809152069091530620
:106EF0000E946FCD60937006709371068093720646
:106F0000909373068091650390916603A091670347
:106F1000B09168038093750390937603A0937703F1
:106F2000B093780381E080936F061BDAE0927503DB
:106F3000F092760300937703109378030C946C4AD5
:106F400080916F06882311F40C946C4A809144065A
:106F500090914506A0914606B091470680939B0606
:106F600090939C06A0939D06B0939E068091480640
:106F700090914906A0914A06B0914B0680939F06D6
:106F80009093A006A093A106B093A20680914C0610
:106F900090914D06A0914E06B0914F068093A306A6
:106FA0009093A406A093A506B093A6066091500600
:106FB000709151068091520690915306209170066F
:106FC0003091710640917206509173060E9470CD07
:106FD0006093A7067093A8068093A9069093AA06CB
:106FE000E0907503F0907603009177031091780399
:106FF00080916D0390916E03A0916F03B091700327
:107000008093750390937603A0937703B0937803EE
:1070100010926F06A6D9E0927503F0927603009362
:107020007703109378030C946C4A85E08093740680
:107030008091750390917603A0917703B0917803C6
:107040008093B6069093B706A093B806B093B9069E
:107050008091500390915103909343068093420690
:1070600084E690E090935103809350030E94171A96
:1070700060938706709388068093890690938A06AA
:1070800081E00E949E7A8091440690914506A091ED
:107090004606B091470680939B0690939C06A0936A
:1070A0009D06B0939E068091480690914906A09156
:1070B0004A06B0914B0680939F069093A006A0933A
:1070C000A106B093A20680914C0690914D06A09126
:1070D0004E06B0914F068093A3069093A406A0930A
:1070E000A506B093A6068091500690915106A091F6
:1070F0005206B09153068093A7069093A806A093DA
:10710000A906B093AA0680E090E0A0E0B0E08093EA
:10711000750390937603A0937703B093780388E583
:1071200052DB882351F489E54EDB882331F48AE56C
:107130004ADB882311F481E001C080E08093790369
:10714000882309F416C10F2EF0E08F2EF0E09F2E59
:10715000F0E0AF2EF0E0BF2EF02D8092440690922A
:107160004506A0924606B092470680924806909245
:107170004906A0924A06B0924B0680924C06909225
:107180004D06A0924E06B0924F0684E496E068E465
:1071900076E04CE456E020E536E00E940C5880E0B2
:1071A00090E8ACEAB3EC80939B0690939C06A09386
:1071B0009D06B0939E0680E090ECA8EAB3E480932D
:1071C0009F069093A006A093A106B093A20680E02C
:1071D00090E8ACEAB3E48093A3069093A406A0934E
:1071E000A506B093A606609140037091410380917B
:1071F00042039091430360937503709376038093E9
:1072000077039093780320E030E040E752E40E9457
:1072100050CE7B018C018BE996E06FE976E043EA82
:1072200056E027EA36E0FCE6CF2EF6E0DF2E0E949D
:10723000215D0E94087C0E94977A80E090E00E9485
:10724000D82E81E090E00E94D82E82E090E00E944B
:10725000D82E84E496E068E476E04CE456E020E53D
:1072600036E00E940C588091440690914506A0910A
:107270004606B091470680939B0690939C06A09388
:107280009D06B0939E068091480690914906A09174
:107290004A06B0914B0680939F069093A006A09358
:1072A000A106B093A20680914C0690914D06A09144
:1072B0004E06B0914F068093A3069093A406A09328
:1072C000A506B093A6066091750370917603809130
:1072D00077039091780320E030E040E752E40E9489
:1072E00050CE7B018C018BE996E06FE976E043EAB2
:1072F00056E027EA36E00E94215D80927503909265
:107300007603A0927703B09278030E94087C0E94D3
:10731000977A80919B0690919C06A0919D06B091D2
:107320009E068093440690934506A0934606B0932C
:10733000470680919F069091A006A091A106B0916A
:10734000A2068093480690934906A0934A06B093FC
:107350004B068091A3069091A406A091A506B0913A
:10736000A60680934C0690934D06A0934E06B093CC
:107370004F0680917903882321F48AE524DA882353
:1073800019F082E090E0DAD880917903882351F4F3
:1073900088E519DA882309F40DC189E514DA882310
:1073A00009F408C180E090E0A0E0B0E080934406DA
:1073B00090934506A0934606B093470680934806EF
:1073C00090934906A0934A06B0934B0684E496E056
:1073D00068E476E04CE456E020E536E00E940C5884
:1073E00080E090E8ACEAB3EC80939B0690939C0617
:1073F000A0939D06B0939E0680E090ECA8EAB3E4CB
:1074000080939F069093A006A093A106B093A20636
:107410002091400330914103409142035091430336
:10742000209375033093760340937703509378034A
:10743000E0904403F0904503009146031091470308
:10744000C801B7010E9449CE882344F4E092750335
:10745000F09276030093770310937803609175039D
:1074600070917603809177039091780320E030E06B
:1074700040E752E40E9450CE7B018C018BE996E0FC
:107480006FE976E043EA56E027EA36E0ECE6CE2EF6
:10749000E6E0DE2E0E94215D0E94087C80E090E004
:1074A0000E94D82E81E090E00E94D82E84E496E0DD
:1074B00068E476E04CE456E020E536E00E940C58A3
:1074C0008091440690914506A0914606B0914706EA
:1074D00080939B0690939C06A0939D06B0939E0676
:1074E0008091480690914906A0914A06B0914B06BA
:1074F00080939F069093A006A093A106B093A20646
:107500006091750370917603809177039091780371
:1075100020E030E040E752E40E9450CE7B018C0135
:107520008BE996E06FE976E043EA56E027EA36E039
:107530000E94215D80E090E0A0E0B0E080937503C0
:1075400090937603A0937703B09378030E94087C0E
:107550000E94977A80919B0690919C06A0919D062F
:10756000B0919E068093440690934506A0934606EC
:10757000B093470680919F069091A006A091A10626
:10758000B091A2068093480690934906A0934A06BC
:10759000B0934B068091A3069091A406A091A506F6
:1075A000B091A60680934C0690934D06A0934E068C
:1075B000B0934F0680917903882321F488E503D99D
:1075C000882321F080E090E00E949E328091790330
:1075D000882321F489E5F7D8882321F081E090E021
:1075E0000E949E3288E5EFD88823C9F030D9611512
:1075F00071058105910599F035D920915406309196
:10760000550640915606509157060E9470CD6093E2
:10761000440670934506809346069093470689E595
:10762000D2D88823C9F013D9611571058105910558
:1076300099F018D9209158063091590640915A0670
:1076400050915B060E9470CD609348067093490686
:1076500080934A0690934B068AE5B5D88823C9F0F3
:10766000F6D8611571058105910599F0FBD8209137
:107670005C0630915D0640915E0650915F060E9467
:1076800070CD60934C0670934D0680934E06909398
:107690004F0684E496E068E476E04CE456E020E5AA
:1076A00036E00E940C5880E00E949E7A8091B606D7
:1076B0009091B706A091B806B091B9068093750372
:1076C00090937603A0937703B0937803809142065A
:1076D0009091430690935103809350030E94171A90
:1076E00060938706709388068093890690938A0634
:1076F0000E94977A0C946C4A1092AB060C946C4AD8
:1077000081E08093AB060C946C4A85E45CD88823B6
:1077100011F40E94087C44E4E42E46E0F42E34E5A3
:10772000C32E36E0D32E00E010E0F801E351FC4F09
:10773000808149D8882321F1033059F493D8F70187
:10774000608371838283938380E596E00E94E5578E
:1077500017C088D8F60120813181428153810E946F
:1077600070CDF701608371838283938384E496E014
:1077700068E476E04CE456E020E536E00E940C58E0
:107780000F5F1F4F24E030E0E20EF31EC20ED31E47
:107790000430110551F60C946C4A8DE414D88823FA
:1077A00011F40C948E495ED80E94B8CE63377105EF
:1077B00011F40C944344643771050CF08DC06A32A7
:1077C000710509F44AC36B3271050CF040C0683191
:1077D000710509F495C169317105D4F464317105FD
:1077E00009F437C16531710554F46131710509F44B
:1077F0002AC16231710511F00C946C4A5DC7663183
:10780000710509F45CC1673171050CF05EC151C1AD
:107810006B31710509F4AFC16C31710554F46931F4
:10782000710509F47DC16A31710511F00C946C4A3F
:107830007DC16E31710509F4E0C16F31710509F444
:107840008BC26C31710511F00C946C4A9AC16C3585
:10785000710509F493C76D357105FCF46235710546
:1078600009F423C76335710554F46035710509F4D3
:1078700016C76135710511F00C946C4A13C7643555
:10788000710509F419C7643571050CF411C7653524
:10789000710511F00C946C4A58C76A36710509F4E9
:1078A00084C66B36710554F46836710509F41DC33E
:1078B0006936710511F00C946C4A48C36D36710538
:1078C00009F416C46237710509F4FCC76B367105FB
:1078D00011F00C946C4AE0C6613D710511F40C94F2
:1078E0001047623D71050CF049C0693C710511F407
:1078F0000C94E5456A3C71050CF56837710511F487
:107900000C9456456937710554F46537710509F4CF
:10791000C9C76737710511F00C946C4A90C06C3878
:10792000710509F402C36E3B710509F474C569372A
:10793000710511F00C946C4A0C945A456D3C71051C
:1079400011F40C9445466E3C710564F46B3C710572
:1079500011F40C9407466C3C710511F00C946C4AC0
:107960000C9425466F3C710511F40C94C146603DA2
:10797000710514F00C94F0460C94A34631E0603984
:10798000730711F40C946A4941E0613974074CF5AE
:1079900051E06D32750711F40C94954781E06E3219
:1079A000780764F46C3D710511F40C9477476D3DD4
:1079B000710511F00C946C4A0C94864791E06F327B
:1079C000790711F40C942A49E1E06F327E0714F430
:1079D0000C941B496053714011F00C946C4A0C9448
:1079E0006D4821E0673F720711F40C94764931E04D
:1079F000683F73079CF441E0653F740711F40C94F1
:107A0000704951E0663F750714F00C947349645F48
:107A1000714011F00C946C4A0C946D4993E0603AFB
:107A2000790709F45EC1E3E0673E7E0711F40C9428
:107A300079496B59734011F00C946C4A29C1EBE7FA
:107A4000F2E00C94654515984698439840980C943C
:107A50006C4AEDEDF7E0949108C08091C00085FF7D
:107A6000FCCF9093C600319694919923B1F7809101
:107A7000C00085FFFCCF8AE08093C60084E494E0D8
:107A80000E94E326EFECF7E0949108C08091C000DB
:107A900085FFFCCF9093C600319694919923B1F75E
:107AA0008091C00085FFFCCF8AE08093C6000C94D3
:107AB0006C4A84E494E00E946F220C946C4A84E443
:107AC00094E00E945E1C0C946C4A8091BA069091DE
:107AD000BB0604966AE270E00E94DFCCFC010097CE
:107AE00011F0319710826091BA067091BB066C5FFD
:107AF0007F4F84E494E041E00E94DC1E0C946C4AC9
:107B000084E494E00E94621C0E94171A6093750638
:107B10007093760680937706909378060C946C4A5F
:107B200084E494E00E94691C0C946C4A8091720475
:107B3000882311F40C946C4A8091EB05882311F092
:107B40000C946C4A83E50E94E333882311F40C946F
:107B50006C4A0E942734AB01BC0140933406509319
:107B60003506809336067093370681E196E00E94D1
:107B70007C6C0C946C4A84E494E00E945F1E0C942C
:107B80006C4A8091BA069091BB0604966AE270E056
:107B90000E94DFCC8C01009719F12091B006309142
:107BA000B10680E690E0AC01249FC001259F900DB6
:107BB000349F900D11248454994F6EE470E00E941C
:107BC000DFCC60E270E00E94DFCC9C012F5F3F4F72
:107BD0003093BB062093BA0601501040F801108282
:107BE0006091BA067091BB066C5F7F4F84E494E0AD
:107BF00040E00E94DC1E0C946C4A80917204882341
:107C000011F40C946C4A8091EB05882311F00C94CC
:107C10006C4A84E494E00E94CE1D8091BA06909153
:107C2000BB0604966AE270E00E94DFCC8C010097EC
:107C300019F12091B0063091B10680E690E0AC01D8
:107C4000249FC001259F900D349F900D11248454D2
:107C5000994F6EE470E00E94DFCC60E270E00E9419
:107C6000DFCC9C012F5F3F4F3093BB062093BA06B9
:107C700001501040F80110826091BA067091BB0665
:107C80006C5F7F4F84E494E00E94FE200C946C4A69
:107C90008091BA069091BB0604966AE270E00E9459
:107CA000DFCCFC01009711F0319710826091BA0689
:107CB0007091BB066C5F7F4F84E494E041E00E94CA
:107CC000DC1E84E494E00E94621C0E94171A6093F8
:107CD00075067093760680937706909378060C94D9
:107CE0006C4A8091BA069091BB0605966AE270E0F4
:107CF0000E94DFCC8C01009719F12091B0063091E1
:107D0000B10680E690E0AC01249FC001259F900D54
:107D1000349F900D11248454994F6EE470E00E94BA
:107D2000DFCC60E270E00E94DFCC9C012F5F3F4F10
:107D30003093BB062093BA0601501040F801108220
:107D40006091BA067091BB066B5F7F4F84E494E04C
:107D50000E94F8200C946C4A0E94171A60937906CE
:107D600070937A0680937B0690937C06209175062B
:107D7000309176064091770650917806621B730B1E
:107D8000840B950B28EE33E040E050E00E9413D5C1
:107D9000F22EE32ED42EC52E2DB73EB728503040FC
:107DA0000FB6F8943EBF0FBE2DBF0DB71EB70F5FC5
:107DB0001F4FCE010196EDB7FEB79283818380EC11
:107DC00097E0F801938382836F2D7E2D842F952F6A
:107DD0002CE330E040E050E00E9413D5F8013583F9
:107DE00024836F2D7E2D8D2D9C2D2CE330E040E0E3
:107DF00050E00E9413D5F801778366830E943FCD3F
:107E0000E4EEF5E094912DB73EB7285F3F4F0FB6F3
:107E1000F8943EBF0FBE2DBF08C08091C00085FF03
:107E2000FCCF9093C600319694919923B1F7FE014F
:107E3000319607C08091C00085FFFCCF31969093AA
:107E4000C60090819923B1F78091C00085FFFCCFD7
:107E50008AE08093C6000C946C4A83E50E94E33369
:107E6000882311F40C946C4A0E9432340E94B8CEDC
:107E70007B018C016B0180E50E94E333882369F06C
:107E8000F7FC0BC03FEFE316F10409F034F40E9455
:107E900032340E94B8CE8B0102C008E010E0E1EF5E
:107EA000F3E0808191818017910711F40C946C4A62
:107EB000329644E0E136F407A1F70730110519F4D2
:107EC000C0926D0604C017FF02C00C946C4A802F4C
:107ED00061E00E94651B802F6C2D0E94181C802F72
:107EE000B6010E94871A0C946C4A88E690E00E94C2
:107EF0003B34882311F00C946C4A83E50E94E333F1
:107F0000882379F00E94323420917E06022F10E0FF
:107F1000000F111F04581F4E0E94B8CEF801718344
:107F200060830E9407840C946C4A83E50E94E333CB
:107F3000882311F40C946C4A0E9432340E94B8CE0B
:107F400070937F1060937E100C946C4A89E690E0E9
:107F50000E943B34882311F00C946C4AEAEBF7E062
:107F6000949108C08091C00085FFFCCF9093C6001B
:107F7000319694919923B1F7E0917E06F0E0EE0FEF
:107F8000FF1FEE0FFF1FEE57FF4E408151816281B0
:107F9000738180ED98E021E030E00E942B54E7EB04
:107FA000F7E0949108C08091C00085FFFCCF9093CA
:107FB000C600319694919923B1F7E0917E06F0E0E6
:107FC000EE0FFF1FE458FF4E60817181882777FD17
:107FD0008095982F0E94EBCEAB01BC0180ED98E01C
:107FE00021E030E00E942B54E3EBF7E0949108C0CD
:107FF0008091C00085FFFCCF9093C600319694918C
:108000009923B1F7409188105091891060918A109E
:1080100070918B1080ED98E021E030E00E942B54AD
:10802000E0EBF7E0949108C08091C00085FFFCCFA1
:108030009093C600319694919923B1F760917E1088
:1080400070917F10882777FD8095982F0E94EBCE46
:10805000AB01BC0180ED98E021E030E00E942B54A0
:10806000ECEAF7E0949108C08091C00085FFFCCF56
:108070009093C600319694919923B1F780917E0632
:108080000E944C83BC0180ED98E04AE050E00E94E1
:108090005853E7EAF7E0949108C08091C00085FF4B
:1080A000FCCF9093C600319694919923B1F78FEF4E
:1080B0009FEF0E944C83BC0180ED98E04AE050E0C5
:1080C0000E945853E4E9F2E007C08091C00085FFA8
:1080D000FCCF31969093C60090819923B1F780919F
:1080E000C00085FFFCCF8AE08093C6000C948D4AC7
:1080F0008DE690E00E943B34882311F00C946C4A8A
:1081000083E08093740683E50E94E333882379F04B
:108110000E94323420917E06022F10E0000F111FC2
:1081200004581F4E0E94B8CEF801718360830E94EC
:1081300007840E94171A4B015C0120917E06022FD2
:1081400010E07724000F111FF801E458FF4E608102
:108150007181882777FD8095982F0E94EBCE000FC4
:10816000111F0E571F4EF80120813181428153812A
:108170000E944CD0181614F477247394CC24CA941B
:10818000DC2C7601E4EAF7E04490E0EAF7E0549072
:10819000ECE9F7E064905AE0352E30C1942DE4EA22
:1081A000F7E008C08091C00085FFFCCF9093C60027
:1081B000319694919923B1F7E0917E06F0E0EE0FAD
:1081C000FF1FEE0FFF1FEE57FF4E4081518162816E
:1081D000738180ED98E021E030E00E942B54952DD2
:1081E000E0EAF7E008C08091C00085FFFCCF9093E3
:1081F000C600319694919923B1F760917E0680ED87
:1082000098E070E04AE050E00E945853962DECE967
:10821000F7E008C08091C00085FFFCCF9093C600B6
:10822000319694919923B1F7F7FE03C0E5E9F2E0A6
:1082300028C00E94171AA70196012854344F4F4FA7
:108240005F4F261B370B480B590BCA01B90128EEAB
:1082500033E040E050E00E9413D580ED98E0BA0191
:10826000A9012AE030E00E9409538091C00085FFF7
:10827000FCCF0EC08091C00085FFFCCF319690935B
:10828000C60090819923B1F78091C00085FFFCCF93
:108290003092C6000E94171A4B015C010E9424888C
:1082A0000E9499300E947691FFEFCF16FFEFDF0614
:1082B000FFEFEF06FFEFFF0609F050C0E0917E06EA
:1082C000772031F1F0E08F01000F111F000F111F17
:1082D0000E571F4EEE0FFF1FE458FF4E6081718155
:1082E000882777FD8095982F0E94EBCE20E030E024
:1082F00040E050E40E946FCD9B01AC01F801608129
:108300007181828193810E944CD087FF5AC060C0E6
:10831000F0E08F01000F111F000F111F0E571F4EAD
:10832000EE0FFF1FE458FF4E60817181882777FDB3
:108330008095982F0E94EBCE20E030E040E050E4A2
:108340000E9470CD9B01AC01F80160817181828136
:1083500093810E9449CE1816A4F53AC0F7FC38C0A4
:10836000E0917E06F0E08F01000F111F000F111F3A
:108370000E571F4EEE0FFF1FE458FF4E60817181B4
:10838000882777FD8095982F0E94EBCE9B01AC014A
:10839000F80160817181828193810E946FCD0E947A
:1083A000B8CE97FF07C090958095709561957F4FE7
:1083B0008F4F9F4F64307105810591054CF07720F8
:1083C00039F40E94171AAC01CB01DA016C017D016E
:1083D000FFEFCF16FFEFDF06FFEFEF06FFEFFF0621
:1083E00069F0F7FE02C00C946F4A0E94171A6C19CC
:1083F0007D09685B7B4010F00C946F4A0E94171A4D
:10840000681979098A099B09695E73408040904028
:1084100008F0C4CE43CF84E08093740683E50E94C5
:10842000E333882341F00E9432340E94B8CE709327
:108430007F1060937E100E94171A5B016C01E9E9BE
:10844000F7E07490E5E9F7E08490E1E9F7E09490D3
:10845000EAE06E2E7DC00E94171A6A197B098C090A
:108460009D09695E73408040904008F46BC0E091C4
:108470006C06F0E0EE0FFF1FEE0FFF1FEE57FF4EF2
:108480004081518162817381972DE9E9F7E008C04D
:108490008091C00085FFFCCF9093C60031969491E7
:1084A0009923B1F780ED98E022E030E00E942B5450
:1084B000982DE5E9F7E008C08091C00085FFFCCF6A
:1084C0009093C600319694919923B1F760916C0610
:1084D00080ED98E070E04AE050E00E945853992DFA
:1084E000E1E9F7E008C08091C00085FFFCCF9093E0
:1084F000C600319694919923B1F74091881050911C
:10850000891060918A1070918B1080ED98E021E0C5
:1085100030E00E942B54E4E9F2E007C08091C000F3
:1085200085FFFCCF31969093C60090819923B1F7D7
:108530008091C00085FFFCCF6092C6000E94171A90
:108540005B016C010E9424880E9499300E94769100
:1085500060917E1070917F10882777FD8095982F0D
:108560000E94EBCE7B018C01609188107091891084
:1085700080918A1090918B1020E030E040E050E430
:108580000E946FCD9B01AC01C801B7010E9449CE8A
:1085900087FD61CF0E94171A609387067093880643
:1085A0008093890690938A0697C783E50E94E333F8
:1085B000882309F464C00E9432347B018C016091ED
:1085C000600370E0882777FD8095982F0E94EBCE9E
:1085D0009B01AC01C801B7010E941ED120E030E030
:1085E00048EC52E40E9450CE20E030E040E050E001
:1085F0000E9449CE882314F460E03EC00E943234C9
:108600007B018C016091600370E0882777FD809585
:10861000982F0E94EBCE9B01AC01C801B7010E94CC
:108620001ED120E030E048EC52E40E9450CE20E021
:1086300030E04FE753E40E944CD0181614F46FEF6B
:108640001BC00E9432347B018C016091600370E09A
:10865000882777FD8095982F0E94EBCE9B01AC0177
:10866000C801B7010E941ED120E030E048EC52E47E
:108670000E9450CE0E94BDCE60936D062DC78091A2
:1086800060039FEF899FC001112464E670E00E949F
:1086900000D560936D0620C710926D061DC7269AFF
:1086A0002E981AC7269A2E9A17C71092410614C7F9
:1086B00081E08093410610C783E50E94E33388235D
:1086C00099F00E94323420E030E04AE754E40E94FE
:1086D0001ED10E94BDCE609371037093720380938C
:1086E000730390937403F8C688E50E94E3338823EC
:1086F00009F00AC789E50E94E333882309F004C71B
:108700008AE50E94E333882309F0FEC685E40E94CF
:10871000E333882309F0F8C60E94087C409A0E943F
:10872000167CDAC6159A89E50E94E3338111469AD0
:108730008AE50E94E3338111439A85E40E94E33382
:10874000882309F4C9C6409AC7C683E50E94E3336B
:10875000882309F4C1C60E94323420E030E04AE7A1
:1087600054E40E941ED10E94BDCE60938B0670938C
:108770008C0680938D0690938E06AEC665EE662EAF
:1087800068E0762E55ED252E58E0352E41E2442E38
:1087900049E0542E88249924F401E351FC4F808150
:1087A0000E94E333882309F45DC053E0851609F085
:1087B00052C00E9432345B016C0120E030E040EA9C
:1087C00051E40E9449CE88230CF03FC0F301608140
:1087D000718182819381A60195010E9450CE7B0117
:1087E0008C016091190970911A0980911B0990916F
:1087F0001C09A80197010E941ED16093190970936A
:108800001A0980931B0990931C09F1016081718101
:1088100082819381A80197010E941ED1F10160839A
:10882000718382839383F20160817181828193815C
:108830000E94E9CEA80197010E941ED10E94BDCEE0
:10884000F2016083718382839383F301A082B182FA
:10885000C282D38207C00E943234F30160837183E5
:10886000828393830894811C911C24E030E0620E83
:10887000731E220E331E420E531E34E083169104E3
:1088800009F08ACF29C6E1EFF6E0949108C0809103
:10889000C00085FFFCCF9093C60031969491992338
:1088A000B1F71AC68091BA069091BB0605966AE2A6
:1088B00070E00E94DFCCFC01009709F40DC63197EF
:1088C00010820AC6EEEEF6E0949108C08091C000D6
:1088D00085FFFCCF9093C600319694919923B1F710
:1088E00040914406509145066091460670914706B6
:1088F00080ED98E022E030E00E942B54EBEEF6E0B1
:10890000949108C08091C00085FFFCCF9093C60071
:10891000319694919923B1F74091480650914906B8
:1089200060914A0670914B0680ED98E022E030E0BD
:108930000E942B54E8EEF6E0949108C08091C000AC
:1089400085FFFCCF9093C600319694919923B1F79F
:1089500040914C0650914D0660914E0670914F0625
:1089600080ED98E022E030E00E942B54E5EEF6E046
:10897000949108C08091C00085FFFCCF9093C60001
:10898000319694919923B1F7409150065091510638
:10899000609152067091530680ED98E022E030E03D
:1089A0000E942B54EAEDF6E0949108C08091C0003B
:1089B00085FFFCCF9093C600319694919923B1F72F
:1089C00080E00E94F27A0E94EBCE2091E50830917F
:1089D000E6084091E7085091E8080E9450CEAB01AC
:1089E000BC0180ED98E022E030E00E942B54E7EDDE
:1089F000F6E0949108C08091C00085FFFCCF909371
:108A0000C600319694919923B1F781E00E94F27AE1
:108A10000E94EBCE2091E9083091EA084091EB08E2
:108A20005091EC080E9450CEAB01BC0180ED98E063
:108A300022E030E00E942B54E4EDF6E0949108C06F
:108A40008091C00085FFFCCF9093C6003196949131
:108A50009923B1F782E00E94F27A0E94EBCE209136
:108A6000ED083091EE084091EF085091F0080E9417
:108A700050CEAB01BC0180ED98E022E030E00E94D6
:108A80002B54E4E9F2E007C08091C00085FFFCCFE1
:108A900031969093C60090819923B1F78091C000E0
:108AA00085FFFCCF8AE08093C60016C580E00E9457
:108AB0009E7A12C581E00E949E7A0EC58091C00008
:108AC00085FFFCCF31969093C60090819923B1F732
:108AD0008091C00085FFFCCF8AE08093C600ECEC5B
:108AE000F6E0949108C08091C00085FFFCCF909380
:108AF000C600319694919923B1F7009B03C0E7E932
:108B0000F2E00AC0ECE9F2E007C08091C00085FF06
:108B1000FCCF31969093C60090819923B1F7809154
:108B2000C00085FFFCCF8AE08093C600E4ECF6E04D
:108B3000949108C08091C00085FFFCCF9093C6003F
:108B4000319694919923B1F7049B03C0E7E9F2E0D1
:108B50000AC0ECE9F2E007C08091C00085FFFCCFBD
:108B600031969093C60090819923B1F78091C0000F
:108B700085FFFCCF8AE08093C600ECEBF6E0949191
:108B800008C08091C00085FFFCCF9093C60031964D
:108B900094919923B1F7079B03C0E7E9F2E00AC07B
:108BA000ECE9F2E007C08091C00085FFFCCF319670
:108BB0009093C60090819923B1F78091C00085FF02
:108BC000FCCF8AE08093C60087C40DEE13E035EF3A
:108BD000E32E38E0F32EF80180810E94E3338823EE
:108BE00049F00E9432340E94BDCEF7016083718348
:108BF000828393830F5F1F4F24E030E0E20EF31E69
:108C000033E0013F130739F70E94BA5765C40DEEF0
:108C100013E025EDE22E28E0F22EF80180810E947B
:108C2000E333882339F00E943234F7016083718383
:108C3000828393830F5F1F4F24E030E0E20EF31E28
:108C400033E0013F130749F747C483E50E94E3334C
:108C5000882351F00E9432346093090970930A0905
:108C600080930B0990930C0984E50E94E3338823D9
:108C700009F432C40E94323460930D0970930E09D6
:108C800080930F099093100927C483E50E94E33372
:108C9000882351F00E9432346093050970930609CD
:108CA000809307099093080984E50E94E3338823A1
:108CB00051F00E94323460931D0970931E09809315
:108CC0001F099093200982E40E94E333882361F016
:108CD0000E9432340E94BDCE6093D1087093D208B6
:108CE0008093D3089093D40888E50E94E3338823C7
:108CF00051F00E94323460931109709312098093ED
:108D00001309909314098AE50E94E333882351F0F4
:108D10000E943234609315097093160980931709E5
:108D20009093180985E40E94E333882309F4D4C39F
:108D30000E9432346093190970931A0980931B09B9
:108D400090931C09C9C30DEE13E094E5E92E96E05B
:108D5000F92EF80180810E94E333882339F00E94C4
:108D60003234F70160837183828393830F5F1F4FD7
:108D700024E030E0E20EF31E33E0003F130749F732
:108D8000ABC383E50E94E333882351F00E94323461
:108D90006093610370936203809363039093640311
:108DA00086E40E94E333882351F00E9432346093BA
:108DB00065037093660380936703909368038AE565
:108DC0000E94E333882309F487C30E9432346093FE
:108DD000690370936A0380936B0390936C037CC365
:108DE00083E50E94E333882351F00E94323460937C
:108DF000700670937106809372069093730686E4F2
:108E00000E94E333882309F467C30E9432346093DD
:108E10006D0370936E0380936F03909370035CC334
:108E200083E50E94E333882309F456C30E94323459
:108E30000E94B8CE672B21F06130710561F405C046
:108E400010926E0610926F0647C381E080936E0603
:108E500010926F0641C3E4EEF5E0949108C0809152
:108E6000C00085FFFCCF9093C60031969491992362
:108E7000B1F7E9EAF6E0949108C08091C00085FF5F
:108E8000FCCF9093C600319694919923B1F720912D
:108E9000B0063091B10680E690E0289FF001299F4E
:108EA000F00D389FF00D1124E454F94F07C0809164
:108EB000C00085FFFCCF31969093C6009081992326
:108EC000B1F7E7EAF6E0949108C08091C00085FF11
:108ED000FCCF9093C600319694919923B1F780917D
:108EE000C00085FFFCCF8AE08093C600F5C283E511
:108EF0000E94E333882309F4EFC20E9432340E94B7
:108F0000B8CE7093510360935003E6C283E50E948C
:108F1000E333882309F4E0C20E9432340E94B8CEC1
:108F20007093530360935203D7C280E50E94E333EA
:108F3000882351F00E94323460938D0370938E0326
:108F400080938F039093900389E40E94E3338823F6
:108F500061F00E9432340E941784609391037093F1
:108F60009203809393039093940384E40E94E333E9
:108F7000882361F00E9432340E9423846093950319
:108F800070939603809397039093980383E40E94D1
:108F9000E333882351F00E94323460939903709335
:108FA0009A0380939B0390939C030E941F83E6EA9D
:108FB000F2E007C08091C00085FFFCCF319690930E
:108FC000C60090819923B1F7E9EAF2E007C08091E9
:108FD000C00085FFFCCF31969093C6009081992305
:108FE000B1F740918D0350918E0360918F03709182
:108FF000900380ED98E022E030E00E942B54EDEAEF
:10900000F2E007C08091C00085FFFCCF31969093BD
:10901000C60090819923B1F76091910370919203FA
:1090200080919303909194030E941D84AB01BC0135
:1090300080ED98E022E030E00E942B54E1EBF2E07A
:1090400007C08091C00085FFFCCF31969093C60089
:1090500090819923B1F76091950370919603809167
:109060009703909198030E942984AB01BC0180ED85
:1090700098E022E030E00E942B54E5EBF2E007C0DC
:109080008091C00085FFFCCF31969093C6009081FF
:109090009923B1F74091990350919A0360919B03F2
:1090A00070919C0380ED98E022E030E00E942B5408
:1090B000E4E9F2E007C08091C00085FFFCCF319663
:1090C0009093C60090819923B1F78091C00085FFED
:1090D000FCCF8AE08093C600FFC180E50E94E333A5
:1090E000882351F00E94323460939D0370939E0355
:1090F00080939F039093A00389E40E94E333882325
:1091000061F00E9432340E9417846093A10370932F
:10911000A2038093A3039093A40384E40E94E33307
:10912000882361F00E9432340E9423846093A50357
:109130007093A6038093A7039093A8030E941F83B4
:10914000E6EAF2E007C08091C00085FFFCCF3196CF
:109150009093C60090819923B1F7E9EAF2E007C045
:109160008091C00085FFFCCF31969093C60090811E
:109170009923B1F740919D0350919E0360919F0305
:109180007091A00380ED98E022E030E00E942B5423
:10919000EDEAF2E007C08091C00085FFFCCF319678
:1091A0009093C60090819923B1F76091A1037091CB
:1091B000A2038091A3039091A4030E941D84AB019C
:1091C000BC0180ED98E022E030E00E942B54E1EBFE
:1091D000F2E007C08091C00085FFFCCF31969093EC
:1091E000C60090819923B1F76091A5037091A60301
:1091F0008091A7039091A8030E942984AB01BC0130
:1092000080ED98E022E030E00E942B54E4E9F2E0A7
:1092100007C08091C00085FFFCCF31969093C600B7
:1092200090819923B1F78091C00085FFFCCF8AE03F
:109230008093C60051C183E50E94E333882329F45B
:1092400060E070E080E090E002C00E9432340E9452
:10925000B15742C185E40E94E333882319F4CC243A
:10926000DD2412C00E9432340E94B8CE6B0177FF19
:109270000BC00F2EF0E0EF2EF0E0FF2EFCE80F2FDA
:10928000F2E41F2FF02D0AC00F2EF0E0EF2EF0E0D9
:10929000FF2EF6E10F2FF3E41F2FF02D83E50E9440
:1092A000E333882321F00E9432347B018C0183E474
:1092B0000E94E333882319F425E030E005C00E94C2
:1092C00032340E94B8CE9B01C801B701A6010E94AA
:1092D000B88A02C10E94087CFFC00E94B42DFCC065
:1092E0000E94B02CF9C00E94C527F6C00E946329D5
:1092F000F3C010927D068091830690918406A09120
:109300008506B091860680937F0690938006A09391
:109310008106B09382060E947232DEC084E50E940C
:10932000E333882309F48DC00E9432340E94BDCEFD
:10933000262F60937E066623B9F1E4EEF5E0949162
:1093400008C08091C00085FFFCCF9093C600319685
:1093500094919923B1F7E9EBF2E007C08091C00046
:1093600085FFFCCF31969093C60090819923B1F789
:1093700080ED98E0622F40E050E00E941453EBEB48
:10938000F2E007C08091C00085FFFCCF319690933A
:10939000C60090819923B1F78091C00085FFFCCF72
:1093A0008AE08093C60098C086E40E94E333882355
:1093B000E1F00E9432347B018C016093AC06709323
:1093C000AD068093AE069093AF0620E030E040E01B
:1093D00050E00E944CD0181644F4E0927503F092CD
:1093E00076030093770310937803E4EEF5E094910D
:1093F00008C08091C00085FFFCCF9093C6003196D5
:1094000094919923B1F7ECECF2E007C08091C00091
:1094100085FFFCCF31969093C60090819923B1F7D8
:1094200060916C0680ED98E070E04AE050E00E94A8
:1094300058538091C00085FFFCCF8AE08093C6001E
:109440004BC0E4EEF5E0949108C08091C00085FF28
:10945000FCCF9093C600319694919923B1F7E4E93B
:10946000F6E0949108C08091C00085FFFCCF9093F6
:10947000C600319694919923B1F72091B0063091AE
:10948000B10680E690E0289FF001299FF00D389FFB
:10949000F00D1124E454F94F07C08091C00085FFFE
:1094A000FCCF31969093C60090819923B1F7E2E901
:1094B000F6E0949108C08091C00085FFFCCF9093A6
:1094C000C600319694919923B1F78091C00085FF31
:1094D000FCCF8AE08093C6000E9470301EC00E94BC
:1094E000171A6093750670937606809377069093AB
:1094F00078060E94171A60938706709388068093F7
:10950000890690938A06E8CF0E94087C88E50E942D
:10951000E333882309F006C906C96E960FB6F8949E
:10952000DEBF0FBECDBFCF91DF911F910F91FF9096
:10953000EF90DF90CF90BF90AF909F908F907F90F3
:109540006F905F904F903F902F9008952F923F9291
:109550004F925F926F927F928F929F92AF92BF9243
:10956000CF92DF92EF92FF920F931F93DF93CF93EF
:10957000CDB7DEB76E970FB6F894DEBF0FBECDBF86
:1095800080E6A82EB12CE3E5F8E084900AE0702E86
:10959000E9ECF8E094906624639409C22D3071F0F0
:1095A0002A3321F480913D08882341F080913E08C0
:1095B00090913F088F3591050CF4D5C1E0913E089C
:1095C000F0913F08309709F40CC3A0914008B09186
:1095D0004108AA9D7001AB9DF00CBA9DF00C1124BE
:1095E000EE0DFF1DE454F94F108280913D08882351
:1095F00009F0B4C110923D08AE54B94F1C928701D6
:109600000454194FC8016EE470E00E94DFCC9C0145
:10961000009709F4F4C09093BB068093BA062F5FBD
:109620003F4F201B310B2E0D3F1DC9018454994F14
:1096300060E070E04AE050E00E94FECA6093420899
:10964000709343088093440890934508C0907F0628
:10965000D0908006E0908106F0908206A7019601E6
:109660002F5F3F4F4F4F5F4F621773078407950778
:1096700009F469C380914008909141089C012A9D9A
:10968000C0012B9D900D3A9D900D11248454994F4B
:1096900062E779E00E94A4CC892B09F054C3EAEE7A
:1096A000F5E0949108C08091C00085FFFCCF9093B5
:1096B000C600319694919923B1F7EFE3F9E09491C4
:1096C00008C08091C00085FFFCCF9093C600319602
:1096D00094919923B1F780ED98E0B701A6012AE0B3
:1096E00030E0B3D78091C00085FFFCCF71C0FE266B
:1096F0004F5FFC01E40FF11DE454F94FE081EA32C1
:10970000B1F73093BB062093BA06C901019660E019
:1097100070E00E9498C90E94B8CE2F2D30E0261725
:10972000370709F45BC0EAEEF5E0949108C0809138
:10973000C00085FFFCCF9093C60031969491992389
:10974000B1F7E0E2F9E0949108C08091C00085FF94
:10975000FCCF9093C600319694919923B1F7409134
:109760007F0650918006609181067091820680ED9F
:1097700098E02AE030E069D78091C00085FFFCCFF7
:1097800027C0EAEEF5E0949108C08091C00085FF03
:10979000FCCF9093C600319694919923B1F7E6EFF0
:1097A000F8E0949108C08091C00085FFFCCF9093B1
:1097B000C600319694919923B1F780ED98E0B701F6
:1097C000A6012AE030E041D78091C00085FFFCCFA0
:1097D0008AE08093C6000E94723249C0809142089C
:1097E00090914308A0914408B091450880937F066A
:1097F00090938006A0938106B09382063DC0C80175
:109800006AE270E00E94DFCC009709F435C0EAEE0E
:10981000F5E0949108C08091C00085FFFCCF909343
:10982000C600319694919923B1F7ECECF8E094914D
:1098300008C08091C00085FFFCCF9093C600319690
:1098400094919923B1F740917F06509180066091E1
:1098500081067091820680ED98E02AE030E0F5D62E
:109860008091C00085FFFCCF8AE08093C6001092F3
:109870003F0810923E0886C28091400890914108AE
:109880008A9D70018B9DF00C9A9DF00C112487012C
:109890000454194FC80167E470E00E94DFCC9C01BA
:1098A000009709F445C09093BB068093BA062F5FDA
:1098B0003F4F201B310B2E0D3F1DC9018454994F82
:1098C00060E070E00E9498C90E94B8CE64307105D3
:1098D00078F580917D068823B9F48091440488232B
:1098E00039F5992DE9ECF8E008C08091C00085FFBA
:1098F000FCCF9093C600319694919923B1F7809153
:10990000C00085FFFCCF12C0982DE3E5F8E008C049
:109910008091C00085FFFCCF9093C6003196949152
:109920009923B1F78091C00085FFFCCF7092C600EB
:109930008091400890914108019664E070E00E9497
:1099400000D59093410880934008809146089091FB
:1099500047080196909347088093460810923F0865
:1099600010923E0824C02B3311F460923D08809180
:109970003D088823E1F420913E0830913F08809112
:109980004008909141088A9DF0018B9DF00D9A9DB1
:10999000F00D1124E20FF31FE454F94F80913C08BD
:1099A00080832F5F3F4F30933F0820933E08809184
:1099B000CC089091CD082091CE083091CF08821B21
:1099C000930B8F779070892B09F4D7C1809146084B
:1099D0009091470804970CF0D0C180ED98E05BD5DA
:1099E000282F80933C088A3009F0D8CDE7CD8091AC
:1099F0003E0890913F08892B09F459C1C3C1929B3D
:109A000005C084E494E00E945E1C31CF1092EB0507
:109A100010923F0810923E08409148085091490822
:109A200060914A0870914B08409334065093350674
:109A3000609336067093370681E196E00E947C6C55
:109A4000A1C1422F20933C082A3099F02D3089F093
:109A50002A3321F480913D08882359F080913E08F3
:109A600090913F088F35910524F42F5F3F4F09F007
:109A7000F9C0209134063091350640913606509158
:109A8000370680912C0690912D06A0912E06B0915C
:109A90002F06281739074A075B0708F49BC0962D45
:109AA000E0E4F8E008C08091C00085FFFCCF90930F
:109AB000C600319694919923B1F78091C00085FF3B
:109AC000FCCF3092C6000E94171A609379067093FB
:109AD0007A0680937B0690937C06209175063091E0
:109AE00076064091770650917806621B730B840BC3
:109AF000950B28EE33E040E050E00E9413D5F22EA3
:109B0000E32ED42EC52EEDB7FEB738970FB6F894D6
:109B1000FEBF0FBEEDBF0DB71EB70F5F1F4FB28266
:109B2000A182F80153824282622F732F842F952FD6
:109B300020E13EE040E050E00E9413D5F80135837B
:109B400024836F2D7E2D8D2D9C2D2CE330E040E065
:109B500050E00E9413D5CA01B9012CE330E040E087
:109B600050E00E9413D5F801778366830E943FCDB1
:109B7000972DE4EEF5E02DB73EB7285F3F4F0FB6C7
:109B8000F8943EBF0FBE2DBF08C08091C00085FF76
:109B9000FCCF9093C600319694919923B1F7F501CB
:109BA00007C08091C00085FFFCCF31969093C6001E
:109BB00090819923B1F78091C00085FFFCCF30924E
:109BC000C60084E494E00E94E91C84E494E061E02F
:109BD0000E944F2320913E0830913F082115310506
:109BE00019F410923D08CEC0809140089091410830
:109BF000889DF001899DF00D989DF00D1124E20FD4
:109C0000F31FE454F94F1082FC01EE54F94F208207
:109C100020914608309147082F5F3F4F3093470807
:109C200020934608019664E070E00E9400D590936E
:109C300041088093400810923D0810923F0810920E
:109C40003E088091340690913506A0913606B09179
:109C500037068093480890934908A0934A08B09328
:109C60004B083AC04B3311F420923D0880913D08D7
:109C7000882391F520913E0830913F08809140085B
:109C800090914108889DF001899DF00D989DF00DFF
:109C90001124E20FF31FE454F94F80913C088083B4
:109CA0002F5F3F4F30933F0820933E0815C010E6CA
:109CB000812E912C22242394E0E4F8E06490BAE011
:109CC0003B2E5E010894A11CB11CACE24A2EA8E018
:109CD0005A2EE4EEF5E0749020913406309135066A
:109CE000409136065091370680912C0690912D06B2
:109CF000A0912E06B0912F06281739074A075B0757
:109D000008F040C080914608909147080497D4F528
:109D10008091190690911A06A0911B06B0911C061D
:109D20008093340690933506A0933606B093370699
:109D300081E196E00E941A709C018091EB058823D6
:109D400009F47FCE5CCE80914008909141088A9DB5
:109D500080018B9D100D9A9D100D1124C801845413
:109D6000994F6AE270E00E94DFCC9C01009709F4F1
:109D700008CDFF2440E0C801BCCC80914604882374
:109D800009F035CE6E960FB6F894DEBF0FBECDBF8C
:109D9000CF91DF911F910F91FF90EF90DF90CF90C7
:109DA000BF90AF909F908F907F906F905F904F90FB
:109DB0003F902F900895CF93DF9380914608909124
:109DC000470803970CF4C2DB84E494E060E00E944F
:109DD0004F238091460890914708892B09F469C068
:109DE00080914404882309F44CC02091B00630913E
:109DF000B10680E690E0289FE001299FD00D389FB2
:109E0000D00D1124C454D94FCE016CE879E00E94E2
:109E1000A4CC892BE1F484E494E0BE010E94E71D08
:109E200080914504882369F5E9E8F9E0949108C038
:109E30008091C00085FFFCCF9093C600319694912D
:109E40009923B1F78091C00085FFFCCF16C084E450
:109E500094E00E94CE1DE7E7F9E0949108C080915C
:109E6000C00085FFFCCF9093C60031969491992352
:109E7000B1F78091C00085FFFCCF8AE08093C600D7
:109E800002C00E945736809146089091470801977A
:109E900090934708809346088091B0069091B10650
:109EA000019664E070E00E9400D59093B106809323
:109EB000B0060E9424880E9499300E9481820E94EC
:109EC0007691DF91CF910895269A2E9880ED98E0B3
:109ED00040E950ED63E070E0AAD2E5E6FAE0949143
:109EE00008C08091C00085FFFCCF9093C6003196DA
:109EF00094919923B1F78091C00085FFFCCF8AE04F
:109F00008093C60044EE55E0FA01949108C0809118
:109F1000C00085FFFCCF9093C600319694919923A1
:109F2000B1F784B7282F80FF15C0EDE5FAE09491D2
:109F300008C08091C00085FFFCCF9093C600319689
:109F400094919923B1F78091C00085FFFCCF8AE0FE
:109F50008093C60021FF15C0EDE4FAE0949108C09B
:109F60008091C00085FFFCCF9093C60031969491FC
:109F70009923B1F78091C00085FFFCCF8AE08093E0
:109F8000C60022FF15C0ECE3FAE0949108C080916E
:109F9000C00085FFFCCF9093C60031969491992321
:109FA000B1F78091C00085FFFCCF8AE08093C600A6
:109FB00023FF15C0ECE2FAE0949108C08091C00044
:109FC00085FFFCCF9093C600319694919923B1F709
:109FD0008091C00085FFFCCF8AE08093C60025FFFA
:109FE00015C0ECE1FAE0949108C08091C00085FFB3
:109FF000FCCF9093C600319694919923B1F780914C
:10A00000C00085FFFCCF8AE08093C60014BEE4E167
:10A01000FAE0949108C08091C00085FFFCCF909336
:10A02000C600319694919923B1F7EEE0FAE094914D
:10A0300008C08091C00085FFFCCF9093C600319688
:10A0400094919923B1F78091C00085FFFCCF8AE0FD
:10A050008093C600FA019491E4EEF5E008C0809187
:10A06000C00085FFFCCF9093C60031969491992350
:10A07000B1F7EEEFF9E0949108C08091C00085FF40
:10A08000FCCF9093C600319694919923B1F7E9EEF5
:10A09000F9E0949108C08091C00085FFFCCF9093B7
:10A0A000C600319694919923B1F7EDEDF9E09491C2
:10A0B00008C08091C00085FFFCCF9093C600319608
:10A0C00094919923B1F7EDECF9E0949108C0809157
:10A0D000C00085FFFCCF9093C600319694919923E0
:10A0E000B1F78091C00085FFFCCF8AE08093C60065
:10A0F000E2ECF9E0949108C08091C00085FFFCCFAC
:10A100009093C600319694919923B1F7E6EBF9E06C
:10A11000949108C08091C00085FFFCCF9093C60049
:10A12000319694919923B1F78091C00085FFFCCFBF
:10A130008AE08093C600FA019491E4EEF5E008C04D
:10A140008091C00085FFFCCF9093C600319694911A
:10A150009923B1F7E7EAF9E0949108C08091C00033
:10A1600085FFFCCF9093C600319694919923B1F767
:10A170000E94B02EBC0180ED98E04AE050E098D2F9
:10A18000E0E9F9E0949108C08091C00085FFFCCF20
:10A190009093C600319694919923B1F780ED98E0A1
:10A1A00060ED74E04AE050E083D28091C00085FF0A
:10A1B000FCCF8AE08093C6001092B2061092B306DC
:10A1C0001092B4061092B5060E94B02C0E943887F7
:10A1D0000E945E5A0E948AC90E94917B0C94D89179
:10A1E000BC01809146089091470804970CF070C01C
:10A1F000209140083091410880E690E0AC01249F16
:10A20000C001259F900D349F900D11248454994FC7
:10A210000E946ECCE4EEF5E0949108C08091C000FD
:10A2200085FFFCCF9093C600319694919923B1F7A6
:10A23000EDE6FAE0949108C08091C00085FFFCCF64
:10A240009093C600319694919923B1F720914008DC
:10A250003091410880E690E0289FF001299FF00DA1
:10A26000389FF00D1124E454F94F07C08091C000CD
:10A2700085FFFCCF31969093C60090819923B1F76A
:10A28000EBE6FAE0949108C08091C00085FFFCCF16
:10A290009093C600319694919923B1F78091C000B4
:10A2A00085FFFCCF8AE08093C600C901019664E077
:10A2B00070E00E9400D590934108809340088091FF
:10A2C0004608909147080196909347088093460866
:10A2D0000895BC01809146089091470804970CF0BE
:10A2E00070C0209140083091410880E690E0AC01B8
:10A2F000249FC001259F900D349F900D11248454FC
:10A30000994F0E94EACCE4EEF5E0949108C0809168
:10A31000C00085FFFCCF9093C6003196949199239D
:10A32000B1F7EAE7FAE0949108C08091C00085FF98
:10A33000FCCF9093C600319694919923B1F7209168
:10A3400040083091410880E690E0289FF001299F65
:10A35000F00D389FF00D1124E454F94F07C080919F
:10A36000C00085FFFCCF31969093C6009081992361
:10A37000B1F7E8E7FAE0949108C08091C00085FF4A
:10A38000FCCF9093C600319694919923B1F78091B8
:10A39000C00085FFFCCF8AE08093C600C90101960A
:10A3A00064E070E00E9400D59093410880934008DB
:10A3B00080914608909147080196909347088093B2
:10A3C000460808951F920F920FB60F920BB60F9288
:10A3D00011242F933F934F938F939F93EF93FF936A
:10A3E0004091C600E091CC08F091CD0831969F01D4
:10A3F0002F77307031978091CE089091CF08281731
:10A40000390739F0E45BF74F40833093CD08209350
:10A41000CC08FF91EF919F918F914F913F912F9198
:10A420000F900BBE0F900FBE0F901F9018959A01C2
:10A43000AB01203081EE380780E0480780E0580704
:10A4400029F182E08093C00060E079E08DE390E044
:10A450000E9413D5215030404040504056954795BA
:10A46000379527953093C5002093C4008091C10093
:10A4700080618093C1008091C10088608093C10099
:10A480008091C10080688093C10008951092C0003F
:10A4900020E130E0E7CF2091CE083091CF088091C5
:10A4A000CC089091CD088217930719F42FEF3FEF56
:10A4B0000EC0F901E45BF74F80812F5F3F4F2F778C
:10A4C00030703093CF082093CE08282F30E0C90198
:10A4D00008958091CE089091CF089093CD088093F5
:10A4E000CC08089508952F923F924F925F926F92F9
:10A4F0007F928F929F92AF92BF92CF92DF92EF9214
:10A50000FF920F931F93DF93CF93CDB7DEB7A09742
:10A510000FB6F894DEBF0FBECDBF1C016A017B01F0
:10A52000411551056105710541F440E350E060E0DB
:10A5300070E020E030E089D053C088249924540191
:10A54000422E55246624772401E010E00C0F1D1FD5
:10A55000080D191DC701B601A30192010E9413D570
:10A56000F80160830894811C911CA11CB11CC701D7
:10A57000B601A30192010E9413D5C901DA016C0151
:10A580007D01C114D104E104F104F1F691E0E92E5A
:10A59000F12CEC0EFD1EE80CF91C3E010894611C28
:10A5A000711CD501C4010197A109B1096C01C8183A
:10A5B000D90813C0F601EE0DFF1D40814A3010F49A
:10A5C000405D01C0495C50E060E070E0C10120E006
:10A5D00030E03BD00894E108F1086E147F0451F795
:10A5E000A0960FB6F894DEBF0FBECDBFCF91DF911E
:10A5F0001F910F91FF90EF90DF90CF90BF90AF90A1
:10A600009F908F907F906F905F904F903F902F9092
:10A6100008952115310539F48091C00085FFFCCFE4
:10A620004093C60008955FCFEF92FF920F931F9360
:10A630009A01E62EFF2400E010E0B801A701E9DF4F
:10A640001F910F91FF90EF900895EF92FF920F935B
:10A650001F93CF93DF93EC017A018B012115310514
:10A6600039F48091C00085FFFCCFE092C60019C08C
:10A670002A303105A9F477FF0FC04DE250E060E0C9
:10A6800070E020E030E0E1DF10950095F094E09478
:10A69000E11CF11C011D111DCE01B801A7012AE02A
:10A6A00022DFDF91CF911F910F91FF90EF900895DE
:10A6B000EF92FF920F931F937B019A010027F7FC03
:10A6C0000095102FB801A701C0DF1F910F91FF90D7
:10A6D000EF9008950F931F938C014DE050E060E0E0
:10A6E00070E020E030E0B1DFC8014AE050E060E017
:10A6F00070E020E030E0A9DF1F910F910895CF9224
:10A70000DF92EF92FF920F931F938C019A016B01DE
:10A71000EE24FF24B701A6017CDFC801DBDF1F9117
:10A720000F91FF90EF90DF90CF9008959F92AF929E
:10A73000BF92CF92DF92EF92FF920F931F93CF932E
:10A74000DF93EC017A018B01922ECB01BA0120E05C
:10A7500030E040E050E00E9449CE882364F4CE010E
:10A760004DE250E060E070E020E030E06EDF17FB8B
:10A77000109517F9109520E030E040E05FE3AA243F
:10A780000BC0CA01B90120E030E040E251E40E9470
:10A7900050CE9B01AC01A394A91498F3C801B70152
:10A7A0000E9470CD7B018C010E94BDCE5B016C01CB
:10A7B0000E94E9CE9B01AC01C801B7010E946FCD98
:10A7C0007B018C01CE01B601A5012AE030E021DF3A
:10A7D000992099F1EEEDF2E007C08091C00085FF6D
:10A7E000FCCF31969093C60090819923B1F725C094
:10A7F000C801B70120E030E040E251E40E941ED1E0
:10A800007B018C010E94B8CE5B016C01CC24B7FCAB
:10A81000C094DC2CCE01B601A5012AE030E015DFA2
:10A82000C601B5010E94EBCE9B01AC01C801B70186
:10A830000E946FCD7B018C019A949920C9F6DF911B
:10A84000CF911F910F91FF90EF90DF90CF90BF902D
:10A85000AF909F9008956ACF08952F923F924F92A4
:10A860005F926F927F928F929F92AF92BF92CF92A0
:10A87000DF92EF92FF920F931F93DF93CF93CDB7A9
:10A88000DEB7CD55D0400FB6F894DEBF0FBECDBFBA
:10A890002F969FAF8EAF2F9761967FAF6EAF619768
:10A8A0002A0162962FAF629763960FAF6397649603
:10A8B000EFAE64976896ACAEBDAECEAEDFAE689735
:10A8C000E22EFF24EE0CFF1CEE0CFF1C9A012E0D55
:10A8D0003F1D2D963FAF2EAF2D97D9016D907D90E6
:10A8E0008D909C90FC01EE0DFF1DC401B3012081F1
:10A8F0003181428153810E9470CD69AF7AAF8BAFB5
:10A900009CAF10E0000F111F000F111FF201E00FAC
:10A91000F11F2B96FFAFEEAF2B97A080B180C280C6
:10A92000D3802F96EEADFFAD2F97E00FF11FC6013C
:10A93000B50120813181428153810E9470CD6DAB80
:10A940007EAB8FAB98AF64962FAD6497E22FF0E0AB
:10A95000EE0FFF1FEE0FFF1F2F96AEADBFAD2F976F
:10A96000AE0FBF1F4D915D916D917C9129964CAFBB
:10A970005DAF6EAF7FAF299761966EAD7FAD61978A
:10A98000E60FF71F608171818281938129962CAD3A
:10A990003DAD4EAD5FAD29970E946FCD69AB7AABEF
:10A9A0008BAB9CAB6196AEADBFAD61971C968D91A4
:10A9B0009D910D90BC91A02D25968CAF9DAFAEAF13
:10A9C000BFAF25972F96AEADBFAD2F971C962D919B
:10A9D0003D914D915C911F9721962CAF3DAF4EAFAD
:10A9E0005FAF2197A401930150582DA73EA74FA711
:10A9F00058ABB601A501705849A75AA76BA77CA709
:10AA000061966EAD7FAD6197E60EF71ED7016D9131
:10AA10007D918D919C9129AD3AAD4BAD5CAD0E947D
:10AA20006FCD3B014C016196EEADFFAD61970E0F0E
:10AA30001F1FD8016D917D918D919C912DA93EA9EB
:10AA40004FA958AD0E946FCD5B016C016DA57EA52D
:10AA50008FA598A9A60195010E941ED17B018C01AA
:10AA600069A57AA58BA59CA5A40193010E941ED17E
:10AA70009B01AC01C801B7010E946FCD1B012C01E5
:10AA80006DA57EA58FA598A9A40193010E941ED152
:10AA90007B018C0169A57AA58BA59CA5A6019501D2
:10AAA0000E941ED19B01AC01C801B7010E9470CD6C
:10AAB0009B01AC01C201B1010E94E3CD5B016C01BD
:10AAC00020E030E040E050E00E9449CE882354F47A
:10AAD000C601B5012BED3FE049EC50E40E9470CD7A
:10AAE0005B016C01E8968FADE897882351F0C601B1
:10AAF000B5012BED3FE049EC50E40E946FCD5B01C6
:10AB00006C01C601B501E7962CAD3DAD4EAD5FAD14
:10AB1000E7970E941ED129A93AA94BA95CA95F77A2
:10AB20000E9459D07B018C012FE632E143E85AE3C1
:10AB30000E9449CE87FDF4C1C801B7010E9426CF0B
:10AB40000E94BDCE78A76FA3672B21F4E1E0F0E06F
:10AB5000F8A7EFA32FA138A5B90180E090E00E94EB
:10AB6000E9CE7B018C01C601B501A80197010E94C5
:10AB700050CE6BA37CA38DA39EA369A97AA98BA9B0
:10AB80009CA9A80197010E9450CE6F8F78A389A33A
:10AB90009AA325966CAD7DAD8EAD9FAD2597219680
:10ABA0002CAD3DAD4EAD5FAD21970E946FCDA8019C
:10ABB00097010E9450CE6B8F7C8F8D8F9E8F6BA1E3
:10ABC0007CA18DA19EA120E030E040E05FEB0E94DF
:10ABD0001ED12BA13CA14DA15EA10E941ED120E05F
:10ABE00030E040E85FE30E9470CD6F8B788F898FF3
:10ABF0009A8F64963FAD6497E32FF0E0EE0FFF1F4E
:10AC0000EE0FFF1F9E012F5F3F4FE20FF31F2996AC
:10AC10004CAD5DAD6EAD7FAD2997408351836283AE
:10AC200073832F96AEADBFAD2F971C964D915D915E
:10AC30006D917C911F974D875E876F87788B41E080
:10AC400050E05A8B498B662462967FAD6297672FDE
:10AC500070E0660F771F660F771FC901860F971F79
:10AC60006A969FAF8EAF6A976396BFAD6397AB2F1F
:10AC7000B0E0AA0FBB1FAA0FBB1F21E030E02C0FD2
:10AC80003D1F2A0F3B1F6C963FAF2EAF6C976E9601
:10AC9000FFAFEEAF6E9719C138E136150CF446C020
:10ACA0006DA57EA58FA598A92BA13CA14DA15EA164
:10ACB0000E941ED17B018C0169A57AA58BA59CA55C
:10ACC0002F89388D498D5A8D0E941ED19B01AC0170
:10ACD000C801B7010E9470CD7B018C016DA57EA5D6
:10ACE0008FA598A92F89388D498D5A8D0E941ED124
:10ACF0005B016C0169A57AA58BA59CA52BA13CA144
:10AD00004DA15EA10E941ED19B01AC01C601B501FF
:10AD10000E946FCD6DA77EA78FA798AB6394C701E4
:10AD2000D80189A79AA7ABA7BCA765C049895A894A
:10AD3000BA0180E090E00E94E9CE2BA13CA14DA198
:10AD40005EA10E941ED17B018C01C8010E944DCEE4
:10AD50006B8B7C8B8D8B9E8BB701C8010E9481D140
:10AD60003B014C012D96AEADBFAD2D97ED90FD9002
:10AD70000D911C9117FB109517F910952B96EEADC0
:10AD8000FFAD2B972080318042805380C801B701EE
:10AD90002B893C894D895E890E941ED15B016C0123
:10ADA000C201B101A40193010E941ED19B01AC011B
:10ADB000C601B5010E9470CD6DA77EA78FA798AB85
:10ADC000C801B701A40193010E941ED17B018C012F
:10ADD000C201B1012B893C894D895E890E941ED137
:10ADE0009B01AC01C801B7010E946FCD69A77AA78A
:10ADF0008BA79CA7662469AD7AAD8BAD9CAD2DA5C4
:10AE00003EA54FA558A90E9470CD6A96AEADBFADC4
:10AE10006A976D937D938D939C9313976DA97EA9EB
:10AE20008FA998AD29A53AA54BA55CA50E9470CD28
:10AE30006C96EEADFFAD6C976083718382839383D4
:10AE40006E96AEADBFAD6E976D917D918D919C91DB
:10AE50002F8D38A149A15AA10E9470CD6E96EEADFA
:10AE6000FFAD6E9760837183828393836D857E854A
:10AE70008F8598892B8D3C8D4D8D5E8D0E9470CD78
:10AE80006D877E878F87988BCE0101960E94332F26
:10AE9000CE010196BE016B5F7F4FAE01475F5F4FF2
:10AEA0009E01235F3F4F6896ECACFDAC0EAD1FAD2D
:10AEB0006897F8E7CF2ED12CCC0EDD1EC2D529899C
:10AEC0003A892F5F3F4F3A8B298B49895A896FA165
:10AED00078A54617570708F4DFCE61964EAD5FADF3
:10AEE0006197485F5F4F61962EAD3FAD6197245FDC
:10AEF0003F4F61968EAD9FAD6197DC0114966196D0
:10AF0000BFAFAEAF6197BD016896ECACFDAC0EADC6
:10AF10001FAD6897E8E7CE2ED12CCC0EDD1E91D563
:10AF2000C35ADF4F0FB6F894DEBF0FBECDBFCF912F
:10AF3000DF911F910F91FF90EF90DF90CF90BF9026
:10AF4000AF909F908F907F906F905F904F903F90C9
:10AF50002F9008958091110E9091120E891B8F7081
:10AF6000089560937E0370937F0380938003909392
:10AF7000810308950F931F93CF93DF93C0E0D0E038
:10AF80008E010F5D164FFE01EB50F74F608171810E
:10AF9000828193810E94E9CEFE01EB51F74F20811F
:10AFA0003181428153810E941ED10E94BDCEF801A1
:10AFB00060837183828393832496C031D10501F726
:10AFC000DF91CF911F910F910895FC0160817181F4
:10AFD000828193812091F1083091F2084091F30829
:10AFE0005091F4080E941ED120917A0330917B0386
:10AFF00040917C0350917D030E941ED10E94EED0AF
:10B0000060933D0970933E0980933F0990934009F6
:10B010008DE399E00C94E17A8F929F92AF92BF9268
:10B02000CF92DF92EF92FF920F931F93FC018B015F
:10B030005A01490160817181828193812091E508E3
:10B040003091E6084091E7085091E8080E941ED12F
:10B050000E94EED031E3C32E39E0D32E6093310944
:10B06000709332098093330990933409F801608119
:10B070007181828193812091E9083091EA084091A1
:10B08000EB085091EC080E941ED10E94EED024E003
:10B09000E22EF12CEC0CFD1C60933509F701718355
:10B0A00082839383F50160817181828193812091F4
:10B0B000ED083091EE084091EF085091F0080E94A1
:10B0C0001ED10E94EED08601085F1F4F60933909A0
:10B0D000F801718382839383F4016081718182819D
:10B0E00093812091F1083091F2084091F30850913A
:10B0F000F4080E941ED120917A0330917B03409185
:10B100007C0350917D030E941ED10E94EED0F60177
:10B110003C9660933D09718382839383C601B70196
:10B12000A8019F010E94A77A80E090E0A0E0B0E033
:10B130008093130E9093140EA093150EB093160ED9
:10B140008093170E9093180EA093190EB0931A0EB9
:10B1500080931B0E90931C0EA0931D0EB0931E0E99
:10B1600080931F0E9093200EA093210EB093220E79
:10B170008093230E9093240EA093250EB093260E59
:10B180001F910F91FF90EF90DF90CF90BF90AF9005
:10B190009F908F9008958F929F92AF92BF92CF927F
:10B1A000DF92EF92FF920F931F93CF93DF93EC0107
:10B1B0006B01009709F45CC08FA9882309F058C07F
:10B1C000EEA0FFA008A519A5FB01B6A0A7A090A41A
:10B1D00081A4C801B7012B2D3A2D492D582D0E946D
:10B1E00049CE88230CF044C0C801B701A8019701DB
:10B1F0000E941ED17B018C016AA97BA98CA99DA903
:10B20000905820E030E040E050EC0E941ED12EA586
:10B210003FA548A959A90E941ED19B01AC01C801B4
:10B22000B7010E9470CD0E948BD17B018C016B2DE8
:10B230007A2D892D982D9701A8010E9449CE882347
:10B2400024F4EB2CFA2C092D182D6B2D7A2D892D39
:10B25000982D9701A8010E9449CE882349F0C70183
:10B26000D801F60186A397A3A0A7B1A781E086AB7A
:10B27000DF91CF911F910F91FF90EF90DF90CF90D2
:10B28000BF90AF909F908F900895EF92FF920F9391
:10B290001F93CF93DF93F090120E00E010E020E0B8
:10B2A00030E04DE4E42E11C0FE9CE0011124CF5BA0
:10B2B000D64FC901B801AE016EDF8F2D8F5F80318F
:10B2C00009F480E0F82E98018E018091110EF81695
:10B2D00059F7C901B80140E050E05DDFDF91CF913F
:10B2E0001F910F91FF90EF900895AF92BF92CF9270
:10B2F000DF92EF92FF920F931F93CF93DF93EB01B7
:10B300008A016115710509F466C04115510509F4FA
:10B3100062C0DAA4CBA4BCA4ADA46EA17FA188A511
:10B3200099A52D2D3C2D4B2D5A2D0E9449CE8823B9
:10B3300009F451C08FA9882309F043C0F801E6A0A1
:10B34000F7A000A511A56D2D7C2D8B2D9A2DA801A0
:10B3500097010E944CD01816A4F5C801B701A801A6
:10B3600097010E941ED17B018C016AA97BA98CA93F
:10B370009DA9905820E030E040E050EC0E941ED1A2
:10B380002EA53FA548A959A90E941ED19B01AC0139
:10B39000C801B7010E9470CD0E948BD17B018C0146
:10B3A0006D2D7C2D8B2D9A2D9701A8010E9449CEE1
:10B3B000882324F4ED2CFC2C0B2D1A2DC701D80169
:10B3C00004C08D2D9C2DAB2DBA2D8EA39FA3A8A7B5
:10B3D000B9A781E08EABDF91CF911F910F91FF90C4
:10B3E000EF90DF90CF90BF90AF900895CF92DF9213
:10B3F000EF92FF920F93DF93CF930F920F92CDB7FF
:10B40000DEB78091110E8FB7F894F090120E8FBFB7
:10B410008091110E90E040968F1991098F70907075
:10B420000497FCF00091110E03500F70CC24DD2422
:10B4300040E050E06DE4E62E12C0802F002309F4B6
:10B4400080E1082F01500E9DC00111248F5B964FA3
:10B450009A838983B60149DFA601C980DA800F1576
:10B4600061F70F900F90CF91DF910F91FF90EF90C8
:10B47000DF90CF90089560916D069091120E8091AB
:10B48000110E9817B9F04091120E242F30E08DE480
:10B4900090E0289FF001299FF00D389FF00D1124B6
:10B4A000E757F64F608102C04F5F4F708091110ED9
:10B4B0004817D1F787E070E00C94871A1092110EAC
:10B4C0001092120E80E1E1E3F9E0DF011D928A950E
:10B4D000E9F780E090E0A0E0B0E08093170E909351
:10B4E000180EA093190EB0931A0E80931B0E909312
:10B4F0001C0EA0931D0EB0931E0E80931F0E9093F2
:10B50000200EA093210EB093220E8093230E9093D1
:10B51000240EA093250EB093260E8093130E9093C5
:10B52000140EA093150EB093160E08952F923F920D
:10B530004F925F926F927F928F929F92AF92BF9243
:10B54000CF92DF92EF92FF920F931F93DF93CF93EF
:10B55000CDB7DEB766970FB6F894DEBF0FBECDBF8E
:10B560009E8B8D8B6A017B0148015901DC01D896C5
:10B570006D917D918D919C91DB970E94E9CE698BB5
:10B580007A8B8B8B9C8BA70196010E941ED10E9407
:10B5900036CE0E94BDCE6D837E838F839887698966
:10B5A0007A898B899C89A50194010E941ED10E94F1
:10B5B00036CE0E94BDCE69837A838B839C832D8196
:10B5C0003E814F815885283731054105510540F4AA
:10B5D00048E750E060E070E04D835E836F837887DA
:10B5E00069817A818B819C8168377105810591051C
:10B5F00040F488E790E0A0E0B0E089839A83AB83D1
:10B60000BC83AD89BE89AC5BBF4FAD90BD90CD9082
:10B61000DC901397A454B040BE8BAD8BDC966D913B
:10B620007D918D919C91DF970E94E9CE6D877E87F9
:10B630008F87988BC601B5010E94EBCE1B012C01B0
:10B6400020E030E040E050E00E9449CE882321F421
:10B65000E0E070E060E028C069897A898B899C8984
:10B660009B01AC010E941ED17B018C016D857E8502
:10B670008F8598899B01AC010E941ED19B01AC0172
:10B68000C801B7010E946FCD7B018C01C201B101DD
:10B69000A20191010E9470CD9B01AC01C801B701CC
:10B6A0000E9450CEE62F692F2E2F372F482F562F6E
:10B6B000B901CA010E9436CE0E94B8CE3B014C01AE
:10B6C000ED89FE89E05CFF4F608171818281938109
:10B6D0000E94E9CE69877A878B879C8766277727C0
:10B6E000CB016A197B098C099D090E94EBCE5B0195
:10B6F0006C0120E030E040E050E00E9449CE882319
:10B7000021F4E0E070E060E028C069857A858B85EF
:10B710009C859B01AC010E941ED17B018C01698933
:10B720007A898B899C899B01AC010E941ED19B0167
:10B73000AC01C801B7010E946FCD7B018C01C6012D
:10B74000B501A60195010E9470CD9B01AC01C80115
:10B75000B7010E9450CEE62F692F2E2F372F482F8A
:10B76000562FB901CA010E9426CFED89FE89A08813
:10B77000B188C288D38886017501E618F7080809E0
:10B7800019090E94B8CEA8019701261B370B480B58
:10B79000590B57FF71C0C201B10120E030E040E019
:10B7A00050E00E9449CE882321F4E0E070E060E0A0
:10B7B00044C0C201B101A20191010E9470CD7B0180
:10B7C0008C01C601B5010E94E9CE9B01AC01C80104
:10B7D000B7010E941ED17B018C016D857E858F850E
:10B7E00098899B01AC010E941ED19B01AC01C8014C
:10B7F000B7010E946FCD7B018C0169857A858B85AD
:10B800009C859B01AC010E941ED19B01AC01C8012B
:10B81000B7010E9470CD7B018C01C201B10120E013
:10B8200030E040E850E40E941ED19B01AC01C80109
:10B83000B7010E9450CEE62F692F2E2F372F482FA9
:10B84000562FB901CA010E9436CE0E94B8CEAC0173
:10B85000CB01DA013C014D0197FE03C06624772439
:10B8600043016A147B048C049D0410F035014601E9
:10B8700020E030E040E050E09FB7F8946D897E8989
:10B88000645B7F4FDB018C91AC54B040BE8BAD8BC1
:10B89000882321F5FD01648A758A868A978A260D98
:10B8A000371D481D591D58962D933D934D935C931C
:10B8B0005B972D813E814F815885DC962D933D937A
:10B8C0004D935C93DF97A05CBF4F29813A814B81F8
:10B8D0005C812D933D934D935C9313979FBF669628
:10B8E0000FB6F894DEBF0FBECDBFCF91DF911F9191
:10B8F0000F91FF90EF90DF90CF90BF90AF909F900F
:10B900008F907F906F905F904F903F902F90089511
:10B910004F925F927F928F929F92AF92BF92CF92FF
:10B92000DF92EF92FF920F931F93CF93DF9370906C
:10B93000120EC0E0D0E07DE4472E512C45C0209788
:10B94000A9F18EA9882361F4849CF001859CF00DF7
:10B95000949CF00D1124EF5BF64F86A9882331F1FA
:10B96000EAA0FBA00CA11DA16EA17FA188A599A5AD
:10B97000A80197010E9450CE5B016C01849CF001EC
:10B98000859CF00D949CF00D1124EF5BF64F66A1A1
:10B9900077A180A591A5A80197010E9450CE8B01A7
:10B9A0009C01CE01B601A501C1DD1EAA739480E100
:10B9B000781609F47724849CE001859CD00D949C32
:10B9C000D00D1124CF5BD64F872C992487FC9094FF
:10B9D0008091110E90E08816990609F0B0CF20975B
:10B9E000E9F0EAA0FBA00CA11DA16EA17FA188A592
:10B9F00099A5A80197010E9450CE5B016C016DECE6
:10BA00007CEC8CE49DE3A80197010E9450CE8B0151
:10BA10009C01CE01B601A50189DD1EAADF91CF915F
:10BA20001F910F91FF90EF90DF90CF90BF90AF905C
:10BA30009F908F907F905F904F900895D7DC25DC8A
:10BA400067CF2F923F924F925F926F927F928F9229
:10BA50009F92AF92BF92CF92DF92EF92FF920F939D
:10BA60001F93DF93CF93CDB7DEB7C859D0400FB641
:10BA7000F894DEBF0FBECDBF5C014B013A01290136
:10BA8000CB56DF4FE882C559D040CA56DF4FF88207
:10BA9000C659D040C956DF4F0883C759D040C85651
:10BAA000DF4F1883C859D040E396DFAECEAEE397A0
:10BAB0008091110E8F5F803109F480E0282F3327A9
:10BAC00027FD30953CA72BA706C00E9424880E9422
:10BAD00099300E9476918091120E90E04BA55CA562
:10BAE0008417950791F36091E5087091E6088091BD
:10BAF000E7089091E808E1966CAF7DAF8EAF9FAFFD
:10BB0000E197D5012D913D914D915C910E941ED1FF
:10BB10000E94EED0C158DF4F6883CF57D040C05845
:10BB2000DF4F7883C058D040CF57DF4F8883C1584C
:10BB3000D040CE57DF4F9883C258D0402091E908BB
:10BB40003091EA084091EB085091EC08AD962CAF8B
:10BB50003DAF4EAF5FAFAD97CA01B901D4012D9192
:10BB60003D914D915C910E941ED10E94EED0CD5727
:10BB7000DF4F6883C358D040CC57DF4F7883C45819
:10BB8000D040CB57DF4F8883C558D040CA57DF4FCE
:10BB90009883C658D0402091ED083091EE0840912E
:10BBA000EF085091F008A9962CAF3DAF4EAF5FAFB4
:10BBB000A997CA01B901D3012D913D914D915C9195
:10BBC0000E941ED10E94EED0C957DF4F6883C7582C
:10BBD000D040C857DF4F7883C858D040C757DF4F91
:10BBE0008883C958D040C657DF4F9883CA58D04081
:10BBF0002091F1083091F2084091F3085091F40837
:10BC0000A5962CAF3DAF4EAF5FAFA597CA01B90166
:10BC1000D2012D913D914D915C910E941ED12091B8
:10BC20007A0330917B0340917C0350917D030E9405
:10BC30001ED10E94EED0C557DF4F6883CB58D0404D
:10BC4000C457DF4F7883CC58D040C357DF4F888329
:10BC5000CD58D040C257DF4F9883CE58D040809106
:10BC60003D0990913E09A0913F09B0914009C55707
:10BC7000DF4F288139814A815B81CB58D04028171A
:10BC800039074A075B0709F4B8C0E0916C06F0E099
:10BC9000EE0FFF1FEE0FFF1FEE57FF4E6081718109
:10BCA0008281938120917E0330917F0340918003B4
:10BCB000509181030E9449CE88230CF033C0C557B0
:10BCC000DF4F488159816A817B81CB58D0404093B6
:10BCD0003D0950933E0960933F0970934009E5E8A0
:10BCE000FAE0949108C08091C00085FFFCCF90934A
:10BCF000C600319694919923B1F7E9EAFAE094915C
:10BD000008C08091C00085FFFCCF9093C60031969B
:10BD100094919923B1F78091C00085FFFCCF8AE010
:10BD20008093C60080913D0990913E09A0913F0902
:10BD3000B0914009C557DF4F288139814A815B8125
:10BD4000CB58D040281B390B4A0B5B0BCA01B901F9
:10BD500057FF07C090958095709561957F4F8F4FE5
:10BD60009F4F0E94EBCE7B018C01A5966CAD7DAD03
:10BD70008EAD9FADA59720E030E843EE53E40E94DE
:10BD80001ED19B01AC01C801B7010E944CD018160E
:10BD90000CF033C0C557DF4F488159816A817B81E0
:10BDA000CB58D04040933D0950933E0960933F09E2
:10BDB00070934009E5E8FAE0949108C08091C000D2
:10BDC00085FFFCCF9093C600319694919923B1F7EB
:10BDD000EBE8FAE0949108C08091C00085FFFCCFA9
:10BDE0009093C600319694919923B1F78091C00049
:10BDF00085FFFCCF8AE08093C6008091110E682FEA
:10BE000070E0A1967FAF6EAFA1978DE490E0689F40
:10BE1000F001699FF00D789FF00D1124EF5BF64F54
:10BE2000E45BFF4F1082EC54F04080913109909117
:10BE30003209A0913309B09134096F968CAF9DAF50
:10BE4000AEAFBFAF6F97C158DF4F288139814A81AC
:10BE50005B81CF57D040281B390B4A0B5B0B6B968D
:10BE60002CAF3DAF4EAF5FAF6B97208331834283E2
:10BE7000538357FF0DC0DA01C901B095A095909585
:10BE800081959F4FAF4FBF4F80839183A283B38330
:10BE90004091350950913609609137097091380900
:10BEA00067964CAF5DAF6EAF7FAF6797CD57DF4FF3
:10BEB00088819981AA81BB81C358D040841B950B8E
:10BEC000A60BB70B63968CAF9DAFAEAFBFAF6397BA
:10BED0008DE490E0A196AEADBFADA197A89FF00113
:10BEE000A99FF00DB89FF00D1124EF5BF64F6396FC
:10BEF0002CAD3DAD4EAD5FAD639724833583468356
:10BF0000578357FF0DC0DA01C901B095A0959095F0
:10BF100081959F4FAF4FBF4F84839583A683B7838F
:10BF20004091390950913A0960913B0970913C095F
:10BF30002F964CAF5DAF6EAF7FAF2F97C957DF4FD6
:10BF400088819981AA81BB81C758D040841B950BF9
:10BF5000A60BB70B2B968CAF9DAFAEAFBFAF2B9799
:10BF60008DE490E0A196AEADBFADA197A89FF00182
:10BF7000A99FF00DB89FF00D1124EF5BF64F2B96A3
:10BF80002CAD3DAD4EAD5FAD2B97208731874287FD
:10BF9000538757FF0DC0DA01C901B095A095909560
:10BFA00081959F4FAF4FBF4F80879187A287B387FF
:10BFB00020903D0930903E0940903F095090400943
:10BFC000C557DF4F488159816A817B81CB58D0406A
:10BFD00042195309640975094DA35EA36FA378A79D
:10BFE000609152037091530327967FAF6EAF2797EE
:10BFF0006DA17EA18FA198A597FF07C09095809510
:10C00000709561957F4F8F4F9F4F2796AEADBFAD17
:10C0100027979D01442737FD4095542F0E94C1D496
:10C0200024E630E040E050E00E9435D58DE490E019
:10C03000A1966EAD7FADA197689FF001699FF00D4D
:10C04000789FF00D1124EF5BF64FDF011C962487DB
:10C0500011963C93119712964C93129713965C93FA
:10C060006080718082809380A480B580C680D780F4
:10C07000E084F18402851385C901DA018E159F05DC
:10C08000A007B10714F4D801C7018A159B05AC05B8
:10C09000BD0514F4D601C5019C01AD0186159705B7
:10C0A000A805B90514F4A40193018DE490E0A196CC
:10C0B000AEADBFADA197A89FB001A99F700DB89F6D
:10C0C000700D11246F5B764FFB01208B318B428BFF
:10C0D000538B263031054105510510F40C945A69F3
:10C0E000E85BFF4F80916D0690E0A0E0B0E08083B8
:10C0F0009183A283B383DB0190961C92C158DF4FDA
:10C10000288139814A815B81CF57D0406F968CADB1
:10C110009DADAEADBFAD6F97281739074A075B07D6
:10C1200024F481E0DB0190968C93CD57DF4F28817A
:10C1300039814A815B81C358D04067966CAD7DAD33
:10C140008EAD9FAD6797261737074807590794F4B8
:10C150008DE490E0A196AEADBFADA197A89FF00190
:10C16000A99FF00DB89FF00D1124EF5BF64F80A151
:10C17000826080A3C957DF4F288139814A815B8162
:10C18000C758D0402F966CAD7DAD8EAD9FAD2F972B
:10C19000261737074807590794F48DE490E0A196D5
:10C1A000AEADBFADA197A89FF001A99FF00DB89FBC
:10C1B000F00D1124EF5BF64F80A1846080A3C5577A
:10C1C000DF4F288139814A815B81CB58D0402215CD
:10C1D00033054405550594F48DE490E0A1964EADE9
:10C1E0005FADA197489FF001499FF00D589FF00D5A
:10C1F0001124EF5BF64F80A1886080A38DE490E06E
:10C20000A1966EAD7FADA197689FF001699FF00D7B
:10C21000789FF00D1124EF5BF64FE396AEADBFAD06
:10C22000E3978C9181A320813181428153812596AE
:10C230002CAF3DAF4EAF5FAF2597211531054105BE
:10C24000510509F015988DE490E0A1964EAD5FADD3
:10C25000A197489FF001499FF00D589FF00D1124C0
:10C26000EF5BF64F6480758086809780611471045F
:10C270008104910409F046988DE490E0A1966EAD9A
:10C280007FADA197689FF001699FF00D789FF00D39
:10C290001124EF5BF64FA084B184C284D384A1142F
:10C2A000B104C104D10409F043988DE490E0A19653
:10C2B000AEADBFADA197A89FF001A99FF00DB89FAB
:10C2C000F00D1124EF5BF64F84859585A685B78523
:10C2D0000097A105B10551F04098209005093090D4
:10C2E0000609409007095090080908C020901D09D0
:10C2F00030901E0940901F0950902009CB56DF4F07
:10C300006881C559D040CA56DF4F7881C659D040A0
:10C31000C956DF4F8881C759D040C856DF4F988132
:10C32000C859D040A20191010E9449CE87FD16C094
:10C33000CB56DF4F8881C559D040CA56DF4F988110
:10C34000C659D040C956DF4FA881C759D040C856FA
:10C35000DF4FB881C859D0401C012D016B966CADE0
:10C360007DAD8EAD9FAD6B970E94EBCEE1962CAD6F
:10C370003DAD4EAD5FADE1970E9450CEEC966FAFF4
:10C38000EC97ED967FAFED97EE968FAFEE97EF9629
:10C390009FAFEF97AC01CB01DA0189839A83AB831E
:10C3A000BC8363966CAD7DAD8EAD9FAD63970E94EF
:10C3B000EBCEAD962CAD3DAD4EAD5FADAD970E94D1
:10C3C00050CEE8966FAFE897E9967FAFE997EA9687
:10C3D0008FAFEA97EB969FAFEB97AC01CB01DA01F9
:10C3E0008D839E83AF83B8872B966CAD7DAD8EAD6C
:10C3F0009FAD2B970E94EBCEA9962CAD3DAD4EADD7
:10C400005FADA9970E9450CEE4966FAFE497E59692
:10C410007FAFE597E6968FAFE697E7969FAFE797F2
:10C42000AC01CB01DA0189879A87AB87BC876DA104
:10C430007EA18FA198A50E94EBCEA5962CAD3DAD17
:10C440004EAD5FADA5970E9450CE7B018C01279623
:10C45000EEADFFAD2797BF01882777FD8095982F18
:10C460000E94EBCE9B01AC01C801B7010E941ED116
:10C4700020E030E048EC52E40E9450CE9B01AC0139
:10C480006D877E878F87988B25966CAD7DAD8EAD41
:10C490009FAD259766307105810591051CF576E005
:10C4A0006716710481049104ECF486E0A816B104C7
:10C4B000C104D104BCF48DE490E0A196AEADBFAD53
:10C4C000A197A89FF001A99FF00DB89FF00D11242E
:10C4D000EF5BF64FDA01C901BF7786A797A7A0AB3C
:10C4E000B1AB55C0EC962FADEC97ED963FADED9707
:10C4F000EE964FADEE97EF965FADEF97B901CA019B
:10C500000E94C9D13B014C01E8962FADE897E9960E
:10C510003FADE997EA964FADEA97EB965FADEB97A3
:10C52000B901CA010E94C9D15B016C01E4962FAD2B
:10C53000E497E5963FADE597E6964FADE697E7962B
:10C540005FADE797B901CA010E94C9D17B018C0197
:10C55000C401B301A60195010E9470CDA801970105
:10C560000E9470CD0E948BD12DE430E0A1964EAD9B
:10C570005FADA197429FF001439FF00D529FF00DD8
:10C580001124EF5BF64F66A777A780AB91AB8DE4E4
:10C5900090E0A1966EAD7FADA197689FF001699F75
:10C5A000F00D789FF00D1124EF5BF64F86A597A54F
:10C5B000A0A9B1A921968CAF9DAFAEAFBFAF219717
:10C5C00060E070E080E89FE321962CAD3DAD4EAD7C
:10C5D0005FAD21970E9450CE9B01AC01C201B10119
:10C5E0000E941ED12B013C018091110E9091120EE0
:10C5F000A82FB0E05096A91BB109AF70B070BAA7D0
:10C60000A9A7A230B1050CF451C05D01CC24B7FC40
:10C61000C094DC2CC601B5010E94EBCE20E030E0D6
:10C6200040E051E40E9449CE88230CF03FC060E016
:10C6300074E284E799E4A30192010E9450CE0E9423
:10C64000EED07B018C016091D1087091D20880916D
:10C65000D3089091D408E616F7060807190730F5B5
:10C660006E197F09800B910B660F771F881F991F2A
:10C67000A60195010E9413D5CA01B9010E94E9CE15
:10C680000E94EED09B01AC012E0D3F1D401F511F9B
:10C69000CA01B9010E94E9CE9B01AC0160E074E2DD
:10C6A00084E799E40E9450CE2B013C018DE490E098
:10C6B000A196EEADFFADA197E89F8001E99F100D17
:10C6C000F89F100D11240F5B164F21966CAD7DADB8
:10C6D0008EAD9FAD2197A30192010E941ED1D8017A
:10C6E00092966D937D938D939C93959750966D91B3
:10C6F0007D918D919C9153970E94E9CEA301920167
:10C700000E941ED10E9436CE0E94BDCEF80160AFBD
:10C7100071AF82AF93AFC157DF4F1882CF58D0406F
:10C72000C057DF4F1882C059D04020E8222E9FE327
:10C73000392E88249924E1E0F0E0EC0FFD1FE80D8C
:10C74000F91DC301B20120813181428153810E94D0
:10C750001ED1E1E1F0E0EC0FFD1FE80DF91D608353
:10C760007183828393835B016C01E894D7F8F401B1
:10C77000EB52F74FE080F18002811381C601B501D1
:10C78000A80197010E944CD01816CCF4C801B7013B
:10C79000A60195010E9450CE6B017C01C157DF4F6D
:10C7A0006881CF58D040C057DF4F7881C059D04002
:10C7B000C101A70196010E9449CE88236CF4C1579C
:10C7C000DF4F8881CF58D040C057DF4F9881C05984
:10C7D000D040D1016C017D0124E030E0820E931E37
:10C7E00030E18316910471F0D701C601C157DF4FC4
:10C7F000C882CF58D040C057DF4F9883C059D0402F
:10C800001D0199CFC701B60120E030E040E85FE3A9
:10C810000E9449CE88230CF04CC08E010F5E1F4F42
:10C8200081E2A82EB12CAC0EBD1ED8016D917D9178
:10C830008D919C91A70196010E941ED1F8016193F0
:10C840007193819391938F01EA15FB0571F78DE444
:10C8500090E0A1962EAD3FADA197289F8001299F22
:10C86000100D389F100D11240F5B164FD8019296B2
:10C870006D917D918D919C919597A70196010E9454
:10C880001ED1F80162A373A384A395A360AD71AD1B
:10C8900082AD93AD0E94E9CEA70196010E941ED100
:10C8A0000E94BDCED801D8966D937D938D939C93B5
:10C8B000DB978DE490E0A196EEADFFADA197E89FE8
:10C8C0008001E99F100DF89F100D11240F5B164F8A
:10C8D000D80150966D917D918D919C9153970E94B6
:10C8E000E9CEF80126A537A540A951A90E9450CE4E
:10C8F0001B012C01F80180819181A281B3810097F5
:10C90000A105B10549F584819581A681B78100977C
:10C91000A105B10509F580859185A285B3850097AC
:10C92000A105B105C9F4C201B10120910D093091F1
:10C930000E0940910F09509110090E941ED10E94CA
:10C9400036CE0C5B1F4F0E94BDCED8016D937D93F8
:10C950008D939C93139771C1C201B1012091090974
:10C9600030910A0940910B0950910C090E941ED187
:10C970000E9436CE0E94BDCE2DE430E0A196EEADF1
:10C98000FFADA197E29F6001E39FD00CF29FD00C16
:10C99000112421E439E0C20ED31EB4E46B2E712CB5
:10C9A0006C0C7D1CD3016D937D938D939C93139799
:10C9B0008090210990902209A0902309B090240929
:10C9C0000E94E9CE7B018C01F60160817181828138
:10C9D00093810E94EBCE9B01AC01C801B7010E947C
:10C9E0001ED17B018C01D60150966D917D918D9168
:10C9F0009C9153970E94E9CE9B01AC01C801B701FD
:10CA00000E9450CE7B018C01C501B4010E94E9CE89
:10CA10009B01AC01C801B7010E944CD018162CF440
:10CA2000F30180829182A282B38280902509909046
:10CA30002609A0902709B09028098DE490E0A196DE
:10CA40002EAD3FADA197289F6001299FD00C389F44
:10CA5000D00C112441E459E0C40ED51EA4E46A2E82
:10CA6000712C6C0C7D1CD3016D917D918D919C91ED
:10CA70000E94E9CE7B018C01F6016481758186817B
:10CA800097810E94EBCE9B01AC01C801B7010E94C7
:10CA90001ED17B018C01D60150966D917D918D91B7
:10CAA0009C9153970E94E9CE9B01AC01C801B7014C
:10CAB0000E9450CE7B018C01C501B4010E94E9CED9
:10CAC0009B01AC01C801B7010E944CD018162CF490
:10CAD000F30180829182A282B38280902D0990908E
:10CAE0002E09A0902F09B09030098DE490E0A19616
:10CAF0002EAD3FADA197289F6001299FD00C389F94
:10CB0000D00C112441E459E0C40ED51EF4E46F2E7C
:10CB1000712C6C0C7D1CD3016D917D918D919C913C
:10CB20000E94E9CE7B018C01F601648575858685BE
:10CB300097850E94EBCE9B01AC01C801B7010E9412
:10CB40001ED17B018C01D60150966D917D918D9106
:10CB50009C9153970E94E9CE9B01AC01C801B7019B
:10CB60000E9450CE7B018C01C501B4010E94E9CE28
:10CB70009B01AC01C801B7010E944CD018162CF4DF
:10CB8000F30180829182A282B382809029099090E1
:10CB90002A09A0902B09B0902C098DE490E0A19671
:10CBA0002EAD3FADA197289F6001299FD00C389FE3
:10CBB000D00C112441E459E0C40ED51EE4E46E2EDD
:10CBC000712C6C0C7D1CD3016D917D918D919C918C
:10CBD0000E94E9CE7B018C01F6016085718582851A
:10CBE00093850E94EBCE9B01AC01C801B7010E9466
:10CBF0001ED17B018C01D60150966D917D918D9156
:10CC00009C9153970E94E9CE9B01AC01C801B701EA
:10CC10000E9450CE7B018C01C501B4010E94E9CE77
:10CC20009B01AC01C801B7010E944CD018162CF42E
:10CC3000F30180829182A282B3828DE490E0A1967A
:10CC40002EAD3FADA197289F6001299FD00C389F42
:10CC5000D00C112441E459E0C40ED51EF601EC5B62
:10CC6000FF4F60817181828193810E94E9CE7B01B7
:10CC70008C01A20191010E9450CED601D2966D93F3
:10CC80007D938D939C93D597C801B7012DEB37E326
:10CC900046E051E40E941ED10E94B8CEF601648F96
:10CCA000758F868F978F6090110970901209809010
:10CCB000130990901409C401B30120E030E040E072
:10CCC0005FE30E941ED15B016C01298D3A8D4B8D73
:10CCD0005C8D29AF3AAF4BAF5CAF409115095091D5
:10CCE000160960911709709118094DAB5EAB6FABD7
:10CCF00078AFCB01BA0120E030E040E05FE30E9472
:10CD00001ED17B018C0169AD7AAD8BAD9CAD9F7757
:10CD1000A80197010E944CD0181644F4C601B50131
:10CD2000A80197010E9449CE882314F48601750159
:10CD30006D8D7E8D8F8D98A169AB7AAB8BAB9CABE3
:10CD40008091190990911A09A0911B09B0911C09B1
:10CD50008DA79EA7AFA7B8ABBC01CD0120E030E006
:10CD600040E05FE30E941ED11B012C0169A97AA952
:10CD70008BA99CA99F77A20191010E944CD0181603
:10CD800044F4C801B701A20191010E9449CE882351
:10CD900014F4170128018DE490E0A196AEADBFAD6B
:10CDA000A197A89FF001A99FF00DB89FF00D112445
:10CDB000EF5BF64F22A133A144A155A129A33AA3C9
:10CDC0004BA35CA3C201B1010E9449CE87FD04C000
:10CDD00029A03AA04BA05CA049A55AA54230510514
:10CDE0000CF405C15091130ECF56DF4F5883C15933
:10CDF000D0406091140ECE56DF4F6883C259D040A8
:10CE00007091150ECD56DF4F7883C359D040809175
:10CE1000160ECC56DF4F8883C459D040652FCE56AE
:10CE2000DF4F7881C259D040CD56DF4F8881C3593A
:10CE3000D040CC56DF4F9881C459D04027E137EB22
:10CE400041ED58E30E944CD018160CF0D0C069890F
:10CE50007A898B899C892091170E3091180E409108
:10CE6000190E50911A0E0E946FCD9B01AC010E94C9
:10CE70001ED17B018C016D897E898F89988D2091CF
:10CE80001B0E30911C0E40911D0E50911E0E0E94E3
:10CE90006FCD9B01AC010E941ED19B01AC01C8016A
:10CEA000B7010E9470CD0E948BD17B018C01A4013F
:10CEB00093010E944CD018165CF00F2EF0E06F2EFC
:10CEC000F0E07F2EF0E88F2EFFE39F2EF02D08C0BC
:10CED000C401B301A80197010E9450CE3B014C014F
:10CEE00069AD7AAD8BAD9CAD20911F0E3091200EB7
:10CEF0004091210E5091220E0E946FCD7B018C013A
:10CF0000E89417F9C801B7012DA93EA94FA958AD5A
:10CF10000E944CD0181694F46DA97EA98FA998ADE3
:10CF2000A80197010E9450CE5B016C01C401B301BE
:10CF3000A60195010E9449CE882314F4640153018F
:10CF400069A97AA98BA99CA92091230E3091240E5E
:10CF50004091250E5091260E0E946FCD7B018C01D1
:10CF6000E89417F9C801B7012DA53EA54FA558A90A
:10CF70000E944CD0181694F46DA57EA58FA598A993
:10CF8000A80197010E9450CE7B018C01C601B5011A
:10CF9000A80197010E9449CE882314F486017501E7
:10CFA00069A17AA18BA19CA1A80197010E941ED121
:10CFB0007B018C01CF56DF4F6881C159D040CE56DE
:10CFC000DF4F7881C259D040CD56DF4F8881C35999
:10CFD000D040CC56DF4F9881C459D040A80197016A
:10CFE0000E9449CE87FD19C0D801C70102C0D201F5
:10CFF000C101CF56DF4F8883C159D040CE56DF4F95
:10D000009883C259D040CD56DF4FA883C359D04032
:10D01000CC56DF4FB883C459D0408DE490E0A19640
:10D02000AEADBFADA197A89F8001A99F100DB89F7D
:10D03000100D11240F5B164FCF56DF4F8881C15959
:10D04000D040CE56DF4F9881C259D040CD56DF4FE9
:10D05000A881C359D040CC56DF4FB881C459D040C5
:10D06000F80182A793A7A4A7B5A762A973A984A969
:10D0700095A9905820E030E040E050EC0E941ED18D
:10D08000D8019E962D913D914D915C91D1970E9432
:10D090001ED12BE037ED43E25BE30E9470CD0E948E
:10D0A0008BD1F62EE72ED82EC92ECF56DF4F6881B2
:10D0B000C159D040CE56DF4F7881C259D040CD56AD
:10D0C000DF4F8881C359D040CC56DF4F9881C45977
:10D0D000D0402F2D3E2D4D2D5C2D0E9449CE87FD39
:10D0E00014C0CF56DF4FF882C159D040CE56DF4F23
:10D0F000E882C259D040CD56DF4FD882C359D040C4
:10D10000CC56DF4FC882C459D0408DE490E0A19640
:10D11000EEADFFADA197E89F8001E99F100DF89F4C
:10D12000100D11240F5B164FCF56DF4F8881C15968
:10D13000D040CE56DF4F9881C259D040CD56DF4FF8
:10D14000A881C359D040CC56DF4FB881C459D040D4
:10D15000F80186A397A3A0A7B1A762A173A184A198
:10D1600095A12F2D3E2D4D2D5C2D0E9449CE1816D8
:10D170002CF081E0D801D7968C9302C0F80117AA51
:10D180008DE490E0A1962EAD3FADA197289FF001D0
:10D19000299FF00D389FF00D1124EF5BF64F81E0D1
:10D1A00086ABA7E1BEE0FE01719680E101900D9291
:10D1B0008150E1F78DE490E0A1964EAD5FADA1976F
:10D1C000489F6001499FD00C589FD00C112461E406
:10D1D00079E0C60ED71ED6019296ED90FD900D9186
:10D1E0001C919597E092130EF092140E0093150E79
:10D1F0001093160E96966D917D918D919C919997B5
:10D20000A80197010E9450CE4B015C01C201B101FF
:10D21000A80197010E9450CE8B019C01C601B50167
:10D22000A4010E94965ABBA5B093110EC557DF4FBB
:10D23000288139814A815B81CB58D04020933D09B8
:10D2400030933E0940933F0950934009C957DF4F3F
:10D25000488159816A817B81C758D0404093390900
:10D2600050933A0960933B0970933C09CD57DF4FC7
:10D27000688179818A819B81C358D0406093350948
:10D28000709336098093370990933809C158DF4F5E
:10D2900088819981AA81BB81CF57D0408093310981
:10D2A00090933209A0933309B09334090E941E5D14
:10D2B0000E94A17AC856DF4F0FB6F894DEBF0FBEAA
:10D2C000CDBFCF91DF911F910F91FF90EF90DF9035
:10D2D000CF90BF90AF909F908F907F906F905F9016
:10D2E0004F903F902F900895FF920F931F93CF93ED
:10D2F000DF938B010E94171AEB01FF24FA9409C0F7
:10D300000E94171A6C1B7D0B6017710710F080E0EC
:10D3100008C0FEBC0DB407FEFDCF8EB58F3F81F770
:10D3200081E0DF91CF911F910F91FF900895FC0153
:10D330004281242F30E0C9019595879580658CBD89
:10D3400040FF02C080E004C080E0463009F081E088
:10D350008DBD808160E00C94181CDF92EF92FF92EB
:10D360000F931F93CF93DF93EC01D62E79018A019F
:10D37000DEDFCE016CE271E0B7DF8D2D80648EBD03
:10D380000DB407FEFDCF28E130E0D801C701022E21
:10D3900004C0B695A795979587950A94D2F78EBD48
:10D3A0000DB407FEFDCF285030408FEF283F3807DF
:10D3B00061F7DD2011F485E906C088E0D81611F484
:10D3C00087E801C08FEF8EBD0DB407FEFDCF8CE066
:10D3D000D81631F48FEF8EBD0DB407FEFDCF8EB59C
:10D3E0009FEF2FEF2EBD0DB407FEFDCF8EB587FF4B
:10D3F00004C0992311F09150F5CF8B83DF91CF9129
:10D400001F910F91FF90EF90DF900895FC018081B4
:10D4100061E00C94181CDC016EBDFA0120E030E0E4
:10D420000DB407FEFDCF80818EBD0DB407FEFDCF8C
:10D4300081818EBD2E5F3F4F329682E020303807CB
:10D4400079F70DB407FEFDCF8FEF8EBD0DB407FE4B
:10D45000FDCF8FEF8EBD0DB407FEFDCF8FEF8EBDDC
:10D460000DB407FEFDCF8EB513968C9313978F7175
:10D47000853011F481E0089583E111968C93119722
:10D48000CD01C4DF80E00895CF92DF92EF92FF924A
:10D490000F931F93CF93DF93EC017A018B01690106
:10D4A0008C81833039F059E0EE0CFF1C001F111FF6
:10D4B0005A95D1F7CE0168E1A80197014EDF882384
:10D4C00011F086E020C0CE016EEFA601A4DF882314
:10D4D000D9F0CE0168E572E007DF882311F487E117
:10D4E00012C0CE016DE020E030E040E050E035DFDA
:10D4F000882341F48FEF8EBD0DB407FEFDCF8EB5AE
:10D50000882371F086E18983CE0180DF80E0DF919E
:10D51000CF911F910F91FF90EF90DF90CF900895E2
:10D52000CE0174DF81E0F3CFBF92CF92DF92EF9212
:10D53000FF920F931F93CF93DF93EC016B018A014E
:10D540000E94171A7B01BB24BA9409C00E94171AC3
:10D550006E197F096D52714010F081E15FC0BEBC51
:10D560000DB407FEFDCF8EB58B838F3F79F38E3FD1
:10D5700011F08FE053C0D801119701151105D9F0B2
:10D580008FEF8EBD20E030E09FEF0BC00DB407FEA3
:10D59000FDCF8EB5F601E20FF31F80839EBD2F5F96
:10D5A0003F4F2A173B0790F30DB407FEFDCF8EB512
:10D5B000AC0DBD1D8C9340E050E060E070E016C003
:10D5C000272F3327F601E40FF51F808190E02827ED
:10D5D0003927220F331F2D53354FF901859194912F
:10D5E000762F6627682779274F5F5F4F40175107CF
:10D5F00038F38FEF8EBD0DB407FEFDCF3EB58FEF34
:10D600008EBD0DB407FEFDCF2EB5932F80E030E028
:10D61000822B932B6817790731F080E28983CE0142
:10D62000F5DE80E003C0CE01F1DE81E0DF91CF9135
:10D630001F910F91FF90EF90DF90CF90BF900895D2
:10D64000AF92BF92DF92EF92FF920F931F93CF930F
:10D65000DF93EC017A018B0159018C81833039F021
:10D6600099E0EE0CFF1C001F111F9A95D1F783E083
:10D67000D82EDA94CE0161E1A80197016EDE8823ED
:10D6800029F0DD2071F484E0898316C0CE01B50154
:10D6900040E052E049DF882311F081E010C0DD2036
:10D6A00059F0CE01B3DECE016CE020E030E040E086
:10D6B00050E053DE1982DDCFCE01A8DE80E0DF919D
:10D6C000CF911F910F91FF90EF90DF90BF90AF909F
:10D6D0000895BF92CF92DF92EF92FF920F931F9324
:10D6E000CF93DF93EC01B62E1C82198248830E94EF
:10D6F000171A6B01888161E00E94651BCE0186DEEE
:10D7000082E360E00E94651B83E361E00E94651B89
:10D7100084E361E00E94651B85E361E00E94651B74
:10D7200085E361E00E94181C85E08A8382E58CBD58
:10D730001DBC80E09FEF9EBD0DB407FEFDCF8F5F47
:10D740008A30C9F709C00E94171A6C197D09615DFA
:10D75000774010F081E059C0CE0160E020E030E079
:10D7600040E050E0FADD182F8B83813061F7CE0165
:10D7700068E02AEA31E040E050E0EFDD82FF02C0DD
:10D780001C8311C080E02FEF2EBD0DB407FEFDCF2E
:10D790009EB58F5F8430C1F79B839A3A11F082E087
:10D7A00034C082E08C838C81823021F0EE24FF240F
:10D7B00087010FC0E12CF12C012D40E4142F09C08A
:10D7C0000E94171A6C197D09615D774010F08AE09C
:10D7D0001CC0CE0167E320E030E040E050E0BDDD5A
:10D7E000CE0169E2A8019701B8DD8B83882341F758
:10D7F0008C81823019F5CE016AE320E030E040E010
:10D8000050E0ABDD882329F088E08983CE01FEDD7E
:10D8100020C08FEF8EBD0DB407FEFDCF8EB5807C8E
:10D82000803C11F483E08C8380E09FEF9EBD0DB4BB
:10D8300007FEFDCF2EB58F5F8330C1F7CE01E6DD49
:10D8400086E08B1518F488E1898303C0BA8281E0F1
:10D8500001C080E0DF91CF911F910F91FF90EF9079
:10D86000DF90CF90BF900895CF93DF93DC01EB0161
:10D87000BA0180E090E020E2FE01E80FF91F20836A
:10D8800001968B309105C1F757E040E022C02E325F
:10D8900019F083EC9CE007C05A3049F15AE048E0A7
:10D8A00017C0321721F1FC01019634913323C9F7D7
:10D8B0005417E8F02132D8F02F37C8F4822F815660
:10D8C0008A3108F42052FE01E40FF11D20834F5FDE
:10D8D00011962C91222311F02F32C9F6FB01B1834E
:10D8E000A08390E08881803219F091E001C090E03F
:10D8F000892FDF91CF9108956F927F928F929F929F
:10D90000AF92BF92CF92DF92EF92FF920F931F934D
:10D91000CF93DF93EC017A018B012B81222309F451
:10D9200080C089899A89AB89BC8984179507A60725
:10D93000B70708F476C085C0E114F10401051105AC
:10D9400051F41C821D821E821F82188619861A8637
:10D950001B8681E067C0288539854A855B85E98D0E
:10D96000FA8D858590E00996215030404040504026
:10D9700039014A01082E04C09694879477946794DD
:10D980000A94D2F72F5F3F4F4F4F5F4F0894E10843
:10D99000F108010911095701680104C0D694C79420
:10D9A000B794A7948A95D2F70894E11CF11C011D45
:10D9B000111DA614B704C804D90428F02115310597
:10D9C0004105510549F48D899E89AF89B88D8C83B5
:10D9D0009D83AE83BF8316C0A618B708C808D908B0
:10D9E00011C04C815D816E817F81898D9A8D9401FA
:10D9F0000E9450780894A108B108C108D108882372
:10DA000031F40FC084E0882E912C8C0E9D1EA11441
:10DA1000B104C104D10429F7E886F9860A871B8777
:10DA200098CF80E0DF91CF911F910F91FF90EF9001
:10DA3000DF90CF90BF90AF909F908F907F906F902E
:10DA40000895223009F078CFE7CFCF93DF93EC0130
:10DA50008C859D85AE85BF8540E0611141E0BC01AC
:10DA6000CD010E941E76882319F420E030E00AC020
:10DA70008889282F30E095E0220F331F9A95E1F72F
:10DA8000235D314FC901DF91CF9108950F931F930B
:10DA9000CF93DF938C01FC0183818823E9F181819D
:10DAA00087FF37C0C80161E0D0DFEC010097A1F12A
:10DAB0008881853E89F1F8018381823040F4818933
:10DAC0009289A389B4898C8F9D8FAE8FBF8FF80107
:10DAD000858996899B8F8A8F85899689A789B08D3C
:10DAE000CD01AA27BB279D8B8C8BE091270EF0914F
:10DAF000280E309751F0BE016A5E7F4FCE014896E6
:10DB00001995888D998D9B8B8A8BF80181818F77F0
:10DB100081830E94E37504C081E0F801808380E086
:10DB2000DF91CF911F910F9108950F931F938C0157
:10DB3000ADDFF80113821F910F910895FC018381DD
:10DB4000882311F0CF01F1CF08956F927F928F92C9
:10DB50009F92AF92BF92CF92DF92EF92FF920F937C
:10DB60001F93DF93CF9300D00F92CDB7DEB77C0128
:10DB70005A016B01DC0113968C911397813009F0E7
:10DB80008EC011968C9181FF8AC09DC00097A1051F
:10DB9000B10511F481E084C0F7016084718482844E
:10DBA0009384C701B601A501A7DE882309F477C0D5
:10DBB000D70159968D919C915A97A114B104C10433
:10DBC000D10489F455964D915D916D917C91589752
:10DBD0000E94C578882309F462C0F701158A168A65
:10DBE000178A108E44C0D70114964D915D916D91A6
:10DBF0007C9117979E012F5F3F4F0E94507888239A
:10DC000009F44DC0D7015996ED91FC915A9749817D
:10DC10005A816B817C818789803149F4483FBFEF0D
:10DC20005B07B0E06B07B0E07B0748F020C0483FDF
:10DC30008FEF58078FEF68078FE07807C0F4CF01A8
:10DC40000E94C578882359F1D70114964D915D91B2
:10DC50006D917C91179759968D919C915A970FEFE2
:10DC60001FEF2FEF3FE00E94CA778823C1F0F70132
:10DC7000A18AB28AC38AD48A818180688183C701DC
:10DC800005DF882361F0B601A5016A147B048C04CA
:10DC90009D0410F4B401A301C7012EDE01C080E091
:10DCA0000F900F900F900F90CF91DF911F910F91D8
:10DCB000FF90EF90DF90CF90BF90AF909F908F90AC
:10DCC0007F906F900895F70181899289A389B48923
:10DCD00084179507A607B70708F058CFE0CFCF9372
:10DCE000DF93EC0140E050E060E070E02EDF88233D
:10DCF00059F0CE0161E0A9DEFC01009729F085EE24
:10DD000080831B8260D701C080E0DF91CF910895AE
:10DD10002F923F924F925F926F927F928F929F923B
:10DD2000AF92BF92CF92DF92EF92FF920F931F9329
:10DD3000CF93DF93EC012A018B81882309F4B5C0CE
:10DD4000898180FFB2C0C7C025014E185F083B0122
:10DD500074E0272E312C2C0E3D1E4201A0C02885D8
:10DD600039854A855B856FEFA62E61E0B62EA2222B
:10DD7000B3228B8179018A0199E016950795F79472
:10DD8000E7949A95D1F7E98DFA8D823049F4428D66
:10DD9000538D648D758D4E0D5F1D601F711F3FC0CB
:10DDA000D480DA94DE20A114B104D9F4DD20C9F4C2
:10DDB000211531054105510549F48D899E89AF89A9
:10DDC000B88D8C839D83AE83BF830BC04C815D81F6
:10DDD0006E817F81CF0191010E945078882309F4E0
:10DDE00064C0E98DFA8D4C815D816E817F814250E6
:10DDF000504060407040058404C0440F551F661FAA
:10DE0000771F0A94D2F786859785A089B189480F34
:10DE1000591F6A1F7B1F4D0D511D611D711D80E033
:10DE200092E08A199B0984018815990508F48C01F0
:10DE300082E00030180709F066C08091290E9091A9
:10DE40002A0EA0912B0EB0912C0E481759076A0785
:10DE50007B0709F458C080912D1090912E109301EA
:10DE6000EFDB882349F421C09501235D314FC301C5
:10DE7000B901A8010E94CBCC600E711E980140E050
:10DE800050E088859985AA85BB85820F931FA41FC2
:10DE9000B51F88879987AA87BB87801A910A811442
:10DEA000910409F05CCFA20102C04FEF5FEFCA01FD
:10DEB000DF91CF911F910F91FF90EF90DF90CF9066
:10DEC000BF90AF909F908F907F906F905F904F909A
:10DED0003F902F900895A988BA88CB88DC88E88481
:10DEE000F9840A851B859A0140E050E0D601C501FE
:10DEF0008E199F09A00BB10B281739074A075B073A
:10DF000008F022CF24CFCB01BA0140E097D6882376
:10DF100009F0AACFCACFCF92DF92EF92FF920F9370
:10DF20001F93CF93DF937C01EB018A01FC01838176
:10DF3000823008F46EC080859185A285B3858F718B
:10DF40009070A070B0700097A105B10509F061C094
:10DF50006CC0F8011082EDE0CE2ED12CC701BE01BD
:10DF600040E250E0D5DE9C018032910521F000971F
:10DF700009F04FC050C04881442309F44CC0453ECD
:10DF800069F34E3259F38B858F738F30E9F50115A4
:10DF90001105D1F18A8D9B8D892BB1F5842F90E0ED
:10DFA0008F719070009781F1833091056CF58C9D95
:10DFB00090018D9D300D9C9D300D11242D503040D1
:10DFC000F801E20FF31F898180838B8181838D812A
:10DFD00082838F818383898584838E8585838889E5
:10DFE00086838A8987838C8980878E898187888DBB
:10DFF00082878C8D83878E8D8487888186FF04C07D
:10E00000F801E20FF31F15868B8583FDA7CF822FC2
:10E0100003C08FEF01C080E0DF91CF911F910F917E
:10E02000FF90EF90DF90CF9008954115510509F0D2
:10E0300090CF91CFDF93CF930F92CDB7DEB7BE01D4
:10E040006F5F7F4F41E050E063DE019719F02FEFE3
:10E050003FEF03C08981282F30E0C9010F90CF9195
:10E06000DF910895EF92FF920F931F93CF93DF9369
:10E07000EC018B81823030F1E884F9840A851B85BC
:10E08000CE01D8DF97FD1EC088859985AA85BB85FE
:10E090004F96A11DB11D88879987AA87BB87A5E0E8
:10E0A00016950795F794E794AA95D1F72E2D30E0B1
:10E0B0002F703070F5E0220F331FFA95E1F7235DE2
:10E0C000314F02C020E030E0C901DF91CF911F91B4
:10E0D0000F91FF90EF9008950F931F93CF93DF93CD
:10E0E000EC018B018B81882309F040C0FB018789FB
:10E0F000803109F041C082E08B831D8A1E8A1F8A0D
:10E10000188E808D918DA0E0B0E045E0880F991FBA
:10E11000AA1FBB1F4A95D1F7898B9A8BAB8BBC8BFF
:10E1200013C083E08B83F801428D538D648D758D10
:10E130004D8B5E8B6F8B788F9E012F5E3F4FC8019A
:10E140000E942179882391F01A8F098F81E08983B9
:10E150001C821D821E821F82188619861A861B86C3
:10E160001C861D861E861F86188A01C080E0DF91EE
:10E17000CF911F910F9108958032C1F7D2CF1F9395
:10E18000CF93DF93EC01142F262F30E0F90175E0D7
:10E19000EE0FFF1F7A95E1F7E35DF14F8385817103
:10E1A00021F0842F827109F067C08091290E90912F
:10E1B0002A0EA0912B0EB0912C0E8C879D87AE87D6
:10E1C000BF87688BF90165E0EE0FFF1F6A95E1F7E5
:10E1D000E35DF14F84899589A0E0B0E0DC019927E7
:10E1E00088278D8B9E8BAF8BB88F228D338DA901A5
:10E1F00060E070E0482B592B6A2B7B2B4D8B5E8B9C
:10E200006F8B788F838590E088719070009751F4C0
:10E21000848D958DA68DB78D898B9A8BAB8BBC8B9E
:10E2200081E00CC0409741F59E012F5E3F4F898DE4
:10E230009A8D0E9421798823F9F084E08B83812FC5
:10E240008F7089831C821D821E821F821886198608
:10E250001A861B8614FF16C0CE0140E050E060E035
:10E2600070E073DC882371F409C049895A896B898D
:10E270007C89CE0141DB02C01B8280E0DF91CF911F
:10E280001F91089515FDF1CF81E0F8CF2F923F92B5
:10E290004F925F926F927F928F929F92AF92BF92B6
:10E2A000CF92DF92EF92FF920F931F93DF93CF9362
:10E2B0000F92CDB7DEB72C015B013A01490100E0B6
:10E2C00010E0EE24EA94FE2C1E010894211C311C5F
:10E2D00011C00A0D1B1DF80160838114910419F40B
:10E2E0006A3039F41BC0C40170E00E94DFCC009793
:10E2F000A9F4860168010894C11CD11CC614D70476
:10E300003CF5C201B10141E050E002DD7C01813009
:10E310009105F1F469816D30E1F6ECCF8601A00E34
:10E32000B11EF5011082C8010F90CF91DF911F91AE
:10E330000F91FF90EF90DF90CF90BF90AF909F90A4
:10E340008F907F906F905F904F903F902F900895A7
:10E35000F7FEE5CF0FEF1FEFE6CFCF93DF93EC0192
:10E360009C012C5F3F4F898D9A8D41E050E060E029
:10E3700070E0D2D78823A1F08D899E89AF89B88DAE
:10E380000097A105B10559F48C819D81AE81BF81B3
:10E390008D8B9E8BAF8BB88F89818068898381E05C
:10E3A000DF91CF9108952F923F924F925F927F928B
:10E3B0008F929F92AF92BF92CF92DF92EF92FF9295
:10E3C0000F931F93DF93CF9300D000D0CDB7DEB76C
:10E3D0006C01162F072F5E834D83DC0113968C9101
:10E3E0001397813009F069C111968C9181FF65C145
:10E3F00082C1F6014189528963897489808591853A
:10E40000A285B38584179507A607B70729F0C6012B
:10E4100073DA882309F451C1812F902F9C011901CF
:10E420004D805E800FC1D6015996ED91FC915A97AF
:10E43000DA01C90149E0B695A795979587954A9560
:10E44000D1F774807A9478228FEF882E81E0982E0D
:10E4500082229322772009F051C08114910409F09F
:10E460004DC0D60114964D915D916D917C91179799
:10E47000411551056105710581F455968D919D9168
:10E480000D90BC91A02D0097A105B10559F1F601A1
:10E4900084839583A683B78331C0CF019E012F5F0C
:10E4A0003F4FFED5882309F408C129813A814B8169
:10E4B0005C81D6015996ED91FC915A9787898031FC
:10E4C00049F4283FBFEF3B07B0E04B07B0E05B07E4
:10E4D00070F008C0283FEFEF3E07EFEF4E07EFE088
:10E4E0005E0728F0C60139DF882341F4E6C0D60173
:10E4F00014962D933D934D935C93179780E092E093
:10E500008819990952018415950508F45C01D60112
:10E510005996ED91FC915A971496ED90FD900D91BE
:10E520001C9117978EEF9FEFAFEFBFEFE80EF91E2C
:10E530000A1F1B1F058404C0EE0CFF1C001F111FC7
:10E540000A94D2F786859785A089B189E80EF91ECD
:10E550000A1F1B1FE70CF11C011D111D90E0A916DD
:10E5600092E0B90639F58091290E90912A0EA0917A
:10E570002B0EB0912C0E8E159F05A007B10771F4DC
:10E5800010922F108FEF9FEFAFEFBFEF8093290E08
:10E5900090932A0EA0932B0EB0932C0E80912D10E9
:10E5A00090912E10B801A70191010E94446A88231E
:10E5B000A9F583C08114910411F5D60118962D9107
:10E5C0003D914D915C911B9751968D919D910D9030
:10E5D000BC91A02D281739074A075B0780F0F3D2BA
:10E5E000882309F46AC081E080932F10E092290EFD
:10E5F000F0922A0E00932B0E10932C0E07C0C80128
:10E60000B70141E01BD3882309F457C09401235D6F
:10E61000314FC901B101A5010E94CBCC950140E069
:10E6200050E0F60180859185A285B385820F931F06
:10E63000A41FB51F80879187A287B3872A0C3B1C34
:10E640004A185B08D60118962D913D914D915C9129
:10E650001B974114510409F0E6CE51968D919D917E
:10E660000D90BC91A02D82179307A407B50748F41D
:10E67000F601218B328B438B548B8181806881839F
:10E6800011C08091270E9091280E892B59F08D8111
:10E690009E81892B39F0D60111968C911197806853
:10E6A00011968C93F601818183FF04C0C601EED9D7
:10E6B000882319F04D815E8105C081E0D6018C93DD
:10E6C0004FEF5FEFCA0126960FB6F894DEBF0FBE7C
:10E6D000CDBFCF91DF911F910F91FF90EF90DF9011
:10E6E000CF90BF90AF909F908F907F905F904F9012
:10E6F0003F902F90089582FD7CCE8ECEDF92EF92D8
:10E70000FF920F931F93CF93DF93EC0189899A892E
:10E71000AB89BC89805E9F4FAF41B04008F06FC0AD
:10E72000CE011BDE882309F46AC04DD2882309F488
:10E7300066C0E98DFA8DEC80FD800E811F818EEF21
:10E740009FEFAFEFBFEFE80EF91E0A1F1B1F0584F6
:10E7500004C0EE0CFF1C001F111F0A94D2F786851F
:10E760009785A089B189E80EF91E0A1F1B1F81E059
:10E7700080932F10E092290EF0922A0E00932B0E18
:10E7800010932C0E80E092E0EDE2FEE0DF019C01B0
:10E790001D9221503040E1F7DD24D39411C0B8011F
:10E7A000A7014D0D511D611D711D80912D1090917E
:10E7B0002E102DE23EE00E94446A882301F1D3949A
:10E7C000E98DFA8D8481D81650F320E032E040E0E4
:10E7D00050E0058404C0220F331F441F551F0A94C4
:10E7E000D2F789899A89AB89BC89820F931FA41FAC
:10E7F000B51F898B9A8BAB8BBC8B81E001C080E00D
:10E80000DF91CF911F910F91FF90EF90DF900895CE
:10E810008F929F92AF92BF92CF92DF92EF92FF9230
:10E820000F931F93CF93DF936C01EB01942E852EF2
:10E83000A22E898D9A8DD6015A969C938E935997C4
:10E84000CB0140E050E060E070E056D8BB2437C018
:10E85000CE0108DCFC01009709F48FC055E0169545
:10E860000795F794E7945A95D1F71E2D1F70808174
:10E87000882311F0853EC9F4BB2099F42091290E1C
:10E8800030912A0E40912B0E50912C0ED6011C96E1
:10E890002D933D934D935C931F9750961C93BB24EF
:10E8A000B3948081882359F418C0892D982DBF0115
:10E8B0004BE050E00E94BECC009709F46CC0E884A5
:10E8C000F9840A851B8589899A89AB89BC89E816F0
:10E8D000F9060A071B0708F4BBCFA6FE4EC0A1FE2F
:10E8E0004CC0BB2049F0F6011089C60161E0ADD8EB
:10E8F000EC01009761F441C08B81823009F43DC086
:10E90000CE01FCDE8823C9F110E0CDE2DEE080E23A
:10E91000DE011D928A95E9F7DE01292D382DC90106
:10E92000FC018BE001900D928150E1F7E091270E00
:10E93000F091280E309739F0BE01625F7F4FCE0113
:10E940004096199508C081E298E2998B888B80E007
:10E9500098E09F878E87888999899B8B8A8B998F6E
:10E96000888F8E859F859F8B8E8B2DD1882329F054
:10E97000C601612F4A2D03DC01C080E0DF91CF91F9
:10E980001F910F91FF90EF90DF90CF90BF90AF90CD
:10E990009F908F900895A7FEEBCFEFCF2F923F92DD
:10E9A0004F925F926F927F928F929F92AF92BF929F
:10E9B000CF92DF92EF92FF920F931F93DF93CF934B
:10E9C000CDB7DEB7C654D0400FB6F894DEBF0FBE49
:10E9D000CDBF3C016B01DE01AE5BBF4F11965C9376
:10E9E0004E9325962FAF25971C861F861FA21AA629
:10E9F0006115710509F47CC0FC018381882309F04D
:10EA000077C0FA0180818F32F1F08601ECE0EE2EC2
:10EA1000F12CEC0EFD1E72E4A72EB12CAC0EBD1E27
:10EA20004E010894811C911C2796FFAEEEAE2797ED
:10EA300067E2262E312C2C0E3D1E270123C0119695
:10EA4000B183A08301C0FD01A081B1818C918F327F
:10EA5000B1F3D60113968C91139782508230A8F2AD
:10EA60008E01095D1F4F59966D917C915A97C8018F
:10EA700033DB882359F63CC0342D252D8701832FA5
:10EA8000922F7C01F50180819181B401A5010E9442
:10EA9000346C882329F42CC03196D501ED93FC9376
:10EAA000D501ED91FC9180818F32B1F38823B9F0CB
:10EAB000C701B801A40121E0ABDE8823C9F00C1521
:10EAC0001D0511F0C80131D82796EEADFFAD27978F
:10EAD000EE16FF0689F6C101322D292FCFCFC301D3
:10EAE000B801A40125962FAD259792DE182F01C0FD
:10EAF00010E0CE01879622D8CE010C961FD8812F28
:10EB0000CA5BDF4F0FB6F894DEBF0FBECDBFCF910B
:10EB1000DF911F910F91FF90EF90DF90CF90BF900A
:10EB2000AF909F908F907F906F905F904F903F90AD
:10EB30002F9008950F931F93DF93CF93CDB7DEB738
:10EB40006B970FB6F894DEBF0FBECDBF9C01AB0133
:10EB500019821C828E010F5F1F4FC801B90122E08C
:10EB60001DDF882311F410E003C0C801B8D8182FA6
:10EB7000CE0101960E949E6D812F6B960FB6F89480
:10EB8000DEBF0FBECDBFCF91DF911F910F910895D2
:10EB9000DB010D900020E9F71197A61BB70B049637
:10EBA000AD0101CCDF93CF930F92CDB7DEB7698370
:10EBB0000496BE016F5F7F4F41E050E0F4DB0F90A1
:10EBC000CF91DF91089580912F10882399F1409182
:10EBD000290E50912A0E60912B0E70912C0E80916F
:10EBE0002D1090912E102DE23EE00E94446A882361
:10EBF00019F14091301050913110609132107091A4
:10EC00003310411551056105710591F080912D106A
:10EC100090912E102DE23EE00E94446A882361F01C
:10EC20001092301010923110109232101092331056
:10EC300010922F1081E0089580E00895DF92EF9206
:10EC4000FF920F931F937B018C01D42E8091290E8C
:10EC500090912A0EA0912B0EB0912C0E8E159F052F
:10EC6000A007B107B9F0AFDF8823E1F080912D1044
:10EC700090912E10B801A7012DE23EE00E94206B7A
:10EC8000882381F0E092290EF0922A0E00932B0E39
:10EC900010932C0EDD2011F481E011C081E08093EF
:10ECA0002F100DC08FEF9FEFAFEFBFEF8093290EB6
:10ECB00090932A0EA0932B0EB0932C0E80E01F9100
:10ECC0000F91FF90EF90DF9008958F929F92AF92F7
:10ECD000BF92CF92DF92EF92FF920F931F93CF9349
:10ECE000DF936C01142F70932E1060932D10FC0194
:10ECF000178A82E090E0A0E0B0E080839183A28355
:10ED0000B38310922F101092301010923110109285
:10ED10003210109233108FEF9FEFAFEFBFEF809361
:10ED2000290E90932A0EA0932B0EB0932C0E442301
:10ED300021F48824992454013FC0453008F01CC1B7
:10ED400060E070E080E090E040E078DF882309F444
:10ED500013C1C12FD0E02197FE0174E0EE0FFF1F19
:10ED60007A95E1F7E35DF14FE254FE4F8081EE5B6F
:10ED7000F14090E08F779070892B09F0FDC0E65349
:10ED8000FE4F80819181A281B38184369105A105D6
:10ED9000B10508F4F1C064E0CC0FDD1F6A95E1F71E
:10EDA000CD50D04F88809980AA80BB808114910477
:10EDB000A104B10409F4E0C0C501B40140E03EDFA4
:10EDC000882309F4D9C08091380E9091390E805073
:10EDD000924009F0D1C020913D0E222309F4CCC00D
:10EDE00080913B0E90913C0E892B09F4C5C0809117
:10EDF0003A0E882309F4C0C0F601228B80913A0EA6
:10EE00008483158661E070E007C04F5FF601458797
:10EE10004150483008F0B0C0F6014585848190E04B
:10EE20009B01042E02C0220F331F0A94E2F78217BF
:10EE3000930759F72091430E3091440E2115310567
:10EE400019F040E050E008C02091510E3091520E70
:10EE50004091530E5091540EF6012583368347831B
:10EE60005087E0903B0EF0903C0E00E010E0E80C84
:10EE7000F91C0A1D1B1DE38AF48A058B168B8091F1
:10EE80003E0E90913F0E918F808F60913D0E70E00D
:10EE900080E090E00E94C1D46E0D7F1D801F911F05
:10EEA000F601628F738F848F958F20913E0E309183
:10EEB0003F0E55E0220F331F5A95E1F721503E4F88
:10EEC000232F3327269540E050E0260F371F481F99
:10EED000591F26873787408B518B8091400E909128
:10EEE000410E009719F0A0E0B0E008C080914D0EEF
:10EEF00090914E0EA0914F0EB091500E850174016D
:10EF0000E21AF30A040B150BA8019701280F391F09
:10EF10004A1F5B1FF601058404C056954795379537
:10EF200027950A94D2F72187328743875487253F54
:10EF3000FFE03F07F0E04F07F0E05F0720F48CE0D0
:10EF4000F601878B19C0255F3F4F4040504018F4B1
:10EF500080E1F6010EC08091590E90915A0EA09159
:10EF60005B0EB0915C0EF601828F938FA48FB58FEC
:10EF700080E2878B81E001C080E0DF91CF911F911B
:10EF80000F91FF90EF90DF90CF90BF90AF909F9048
:10EF90008F9008956F927F928F929F92AF92BF92BF
:10EFA000CF92DF92EF92FF920F931F93CF93DF9355
:10EFB000EC015A016B0138014901423051056105EC
:10EFC000710508F45DC089859A85AB85BC8501967D
:10EFD000A11DB11D84179507A607B70708F450C0F7
:10EFE0008F89803129F4E52EF62E072F11270CC0CA
:10EFF000803209F045C07A018B0187E016950795AC
:10F00000F794E7948A95D1F78B899C89AD89BE895D
:10F01000E80EF91E0A1F1B1FC801B70141E00EDEF2
:10F02000882371F18F89803149F4F501F070EE0F7A
:10F03000FF1FE35DF14F718260820DC0F501EF7734
:10F04000F070EE0FFF1FEE0FFF1FE35DF14F6082C8
:10F050007182828293828A89823080F08D819E8142
:10F06000AF81B885E80EF91E0A1F1B1FE092301011
:10F07000F0923110009332101093331081E001C0F0
:10F0800080E0DF91CF911F910F91FF90EF90DF9083
:10F09000CF90BF90AF909F908F907F906F9008958A
:10F0A000CF92DF92EF92FF920F931F93CF93DF9354
:10F0B000EC017A018B01690189859A85AB85BC8554
:10F0C0000196A11DB11D84179507A607B70708F47F
:10F0D00052C08F89803129F45527412F302F2F2D91
:10F0E0000CC0803209F047C09A01AB0167E0569529
:10F0F0004795379527956A95D1F78B899C89AD8976
:10F10000BE89280F391F4A1F5B1F8091290E9091DD
:10F110002A0EA0912B0EB0912C0E281739074A0702
:10F120005B0731F0CA01B90140E088DD882319F19D
:10F130008F89803159F4F701F070EE0FFF1FE35D06
:10F14000F14F80819181A0E0B0E00EC0F701EF7730
:10F15000F070EE0FFF1FEE0FFF1FE35DF14F808198
:10F160009181A281B381BF70F60180839183A283D4
:10F17000B38381E001C080E0DF91CF911F910F91B7
:10F18000FF90EF90DF90CF900895AF92BF92CF9213
:10F19000DF92EF92FF920F931F93DF93CF9300D0F4
:10F1A0000F92CDB7DEB76C017A018B0182E090E05F
:10F1B000A0E0B0E0F60180839183A283B3835E0177
:10F1C0000894A11CB11CC601B801A701950168DF14
:10F1D000882339F1C601B801A70100E010E020E062
:10F1E00030E0D8DE8823E9F0E980FA800B811C81C9
:10F1F000F6018789803151F4F8EFEF16FFEFFF0633
:10F20000F0E00F07F0E01F07F0F209C088EFE81602
:10F210008FEFF8068FEF08078FE01807A0F281E064
:10F2200001C080E00F900F900F900F90CF91DF9171
:10F230001F910F91FF90EF90DF90CF90BF90AF9014
:10F2400008954F925F926F927F928F929F92AF92AA
:10F25000BF92CF92DF92EF92FF920F931F93DF93B3
:10F26000CF9300D00F92CDB7DEB76C0149835A839C
:10F270006B837C833901EE24FF2487012E010894DF
:10F28000411C511C812CE2E09E2EA12CB12C498105
:10F290005A816B817C81C601920102DF882339F19A
:10F2A000D501C401F601058404C0880F991FAA1F67
:10F2B000BB1F0A94D2F7E80EF91E0A1F1B1F2981F3
:10F2C0003A814B815C818789803131F4285F3F4FDF
:10F2D00040405040E0F205C0285F3F4F4F4F5F4035
:10F2E000B0F2F301E082F1820283138381E00F9098
:10F2F0000F900F900F90CF91DF911F910F91FF9082
:10F30000EF90DF90CF90BF90AF909F908F907F90C5
:10F310006F905F904F9008952F923F924F925F921F
:10F320006F927F928F929F92AF92BF92CF92DF9215
:10F33000EF92FF920F931F93DF93CF93CDB7DEB77A
:10F340002F970FB6F894DEBF0FBECDBF1C014A87C2
:10F350005B876C877D873F872E87DC0119968D91AF
:10F360009D910D90BC91A02D0196A11DB11D8E8384
:10F370009F83A887B987F901008111812281338198
:10F38000011511052105310549F04801590108947D
:10F39000811C911CA11CB11C1D8210C0D1018D903B
:10F3A0009D90AD90BC901D828A859B85AC85BD8566
:10F3B0000197A105B10511F491E09D8375016401E8
:10F3C0004424552432018E010F5F1F4FF1018185C6
:10F3D0009285A385B485481659066A067B0608F00F
:10F3E0008CC08E819F81A885B9858C159D05AE0541
:10F3F000BF0550F4A2E08A2E912CA12CB12CF2E092
:10F40000CF2ED12CE12CF12CC101B701A60198011E
:10F4100047DE882309F471C089819A81AB81BC8160
:10F42000A70196012F5F3F4F4F4F5F4F0097A105F8
:10F43000B10519F049015A010DC0281939094A09C5
:10F440005B098A859B85AC85BD85281739074A07E6
:10F450005B0759F00894411C511C611C711C0894F5
:10F46000C11CD11CE11CF11CB1CFC101A601B70127
:10F470000FEF1FEF2FEF3FE08DDD882391F43DC0AC
:10F480002601370108944108510861087108C1013B
:10F49000B301A201970186017DDD882371F173011B
:10F4A00062018C149D04AE04BF0450F3AE85BF8589
:10F4B0004D915D916D917C914115510561057105ED
:10F4C00031F0C1019501840165DD8823B1F0EE853D
:10F4D000FF8580829182A282B382FD81FF2359F051
:10F4E0000894811C911CA11CB11CD1018D929D928C
:10F4F000AD92BC92139781E001C080E02F960FB6C9
:10F50000F894DEBF0FBECDBFCF91DF911F910F9159
:10F51000FF90EF90DF90CF90BF90AF909F908F9033
:10F520007F906F905F904F903F902F900895109232
:10F53000681010926A1010926C10089580938C03DA
:10F540000895EFE6F0E080818260808308951F9344
:10F55000FC011FB7F89480819181A281B3818093CF
:10F56000421090934310A0934410B0934510FB01B8
:10F5700080819181A281B38180934610909347103E
:10F58000A0934810B0934910FA0180819181A28123
:10F59000B38180934A1090934B10A0934C10B0937A
:10F5A0004D10F90180819181A281B38180934E1029
:10F5B00090934F10A0935010B09351101FBF1F9104
:10F5C0000895FC012FB7F89480819181A281B381C5
:10F5D00080934E1090934F10A0935010B093511001
:10F5E0002FBF0895E82F8FB7F894F0E0EE0FFF1FBC
:10F5F000EE0FFF1FEE5BFF4E208131814281538170
:10F600008FBFB901CA01089580916F008D7F8093EB
:10F610006F0006C08091120E8F5F8F708093120E64
:10F620009091110E8091120E981751F4109235108E
:10F630001092341080916F00826080936F00089563
:10F640009091110E8091120E981751F3E3CF9B0108
:10F65000882399F4B901882777FD8095982F2FEF9B
:10F6600030E040E050E00E94C1D420ED37E040E0BF
:10F6700050E00E9435D58CE214C08130A9F4B90164
:10F68000882777FD8095982F2FEF30E040E050E0FD
:10F690000E94C1D420ED37E040E050E00E9435D513
:10F6A0008DE2B9010C94871A8230A9F4B901882738
:10F6B00077FD8095982F2FEF30E040E050E00E94DA
:10F6C000C1D420ED37E040E050E00E9435D58EE215
:10F6D000B9010C94871A08958CE261E00E94651BC1
:10F6E0008DE261E00E94651B8EE261E00E94651B75
:10F6F000609182037091830380E0A9DF60918403AD
:10F700007091850381E0A3DF609186037091870388
:10F7100082E09DDFE1E2F1E08081887F816080838B
:10F720000895DADF099A3C9A399AEAE0F1E080819B
:10F73000806480838081846080830D9A159A3E9ACC
:10F74000469A3B9A439A389A409A80818260808395
:10F750009FB7F894EBE0F1E08081826080839FBFE7
:10F760000898109A0C98149A0F98179A0B9A139855
:10F77000159A3D9A4598469A3A9A4298439AEAE0F1
:10F78000F1E08081806880839FB7F894EBE0F1E03E
:10F7900080818F7780839FBF409AEAE0F1E080818B
:10F7A000816080839FB7F894EBE0F1E080818E7FE9
:10F7B00080839FBFA1E8B0E08C918F7E8C938C9169
:10F7C00088608C93E0E8F0E080818D7F8083808189
:10F7D0008E7F808380818F73808380818F7C808304
:10F7E0008C91887F82608C9380E090E49093890074
:10F7F000809388001092850010928400EFE6F0E07C
:10F8000080818260808381E080938C037894089566
:10F810009091110E8091120E981739F00E94248851
:10F820000E9499300E947691F3CF0895F1DF159AE6
:10F83000469A439A409A08951F920F920FB60F92DC
:10F840000BB60F921124AF92BF92CF92DF92EF923C
:10F85000FF920F931F932F933F934F935F936F9359
:10F860007F938F939F93AF93BF93CF93DF93EF9348
:10F87000FF938091341090913510892B09F094C139
:10F880009091110E8091120E981719F4E0E0F0E0BB
:10F8900014C08091120E90E02DE430E0829FF001C0
:10F8A000839FF00D929FF00D1124EF5BF64FE45B08
:10F8B000FF4F81E08083EC54F040F0933510E093EB
:10F8C0003410309709F46AC1E45BFF4F81E0808314
:10F8D000EC54F04010927410109275101092761043
:10F8E0001092771060AD71AD2CE96134720718F099
:10F8F00060E47CE904C03EE46132730730F0769541
:10F9000067957695679584E007C047E26131740793
:10F9100030F07695679582E080936D1007C08093F4
:10F920006D106032710510F460E270E0605270405A
:10F9300058E060307507E8F0472F50E0440F551F3E
:10F94000440F551F4950534F9A012E5F3F4FF90105
:10F95000859194919C01AA27639FC001629F810DAC
:10F960009A1F06948A1F9A1F1124FA0145915491F7
:10F970001EC0CB01969587958C7F89509F4EFC01C8
:10F9800045915491FC01329625913491862F90E057
:10F9900087709070FC012E9FC0012F9F900D3E9F9D
:10F9A000900D1124B3E096958795BA95E1F7481B21
:10F9B000590B44365105A8F4E0EEF2E007C08091FF
:10F9C000C00085FFFCCF31969093C60090819923AB
:10F9D000B1F780ED98E04AE050E00E947F5344E6A2
:10F9E00050E0509379104093781080916D1080937F
:10F9F0007A1010927B10E0913410F091351064ADC4
:10FA000075AD7093731060937210FCE961347F07D9
:10FA100018F060E47CE904C02EE46132720730F033
:10FA2000769567957695679584E007C037E26131F2
:10FA3000730730F07695679582E080936D1008C06B
:10FA400081E080936D106032710510F460E270E027
:10FA50006052704048E060307407E8F0472F50E093
:10FA6000440F551F440F551F4950534F9A012E5FA5
:10FA70003F4FF901859194919C01AA27639FC00192
:10FA8000629F810D9A1F06948A1F9A1F1124FA0102
:10FA9000459154911EC0CB01969587958C7F8950D6
:10FAA0009F4EFC0145915491FC0132962591349171
:10FAB000862F90E087709070FC012E9FC0012F9FD1
:10FAC000900D3E9F900D112433E0969587953A95C1
:10FAD000E1F7481B590B44365105A8F4E0EEF2E07B
:10FAE00007C08091C00085FFFCCF31969093C6007F
:10FAF00090819923B1F780ED98E04AE050E00E94B0
:10FB00007F5344E650E0CA01A0E0B0E080936E105D
:10FB100090936F10A0937010B09371105093890060
:10FB200040938800E0913410F091351080899189DC
:10FB3000A289B389B695A79597958795B095A09515
:10FB4000909581959F4FAF4FBF4F809352109093E8
:10FB50005310A0935410B093551080935610909367
:10FB60005710A0935810B093591080935A10909347
:10FB70005B10A0935C10B0935D1080935E10909327
:10FB80005F10A0936010B0936110109262101092F9
:10FB90006310109264101092651006C080ED97E01B
:10FBA0009093890080938800C0913410D0913510D3
:10FBB000209709F489C488A18093661080FF03C050
:10FBC000119A8FEF02C0119881E080938803809191
:10FBD000661081FF03C044988FEF02C0449A81E011
:10FBE000809389038091661080FF36C080918C03DA
:10FBF000882391F120B1217031E0232759F18091C0
:10FC00006710882339F188819981AA81BB811816F0
:10FC100019061A061B06F4F48091421090914310C5
:10FC2000A0914410B09145108093361090933710F6
:10FC3000A0933810B093391030936810888999894F
:10FC4000AA89BB898093621090936310A09364107B
:10FC5000B0936510209367108091661081FD3AC0C3
:10FC600080918C038823B1F180B182958F7080954B
:10FC7000282F217080FF2CC080916910882341F1CA
:10FC80008C819D81AE81BF81181619061A061B064C
:10FC9000FCF48091461090914710A0914810B091CB
:10FCA000491080933A1090933B10A0933C10B0936E
:10FCB0003D1081E080936A1088899989AA89BB895F
:10FCC0008093621090936310A0936410B0936510BA
:10FCD000209369108091661082FF05C0419A8FEFD2
:10FCE00080938A0339C0419881E080938A03809190
:10FCF0008C03882389F120E007992CC021E08091B2
:10FD00006B10882339F188859985AA85BB851816DB
:10FD100019061A061B06F4F480914A1090914B10B4
:10FD2000A0914C10B0914D1080933E1090933F10D5
:10FD3000A0934010B093411020936C10888999894A
:10FD4000AA89BB898093621090936310A09364107A
:10FD5000B093651020936B108091661083FF0AC0EA
:10FD60008FB7F89490910B019F7B90930B018FBFFD
:10FD70008FEF09C08FB7F89490910B019064909326
:10FD80000B018FBF81E080938B0360E070E079C14D
:10FD90008091C00087FF19C04091C600E091CC0857
:10FDA000F091CD0831969F012F7730703197809177
:10FDB000CE089091CF082817390739F0E45BF74F48
:10FDC00040833093CD082093CC08288139814A8123
:10FDD0005B818091521090915310A0915410B0917A
:10FDE0005510280F391F4A1F5B1F20935210309364
:10FDF00053104093541050935510121613061406C6
:10FE000015066CF5139A88899989AA89BB89281BDC
:10FE1000390B4A0B5B0B20935210309353104093D5
:10FE2000541050935510209142103091431040913E
:10FE300044105091451080918803992787FD909533
:10FE4000A92FB92F820F931FA41FB51F80934210B3
:10FE500090934310A0934410B093451013982C81B5
:10FE60003D814E815F818091561090915710A091F5
:10FE70005810B0915910280F391F4A1F5B1F20934B
:10FE80005610309357104093581050935910121633
:10FE90001306140615066CF5459A88899989AA896E
:10FEA000BB89281B390B4A0B5B0B209356103093F0
:10FEB000571040935810509359102091461030918C
:10FEC000471040914810509149108091890399271B
:10FED00087FD9095A92FB92F820F931FA41FB51FDF
:10FEE0008093461090934710A0934810B093491008
:10FEF0004598288539854A855B8580915A1090916F
:10FF00005B10A0915C10B0915D10280F391F4A1F43
:10FF10005B1F20935A1030935B1040935C105093FA
:10FF20005D1012161306140615066CF5429A8889A0
:10FF30009989AA89BB89281B390B4A0B5B0B209333
:10FF40005A1030935B1040935C1050935D102091D9
:10FF50004A1030914B1040914C1050914D108091AF
:10FF60008A03992787FD9095A92FB92F820F931F98
:10FF7000A41FB51F80934A1090934B10A0934C1070
:10FF8000B0934D1042982C853D854E855F858091BC
:10FF90005E1090915F10A0916010B0916110280FD9
:10FFA000391F4A1F5B1F20935E1030935F104093F0
:10FFB0006010509361101216130614061506DCF536
:10FFC0009FB7F89480910B01806880930B019FBFCD
:10FFD00088899989AA89BB89281B390B4A0B5B0B35
:10FFE00020935E1030935F10409360105093611027
:10FFF00020914E1030914F1040915010509151105F
:020000021000EC
:1000000080918B03992787FD9095A92FB92F820F97
:10001000931FA41FB51F80934E1090934F10A09371
:100020005010B09351109FB7F89480910B018F77C7
:1000300080930B019FBF8091621090916310A091FB
:100040006410B09165100196A11DB11D80936210DE
:1000500090936310A0936410B09365102091621088
:100060003091631040916410509165106F5F7F4F25
:1000700088899989AA89BB89281739074A075B07A4
:1000800038F480916D1090E0681779070CF480CEF9
:10009000209162103091631040916410509165106E
:1000A0008C899D89AE89BF8982179307A407B507FC
:1000B00008F4E3C0E0906E10F0906F1000917010A3
:1000C00010917110AC8CBD8CCE8CDF8CA801970187
:1000D000C601B501AA27279FB12D389FF001489F7F
:1000E000F00D479FE00DF11D289FB00DE11DFA1F97
:1000F000379FB00DE11DFA1F469FB00DE11DFA1F9D
:10010000369FB10DEA1FFA1FB695EA1FFA1F112498
:100110008CAD9DAD8E0F9F1F9093731080937210C6
:1001200028AD39AD4AAD5BADA0E0B0E02817390786
:100130004A075B0720F4309373102093721060918C
:100140007210709173108CE96134780718F060E4D4
:100150007CE904C09EE46132790730F076956795BA
:100160007695679584E007C0E7E261317E0730F05D
:100170007695679582E080936D1008C081E080934A
:100180006D106032710510F460E270E060527040F2
:10019000F8E060307F07E8F0472F50E0440F551F2C
:1001A000440F551F4950534F9A012E5F3F4FF9019D
:1001B000859194919C01AA27639FC001629F810D44
:1001C0009A1F06948A1F9A1F1124FA01459154918F
:1001D0001EC0CB01969587958C7F89509F4EFC0160
:1001E00045915491FC01329625913491862F90E0EF
:1001F00087709070FC012E9FC0012F9F900D3E9F35
:10020000900D1124B3E096958795BA95E1F7481BB8
:10021000590B44365105A8F4E0EEF2E007C0809196
:10022000C00085FFFCCF31969093C6009081992342
:10023000B1F780ED98E04AE050E00E947F5344E639
:1002400050E050938900409388009A0140E050E0CC
:1002500080916E1090916F10A0917010B0917110FC
:10026000820F931FA41FB51F80936E1090936F1081
:10027000A0937010B093711002C120916210309160
:1002800063104091641050916510888D998DAA8DEE
:10029000BB8D82179307A407B50708F0E4C06091EF
:1002A00074107091751080917610909177102C8D4C
:1002B0003D8D4E8D5F8DAA27639FB12D749FF001F8
:1002C000849FF00D839FE00DF11D649FB00DE11D33
:1002D000FA1F739FB00DE11DFA1F829FB00DE11D43
:1002E000FA1F729FB10DEA1FFA1FB695EA1FFA1F97
:1002F000112480917210909173108E179F0738F41B
:10030000C05CDF4F68817981C054D04003C0BC011C
:100310006E1B7F0BC05CDF4F288139814A815B8176
:10032000CB01A0E0B0E082179307A407B50708F45B
:10033000B901FCE961347F0718F060E47CE904C08E
:100340002EE46132720730F0769567957695679561
:1003500084E007C037E26131730730F07695679526
:1003600082E080936D1008C081E080936D10603250
:10037000710510F460E270E06052704048E0603057
:100380007407E8F0472F50E0440F551F440F551FE6
:100390004950534F9A012E5F3F4FF9018591949137
:1003A0009C01AA27639FC001629F810D9A1F06943A
:1003B0008A1F9A1F1124FA01459154911EC0CB0146
:1003C000969587958C7F89509F4EFC01459154915D
:1003D000FC01329625913491862F90E087709070C1
:1003E000FC012E9FC0012F9F900D3E9F900D112468
:1003F00023E0969587952A95E1F7481B590B4436DB
:100400005105A8F4E0EEF2E007C08091C00085FF3E
:10041000FCCF31969093C60090819923B1F780ED7F
:1004200098E04AE050E00E947F5344E650E0509349
:100430008900409388009A0140E050E08091741058
:1004400090917510A0917610B0917710820F931F44
:10045000A41FB51F8093741090937510A09376100D
:10046000B09377100CC08091781090917910909390
:1004700089008093880080917A1080936D1020917C
:100480006210309163104091641050916510E091BA
:100490003410F091351080899189A289B389281789
:1004A00039074A075B0780F010923510109234101C
:1004B0009091110E8091120E981731F08091120ECA
:1004C0008F5F8F708093120EFF91EF91DF91CF912C
:1004D000BF91AF919F918F917F916F915F914F915C
:1004E0003F912F911F910F91FF90EF90DF90CF9050
:1004F000BF90AF900F900BBE0F900FBE0F901F904C
:10050000189580916810882349F480916A10882397
:1005100029F480916C10882309F490C0E7EFF4E18E
:10052000949108C08091C00085FFFCCF9093C600D5
:10053000319694919923B1F7E9E0F5E1949108C0DF
:100540008091C00085FFFCCF9093C60031969491B6
:100550009923B1F7809168108823D1F0609136100B
:100560007091371080913810909139100E94EBCE25
:100570002091E5083091E6084091E7085091E8089D
:100580000E9450CEAB01BC0185E095E10E94013490
:1005900080916A108823D1F060913A1070913B10DD
:1005A00080913C1090913D100E94EBCE2091E90883
:1005B0003091EA084091EB085091EC080E9450CE2F
:1005C000AB01BC0181E095E10E94013480916C1087
:1005D0008823D1F060913E1070913F1080914010BF
:1005E000909141100E94EBCE2091ED083091EE08E1
:1005F0004091EF085091F0080E9450CEAB01BC0131
:100600008DEF94E10E940134E4EFF2E007C08091A5
:10061000C00085FFFCCF31969093C600908199234E
:10062000B1F78091C00085FFFCCF8AE08093C600BF
:100630001092681010926A1010926C10089560E089
:1006400070E08FE793E42091910330919203409101
:100650009303509194030E9450CE6093A81070931E
:10066000A9108093AA109093AB1060E070E08FE720
:1006700093E42091A1033091A2034091A3035091F0
:10068000A4030E9450CE6093B0107093B110809379
:10069000B2109093B3100895FC0197FF03C08091AE
:1006A0008D1003C0E457FF4E808190E008952F9293
:1006B0003F924F925F926F927F928F929F92AF92F2
:1006C000BF92CF92DF92EF92FF920F931F93CF933F
:1006D000DF93EC0121E030E0A901440F551F440FE6
:1006E000551FFA01E053FA4E85919491C817D90726
:1006F0000CF059C0B90161507040660F771F660F4A
:10070000771FCB018E529A4EFC01059114916053D4
:100710007A4EFB01C590D490FA01EE52FA4EE59064
:10072000F490FA01E053FA4EA590B490B8018827EE
:1007300077FD8095982F0E94EBCE1B012C01CC19E0
:10074000DD09BE01882777FD8095982F0E94EBCEAA
:100750003B014C01E01AF10A0027F7FC0095102F2D
:10076000C801B7010E94EBCE9B01AC01C401B301EB
:100770000E941ED17B018C01AC18BD08CC24B7FCB3
:10078000C094DC2CC601B5010E94EBCE9B01AC01EC
:10079000C801B7010E9450CE9B01AC01C201B1015A
:1007A0000E9470CD19C0822F8F5F2F5F3F4F213382
:1007B000310509F091CF813329F0E0E070E080E06D
:1007C00060E00CC0E2E9F6E165917491882777FD5D
:1007D0008095982F0E94EBCEE62F692F2E2F372F72
:1007E000482F562FB901CA01DF91CF911F910F9168
:1007F000FF90EF90DF90CF90BF90AF909F908F9041
:100800007F906F905F904F903F902F900895089544
:1008100010927D1010927C1010928C10749810928F
:100820007F1010927E1010928D10A59808952DEBD8
:1008300037E346E05EE30C941ED12DEB37E346E050
:100840005EE30C9450CE2DEB37E346E05EE30C9470
:1008500050CE2DEB37E346E05EE30C941ED1A59815
:100860000E94C52F882319F5E8E1F5E1949108C0AD
:100870008091C00085FFFCCF9093C6003196949183
:100880009923B1F7EFE1F5E1949108C08091C000A0
:1008900085FFFCCF9093C600319694919923B1F7D0
:1008A0008091C00085FFFCCF8AE08093C60083E082
:1008B0000C9401301F93182FABDF0E94C52F8823A3
:1008C00091F5E8E1F5E1949108C08091C00085FFC1
:1008D000FCCF9093C600319694919923B1F780EDA7
:1008E00098E0612F70E04AE050E00E9458538091F8
:1008F000C00085FFFCCF8AE08093C600E9E5F5E102
:10090000949108C08091C00085FFFCCF9093C600F1
:10091000319694919923B1F78091C00085FFFCCF67
:100920008AE08093C60082E00E9401301F91089502
:100930001F93182F6DDF0E94C52F882391F5E8E1E2
:10094000F5E1949108C08091C00085FFFCCF9093A1
:10095000C600319694919923B1F780ED98E0612F0C
:1009600070E04AE050E00E9458538091C00085FF3B
:10097000FCCF8AE08093C600E6E8F5E1949108C0D8
:100980008091C00085FFFCCF9093C6003196949172
:100990009923B1F78091C00085FFFCCF8AE0809356
:1009A000C60081E00E9401301F9108951F920F92AE
:1009B0000FB60F920BB60F9211242F933F934F93C4
:1009C0005F936F937F938F939F93AF93BF93EF93B7
:1009D000FF939091AD03992361F480918C108093E3
:1009E00092108111749A80918D10809391108111D1
:1009F000A59A80919210981708F0749880919110A0
:100A0000981708F0A5989F5F9F779093AD0380910A
:100A1000AE03843009F471C0853050F4813021F187
:100A2000813098F08230F1F1833009F07AC049C00A
:100A3000863009F468C0863008F463C0873009F452
:100A400066C0883009F06DC06AC088E080937B0082
:100A500080E480937C0080917A00806480937A00A7
:100A60000E94358F81E01BC08091780090917900C1
:100A7000A0E0B0E020919F103091A0104091A11013
:100A80005091A210280F391F4A1F5B1F20939F10FF
:100A90003093A0104093A1105093A21082E0809355
:100AA000AE033FC088E080937B0082E480937C00AB
:100AB00080917A00806480937A000E94358F83E071
:100AC000EECF8091780090917900A0E0B0E0209185
:100AD0009310309194104091951050919610280FDA
:100AE000391F4A1F5B1F209393103093941040933B
:100AF00095105093961084E0D2CF0E94358F85E0F8
:100B0000CECF86E0CCCF0E94358F87E0C8CF109241
:100B1000AE038091A3108F5F8093A31002C0109248
:100B2000AE038091A310803108F463C080918E10D1
:100B3000882381F480919F109091A0109093811050
:100B400080938010809193109091941090938710CF
:100B50008093861081E080938E101092A3101092E3
:100B60009F101092A0101092A1101092A21010923B
:100B70009B1010929C1010929D1010929E1010923B
:100B80009710109298101092991010929A1010923B
:100B9000931010929410109295101092961020912C
:100BA0008010309181108091A9039091AA03281799
:100BB000390714F080E0BCDE209180103091811064
:100BC00080918F10909190108217930714F080E01D
:100BD00071DE20918610309187108091AB03909147
:100BE000AC03281739072CF010927F1010927E105A
:100BF00036DEFF91EF91BF91AF919F918F917F91E1
:100C00006F915F914F913F912F910F900BBE0F907D
:100C10000FBE0F901F9018952F926F927F928F9218
:100C20009F92AF92BF92CF92DF92EF92FF920F937B
:100C30001F93DF93CF93CDB7DEB729970FB6F89404
:100C4000DEBF0FBECDBF8C01E62E662369F1E8E161
:100C5000F5E1949108C08091C00085FFFCCF90938E
:100C6000C600319694919923B1F780ED98E06E2DEE
:100C700070E04AE050E00E945853E3EBF5E19491B4
:100C800008C08091C00085FFFCCF9093C6003196CC
:100C900094919923B1F78091C00085FFFCCF8AE041
:100CA0008093C6000E944130AE2DB0E0FD01EE0FF2
:100CB000FF1FEF5CFB4F6081718179876887672B2D
:100CC00009F49FC0AD5CBB4F7C917B8322242394AD
:100CD00079C0222D30E0A901440F551F440F551F44
:100CE000E885F985E40FF51F859194910817190798
:100CF0000CF067C0C9010197880F991F880F991FD1
:100D0000FC013296A885B985EA0FFB1FC590D490E7
:100D10008A0F9B1FFC01659174917A836983FA01A4
:100D20003296EA0FFB1FE590F490FD01E40FF51FEA
:100D3000A590B490B601882777FD8095982F0E94E2
:100D4000EBCE6C837D838E839F8389819A81081B80
:100D5000190BB801882777FD8095982F0E94EBCE5C
:100D60003B014C01EC18FD080027F7FC0095102F03
:100D7000C801B7010E94EBCE9B01AC01C401B301D5
:100D80000E941ED17B018C01A981BA81AA1ABB0ADB
:100D9000CC24B7FCC094DC2CC601B5010E94EBCE7C
:100DA0009B01AC01C801B7010E9450CE9B01AC0170
:100DB0006C817D818E819F810E9470CDE62F692F8D
:100DC00009C02394BB812B1608F483CFE0E070E0C8
:100DD00080E060E0FB812F1679F5E22DF0E0EE0F68
:100DE000FF1FEE0FFF1F329768857985E60FF71F0B
:100DF00065917491882777FD8095982F0E94EBCE9E
:100E000019C0B801882777FD8095982F0E94EBCEF6
:100E100020E030E04AEF5EE30E941ED120E030E0A7
:100E200040E85DE30E941ED120E030E040E050E069
:100E30000E9470CDE62F692F2E2F372F482F562F67
:100E4000B901CA0129960FB6F894DEBF0FBECDBF17
:100E5000CF91DF911F910F91FF90EF90DF90CF9096
:100E6000BF90AF909F908F907F906F902F9008953C
:100E7000EF92FF920F931F93CF93DF930F2EF0E02B
:100E8000EF2EF0E0FF2EF0E00F2FF0E01F2FF02DFF
:100E9000E092A410F092A5100093A6101093A71052
:100EA00060E070E08FE793E420919103309192032A
:100EB00040919303509194030E9450CE6093A810E8
:100EC0007093A9108093AA109093AB10E092AC108D
:100ED000F092AD100093AE101093AF1060E070E090
:100EE0008FE793E42091A1033091A2034091A303E3
:100EF0005091A4030E9450CE6093B0107093B11033
:100F00008093B2109093B3106C9A6D9A9D9A8091D1
:100F1000010180618093010187ED80937A00109236
:100F20007E0010927D0080917D00816080937D0025
:100F300080917D00826080937D0080917D0084603F
:100F400080937D0080E888BD80916E0084608093EE
:100F50006E0085E090E09093B5108093B41009C0C6
:100F600080918F1090919010409690939010809364
:100F70008F1080918F109091901060E04DDE20E0F6
:100F800030E040EA50E40E9449CE87FDE9CF83E19A
:100F900091E09093B0038093AF0309C08091A903BF
:100FA0009091AA0340979093AA038093A9038091FC
:100FB000A9039091AA0360E02FDE20E030E849E821
:100FC00053E40E944CD018164CF3C091AB03D0915F
:100FD000AC03EC2E1D2FCE016ADB609720E030E0E1
:100FE00048E453E40E944CD018169CF3E092AB0303
:100FF0001093AC03DF91CF911F910F91FF90EF9071
:101000000895809180109091811060E005DE6093DA
:101010008210709383108093841090938510809138
:1010200086109091871043DB60938810709389102D
:1010300080938A1090938B100E9496C98FB7F89472
:1010400010928E108FBF08952F923F924F925F9211
:101050006F927F928F929F92AF92BF92CF92DF92C8
:10106000EF92FF920F931F9380918E10882309F4C3
:101070006EC2C7DF609082107090831080908410E1
:1010800090908510C0907C10D0907D10B60188277C
:1010900077FD8095982F0E94EBCEA40193010E94CA
:1010A0006FCD7B018C016093B6107093B710809365
:1010B000B8109093B91020E030E04AE754E40E9461
:1010C0004CD0181624F481E08093BA10E9C0C8010E
:1010D000B70120E030E04AE754EC0E9449CE87FD9A
:1010E00002C0CD2821F481E08093BA10C4C0809161
:1010F000BA10882371F080E090E0A0E0B0E0809327
:10110000BB109093BC10A093BD10B093BE10109272
:10111000BA10C801B70120918D0330918E03409120
:101120008F03509190030E941ED11B012C016093EC
:10113000BF107093C0108093C1109093C210C8016B
:10114000B7012091BB103091BC104091BD1050915F
:10115000BE100E9470CD5B016C01E090A410F09075
:10116000A5100091A6101091A710A80197010E9448
:1011700049CE87FD12C0E090A810F090A910009110
:10118000AA101091AB10C601B501A80197010E94E9
:101190004CD0181614F086017501E092BB10F09245
:1011A000BC100093BD101093BE10C801B701209170
:1011B00091033091920340919303509194030E94C4
:1011C0001ED15B016C016093C3107093C4108093B7
:1011D000C5109093C610C401B3012091C71030917F
:1011E000C8104091C9105091CA100E946FCD209133
:1011F00095033091960340919703509198030E9474
:101200001ED120E037ED43E25CE30E941ED17B015A
:101210008C016091CB107091CC108091CD10909189
:10122000CE1024EA30E74DE75FE30E941ED19B0118
:10123000AC01C801B7010E9470CD7B018C016093A5
:10124000CB107093CC108093CD109093CE10C20130
:10125000B101A60195010E9470CDA80197010E94DD
:101260006FCD7B018C0120E030E040E050E00E9437
:1012700049CE88235CF40F2EF0E0EF2EF0E0FF2E35
:10128000F0E00F2FF0E01F2FF02D14C0C801B701C0
:1012900020E030E04FE753E40E944CD0181654F49D
:1012A0000F2EF0E0EF2EF0E0FF2EFFE70F2FF3E41C
:1012B0001F2FF02D6092C7107092C8108092C91035
:1012C0009092CA106091B4107091B510882777FD84
:1012D0008095982F0E94EBCE9B01AC01C401B30115
:1012E0000E944CD01816DCF46091AF037091B003EB
:1012F000882777FD8095982F0E94EBCE9B01AC014B
:10130000C401B3010E9449CE88234CF4C801B7013F
:101310000E94B8CE7595679560938C1002C01092AC
:101320008C10609088107090891080908A10909036
:101330008B1060917E1070917F10882777FD8095CB
:10134000982F0E94EBCEA40193010E946FCD7B01E8
:101350008C016093CF107093D0108093D110909334
:10136000D21020919D0330919E0340919F03509194
:10137000A0030E941ED11B012C016093D310709317
:10138000D4108093D5109093D610C801B701209146
:10139000D7103091D8104091D9105091DA100E9496
:1013A00070CD5B016C01E090AC10F090AD1000913D
:1013B000AE101091AF10A80197010E9449CE87FD91
:1013C00012C0E090B010F090B1100091B2101091E6
:1013D000B310C601B501A80197010E944CD01816A0
:1013E00014F086017501E092D710F092D8100093A6
:1013F000D9101093DA10C801B7012091A1033091E0
:10140000A2034091A3035091A4030E941ED15B014B
:101410006C016093DB107093DC108093DD1090936F
:10142000DE10C401B3012091DF103091E010409133
:10143000E1105091E2100E946FCD2091A5033091F0
:10144000A6034091A7035091A8030E941ED120E05B
:1014500037ED43E25CE30E941ED17B018C01609179
:10146000E3107091E4108091E5109091E61024EA69
:1014700030E74DE75FE30E941ED19B01AC01C8013C
:10148000B7010E9470CD7B018C016093E3107093D3
:10149000E4108093E5109093E6106092DF10709254
:1014A000E0108092E1109092E210C201B101A60119
:1014B00095010E9470CDA80197010E946FCD7B011C
:1014C0008C0120E030E040E050E00E9449CE8823CB
:1014D0005CF40F2EF0E0EF2EF0E0FF2EF0E00F2F87
:1014E000F0E01F2FF02D14C0C801B70120E030E05C
:1014F0004FE753E40E944CD0181654F40F2EF0E03E
:10150000EF2EF0E0FF2EFFE70F2FF3E41F2FF02D5B
:10151000C401B30120E030E040EA50E40E944CD026
:1015200018169CF4C401B30120E030E048E453E411
:101530000E9449CE88234CF4C801B7010E94B8CE5E
:101540007595679560938D1002C010928D101F9154
:101550000F91FF90EF90DF90CF90BF90AF909F9052
:101560008F907F906F905F904F903F902F90089555
:101570002F923F924F925F926F927F928F929F92A3
:10158000AF92BF92CF92DF92EF92FF920F931F9391
:10159000DF93CF93CDB7DEB7E6970FB6F894DEBFF3
:1015A0000FBECDBF6C8F7D8F8E8F9F8F5EAB4DAB8F
:1015B00039A328A30E94171A698B7A8B8B8B9C8B7B
:1015C0002DA93EA9223031051CF4E5EFF2E019C047
:1015D000E8E0F3E007C08091C00085FFFCCF3196C2
:1015E0009093C60090819923B1F78091C00085FF48
:1015F000FCCF12C48091C00085FFFCCF3196909340
:10160000C60090819923B1F78091C00085FFFCCF7F
:101610008AE08093C600FCD84DA95EA957FF74C02C
:101620008FE780938D1089899A89AB89BC898D87D2
:101630009E87AF87B88B89879A87AB87BC8719AAA3
:101640001AAA1BAA1CAA1F8A1E8A91E09D8B1D82C2
:101650001E821F8218869FE7A92EB12CC12CD12C87
:101660008FE7282E312C412C512C20E030E040E037
:1016700050E029833A834B835C830F2EF0E06F2E7A
:10168000F0E47F2EFCE18F2EF6E49F2EF02D4DA985
:101690005EA944575F4E5BA34AA3E5E7F7E1549187
:1016A0005CA3E0E7F7E184918DA3E9E6F7E194918B
:1016B0009EA3E2E6F7E1A491AFA3ECE5F7E1B491D4
:1016C000B8A7E6E5F7E1249129A7E9E4F7E1349129
:1016D0003AA7E3E4F7E144914BA7EDE3F7E1549136
:1016E0005CA7E7E3F7E184918DA7ADA9BEA9AA0F96
:1016F000BB1FAA0FBB1FAE57BF4EBFA7AEA7EDEFD4
:10170000F6E1B491B8AB07C0EDA9FEA9E457FF4ECE
:101710008FE7808388CF80918E10882309F4A2C23E
:1017200070DCEDA9FEA9F7FF0DC0F0918810F9ABB0
:10173000209189102AAB30918A103BAB40918B10DD
:101740004CAB11C0AEA5BFA5BC91B9ABEEA5FFA532
:10175000F181FAABAEA5BFA51296BC91BBABEEA5CD
:10176000FFA5F381FCAB69817A818B819C8129A9DA
:101770003AA94BA95CA90E944CD0181644F089A93B
:101780009AA9ABA9BCA989839A83AB83BC83C40102
:10179000B30129A93AA94BA95CA90E9449CE87FDAA
:1017A00006C089A99AA9ABA9BCA93C014D012D8904
:1017B000222309F451C069A97AA98BA99CA92C8D6F
:1017C0003D8D4E8D5F8D0E944CD018160CF04AC294
:1017D0000E94171A29853A854B855C85621B730B1D
:1017E000840B950B695873418040904008F43AC2CD
:1017F000D601C50182199309A409B5094DA95EA9AD
:1018000057FF07C0B595A7959795879580938D103D
:1018100007C0B595A79597958795EAA1FBA1808309
:101820000E94171A6D877E878F87988B9B01AC016A
:1018300089859A85AB85BC85281B390B4A0B5B0BC8
:101840002D833E834F8358872C8D3D8D4E8D5F8D2C
:1018500029833A834B835C8369A97AA98BA99CA9C4
:101860002C8D3D8D4E8D5F8D0E9449CE88230CF0CE
:10187000F8C10E94171A2D853E854F855889621B35
:10188000730B840B950B695873418040904008F4AA
:10189000E8C10E94171A69877A878B879C874E89CF
:1018A0005F89452B09F4B8C1DC01CB012D853E854C
:1018B0004F855889821B930BA40BB50B2D813E815C
:1018C0004F815885280F391F4A1F5B1F288F398F7A
:1018D0004A8F5B8F2D813E814F815885281B390BA4
:1018E0004A0B5B0BCA01B901A20191010E94C1D44C
:1018F000288D398D4A8D5B8D0E9435D52A0D3B1D73
:101900004C1D5D1D24313105410551055CF4E4E1B8
:101910002E2E312C412C512C74E1A72EB12CC12C30
:10192000D12C1FC059016A013CEEA316B104C104B9
:10193000D1042CF06BEEA62EB12CC12CD12C40E89A
:10194000A416B104C104D1041CF41501260109C078
:101950005EEF252E312C412C512C2A183B084C08C7
:101960005D089CA1E5E7F7E108C08091C00085FF14
:10197000FCCF9093C600319694919923B1F780EDF6
:1019800098E0B601A5012AE030E00E9425539DA110
:10199000E0E7F7E108C08091C00085FFFCCF90939D
:1019A000C600319694919923B1F780ED98E0B20189
:1019B000A1012AE030E00E9425539EA1E9E6F7E16B
:1019C00008C08091C00085FFFCCF9093C60031967F
:1019D00094919923B1F780ED98E0B401A30122E03E
:1019E00030E00E942B549FA1E2E6F7E108C080910D
:1019F000C00085FFFCCF9093C60031969491992347
:101A0000B1F780ED98E049815A816B817C8122E0B9
:101A100030E00E942B548091C00085FFFCCF8AE00B
:101A20008093C6008E899F8903970CF4F5C0C2018C
:101A3000B1010E94EBCE20E030E040E850E40E948B
:101A40001ED17B018C0169817A818B819C81A401EB
:101A500093010E946FCD20ED3FE049E450E40E94E5
:101A60001ED120E030E040E05FE30E941ED19B01E8
:101A7000AC01C801B7010E9450CE7B018C01688D7A
:101A8000798D8A8D9B8D0E94EBCE20E030E04AE775
:101A900054E40E9450CE3B014C0198A5ECE5F7E1DF
:101AA00008C08091C00085FFFCCF9093C60031969E
:101AB00094919923B1F780ED98E0B801A70122E055
:101AC00030E00E942B5499A5E6E5F7E108C080912B
:101AD000C00085FFFCCF9093C60031969491992366
:101AE000B1F780ED98E0B401A30122E030E00E945C
:101AF0002B548091C00085FFFCCF8AE08093C60004
:101B0000C801B7012AE939E949E15FE30E941ED122
:101B10007B018C019AA5E9E4F7E108C08091C0003F
:101B200085FFFCCF9093C600319694919923B1F72D
:101B30008091C00085FFFCCF8AE08093C6009BA502
:101B4000E3E4F7E108C08091C00085FFFCCF9093EB
:101B5000C600319694919923B1F780ED98E0B801D1
:101B6000A70122E030E00E942B548091C00085FF45
:101B7000FCCF8AE08093C6009CA5EDE3F7E108C0A6
:101B80008091C00085FFFCCF9093C6003196949160
:101B90009923B1F7C801B701A80197010E9470CD40
:101BA000A40193010E9450CEAB01BC0180ED98E0EE
:101BB00022E030E00E942B548091C00085FFFCCFD2
:101BC0008AE08093C6009DA5E7E3F7E108C0809115
:101BD000C00085FFFCCF9093C60031969491992365
:101BE000B1F7C801B701A40193010E941ED120E002
:101BF00030E040E05EE30E941ED1AB01BC0180ED0D
:101C000098E022E030E00E942B548091C00085FFD4
